:100000000C94970F0C94C80F0C94C80F0C94C80F45
:100010000C94C80F0C94C80F0C94C80F0C94C80F04
:100020000C94C80F0C94C80F0C94C80F0C94C80FF4
:100030000C94C80F0C94FEB00C94C80F0C94C80F0D
:100040000C94C80F0C947E8F0C94C80F0C94C80F9E
:100050000C94C80F0C94C80F0C94AB260C94C4AC31
:100060000C94C80F0C94898C0C94C80F0C94C80F76
:100070000C94C80F0C94C80F0C94C80F0C94C80FA4
:100080000C94C80F0C94C80F0C94C80F0C94C80F94
:100090000C94C80F0C94C80F0C94C80F0C94F6A9BC
:1000A0000C94C80F0C94C80F0C94C80F0C94C80F74
:1000B0000C94C80F0C94C80F0C94C80F0C94C80F64
:1000C0000C94C80F0C94C80F0C94C80F0C94C80F54
:1000D0000C94C80F0C94C80F0C94C80F0C94C80F44
:1000E0000C94C80FF8260627222730274A275827BE
:1000F0007227762778277C27842748AB4DAB52ABF5
:100100005CABD5AB66AB6EAB76AB80AB8AAB94AB7E
:10011000A3ABADABD5ABB7ABC1ABCBABF3ABF6AB36
:10012000E9ABEDAB2DACFAABFEAB04AC08AC0CAC60
:1001300012AC16AC1AAC2DAC20AC24AC28AC084ADE
:10014000D73B3BCE016E84BCBFFDC12F3D6C7431EB
:100150009ABD56833DDA3D00C77F11BED9E4BB4C42
:100160003E916BAAAABE000000803F05A84CCDB20C
:10017000D44EB93836A9020C50B9918688083CA6ED
:10018000AAAA2ABE000000803F007C3C3E5E2B3DB8
:100190003F2F5B5D3B2C2A225C004572723A204D5A
:1001A000415854454D50204245440054656D70659A
:1001B000726174757265206865617465642062653A
:1001C00064207377697463686564206F66662E20A7
:1001D0004D415854454D502074726967676572658A
:1001E00064202121004572723A204D494E54454DFC
:1001F00050003A204578747275646572207377698F
:100200007463686564206F66662E204D494E5445C0
:100210004D502074726967676572656420210045DE
:1002200072723A204D415854454D50003A2045785D
:10023000747275646572207377697463686564208D
:100240006F66662E204D415854454D50207472699A
:10025000676765726564202100202D20496E7661F4
:100260006C6964206578747275646572206E756D52
:10027000626572202100504944204175746F747585
:100280006E652066696E69736865642120507574B7
:1002900020746865206C617374204B702C204B694E
:1002A00020616E64204B6420636F6E7374616E74A2
:1002B000732066726F6D2061626F766520696E745F
:1002C0006F20436F6E66696775726174696F6E2E19
:1002D0006800504944204175746F74756E652066DE
:1002E00061696C6564212074696D656F75740020A7
:1002F000403A006F6B20543A006F6B20423A005036
:100300004944204175746F74756E65206661696C2F
:100310006564212054656D70657261747572652025
:10032000746F6F206869676800204B643A20002072
:100330004B693A2000204B703A200020436C6173D7
:100340007369632050494420002054753A200020EE
:100350004B753A2000206D61783A2000206D696E5F
:100360003A200020643A200020626961733A20003C
:100370001000C90210012C01400122017001180176
:10038000B0010E01F00104015002FA00B002F000C9
:100390003003E600D003DC009004D2007005C800F2
:1003A000A006BE000008B400B009AA00D00BA0004F
:1003B000600E960060118C000015820020197800F4
:1003C000C01D6E00A0226400B0275A00902C50007F
:1003D00000314600E0343C0010383200903A2800EA
:1003E000603C1E00A03D1400803E0A00203F00003B
:1003F00070012C0190012701B0012201C0011D01F3
:10040000F00118011002130130020E01600209010F
:1004100090020401C002FF000003FA004003F5004F
:100420008003F000D003EB002004E6007004E1003C
:10043000E004DC004005D700C005D2004006CD0036
:10044000D006C8008007C3003008BE00F008B9001D
:10045000C009B400B00AAF00B00BAA00D00CA500D0
:10046000000EA000500F9B00C0109600501291008B
:1004700000148C00C0158700B0178200B0197D00F1
:10048000D01B7800001E730040206E00902269008F
:10049000F024640040275F0090295A00E02B5500AB
:1004A000102E500020304B0010324600E033410047
:1004B00090353C001037370070383200A0392D00DD
:1004C000B03A2800A03B2300603C1E00103D1900FC
:1004D000903D1400103E0F00703E0A00C03E050023
:1004E000003F00004D383420582059205A20450044
:1004F00043616E6E6F7420656E74657220737562F1
:100500006469723A20004D3234004D323320257335
:10051000006175746F25692E67006572726F7220B5
:1005200077726974696E6720746F2066696C650004
:100530004E6F74207072696E74696E67000A002FC6
:10054000005344207072696E74696E67206279741A
:100550006520000A002E0044656C6574696F6E208A
:100560006661696C65642C2046696C653A200046BA
:10057000696C652064656C657465643A002E006F73
:1005800070656E206661696C65642C2046696C65D7
:100590003A200057726974696E6720746F2066692B
:1005A0006C653A20002E006F70656E206661696C84
:1005B00065642C2046696C653A20002E006F7065DA
:1005C0006E206661696C65642C2046696C653A2012
:1005D0000046696C652073656C6563746564002012
:1005E00053697A653A200046696C65206F70656EC4
:1005F00065643A20002E006F70656E206661696C3C
:1006000065642C2046696C653A20004E6F77206641
:10061000726573682066696C653A20004E6F7720BA
:10062000646F696E672066696C653A2000222070ED
:100630006F73002220706172656E743A2200535508
:1006400042524F5554494E452043414C4C20746111
:10065000726765743A2200747279696E6720746FEC
:100660002063616C6C207375622D67636F64652015
:1006700066696C6573207769746820746F6F206D8C
:10068000616E79206C6576656C732E204D41582023
:100690006C6576656C2069733A005344206361721F
:1006A00064206F6B006F70656E526F6F74206661AF
:1006B000696C656400766F6C756D652E696E697422
:1006C000206661696C656400534420696E6974201A
:1006D0006661696C0000002110422063308440A5EF
:1006E00050C660E770088129914AA16BB18CC1ADF9
:1006F000D1CEE1EFF13112100273325222B5529491
:1007000042F772D662399318837BB35AA3BDD39C48
:10071000C3FFF3DEE36224433420040114E664C71C
:1007200074A44485546AA54BB528850995EEE5CF98
:10073000F5ACC58DD55336722611163006D776F630
:10074000669556B4465BB77AA719973887DFF7FEE8
:10075000E79DD7BCC7C448E5588668A778400861BC
:100760001802282338CCC9EDD98EE9AFF948896938
:10077000990AA92BB9F55AD44AB77A966A711A50D0
:100780000A333A122AFDDBDCCBBFFB9EEB799B5888
:100790008B3BBB1AABA66C877CE44CC55C222C035C
:1007A0003C600C411CAEED8FFDECCDCDDD2AAD0BD8
:1007B000BD688D499D977EB66ED55EF44E133E3270
:1007C0002E511E700E9FFFBEEFDDDFFCCF1BBF3A28
:1007D000AF599F788F8891A981CAB1EBA10CD12D17
:1007E000C14EF16FE18010A100C230E3200450251A
:1007F0004046706760B9839893FBA3DAB33DC31C8E
:10080000D37FE35EF3B1029012F322D23235421469
:100810005277625672EAB5CBA5A89589856EF54FD9
:10082000E52CD50DC5E234C324A0148104667447B9
:100830006424540544DBA7FAB79987B8975FE77E2D
:10084000F71DC73CD7D326F2369106B01657667609
:1008500076154634564CD96DC90EF92FE9C899E979
:10086000898AB9ABA94458654806782768C018E159
:10087000088238A3287DCB5CDB3FEB1EFBF98BD8CD
:100880009BBBAB9ABB754A545A376A167AF10AD0A9
:100890001AB32A923A2EFD0FED6CDD4DCDAABD8B19
:1008A000ADE89DC98D267C076C645C454CA23C83F9
:1008B0002CE01CC10C1FEF3EFF5DCF7CDF9BAFBA6D
:1008C000BFD98FF89F176E367E554E745E932EB249
:1008D0003ED10EF01E53544F505045442E20005030
:1008E00072696E7465722073746F707065642064D1
:1008F000756520746F206572726F72732E20466961
:100900007820746865206572726F7220616E642051
:10091000757365204D39393920746F207265737491
:100920006172742E202854656D70657261747572E1
:10093000652069732072657365742E205365742079
:100940006974206166746572207265737461727473
:10095000696E6729004B494C4C45442E200050726B
:10096000696E7465722068616C7465642E206B69B1
:100970006C6C28292063616C6C656421006F6B00CE
:10098000526573656E643A20002200556E6B6E6F7F
:10099000776E20636F6D6D616E643A2022004D3278
:1009A000323020532569005A204F666673657420E3
:1009B0003A20007A5F6D61783A20007A5F6D696E47
:1009C0003A20005A204F6666736574005A204F66BD
:1009D00066736574206F6B002200556E6B6E6F77C7
:1009E0006E20636F6D6D616E643A2022007A5F6DD8
:1009F00061783A20007A5F6D696E3A2000795F6D08
:100A000061783A2000795F6D696E3A2000785F6DF9
:100A100061783A2000785F6D696E3A2000205A3A7A
:100A20000020593A0020436F756E7420583A200018
:100A300020453A00205A3A0020593A00583A0046D8
:100A400049524D574152455F4E414D453A4D6172B5
:100A50006C696E2056312E302E323B2053707269F5
:100A60006E7465722F6772626C206D617368757049
:100A700020666F722067656E36204649524D574199
:100A800052455F55524C3A68747470733A2F2F6711
:100A900069746875622E636F6D2F4D61726C696E3B
:100AA0004669726D776172652F4D61726C696E2057
:100AB00050524F544F434F4C5F56455253494F4E3F
:100AC0003A312E30204D414348494E455F545950EC
:100AD000453A507275736120693320455854525518
:100AE0004445525F434F554E543A31205555494481
:100AF0003A30303030303030302D303030302D30F2
:100B00003030302D303030302D30303030303030EB
:100B100030303030300A00507275736120693320F4
:100B20004F66662E005072757361206933207265BE
:100B30006164792E0042656420646F6E652E00202A
:100B4000423A0020453A00543A0042656420486524
:100B50006174696E672E0048656174696E67206410
:100B60006F6E652E0020573A0020453A00543A0037
:100B700048656174696E672E2E2E002042403A004F
:100B800020403A00202F003A00205400202F00205F
:100B9000423A00202F006F6B20543A002569206DE7
:100BA000696E2C2025692073656300456E6420669C
:100BB000696C65206C69737400426567696E2066B4
:100BC000696C65206C697374004E6F206D6F76657B
:100BD0002E005072757361206933207265616479EB
:100BE0002E00526573756D696E67207072696E7440
:100BF000005761697420666F7220757365722E2EBE
:100C00002E00536C6565702E2E2E00256920686FAE
:100C1000757273202569206D696E75746573004463
:100C20006F6E65207072696E74696E672066696C9C
:100C3000650053544F505045442E20005072696E49
:100C40007465722073746F707065642064756520BC
:100C5000746F206572726F72732E204669782074EB
:100C60006865206572726F7220616E6420757365AD
:100C7000204D39393920746F207265737461727434
:100C80002E202854656D70657261747572652069D7
:100C9000732072657365742E205365742069742007
:100CA00061667465722072657374617274696E67CF
:100CB00029004E6F204C696E65204E756D6265721D
:100CC000207769746820636865636B73756D2C2089
:100CD0004C617374204C696E653A20004E6F20435E
:100CE0006865636B73756D2077697468206C696ED5
:100CF00065206E756D6265722C204C617374204C9A
:100D0000696E653A2000636865636B73756D206D6D
:100D100069736D617463682C204C617374204C6935
:100D20006E653A20004C696E65204E756D62657285
:100D3000206973206E6F74204C617374204C696E4F
:100D400065204E756D6265722B312C204C61737479
:100D5000204C696E653A20004D31313000446F6E91
:100D60006520736176696E672066696C652E006F19
:100D70006B004D3239002020506C616E6E657242FE
:100D8000756666657242797465733A200020467212
:100D90006565204D656D6F72793A20004665622069
:100DA0002033203230313600436F6D70696C6564DA
:100DB0003A2000286E6F6E652C2064656661756C44
:100DC0007420636F6E6669672900207C204175740A
:100DD000686F723A2000466562202033203230313D
:100DE000362030393A35363A343100204C6173744C
:100DF00020557064617465643A2000312E302E32C3
:100E0000004D61726C696E0020536F667477617279
:100E10006520526573657400205761746368646F60
:100E200067205265736574002042726F776E206F81
:100E30007574205265736574002045787465726E10
:100E4000616C20526573657400506F7765725570E0
:100E5000007374617274002200656E717565696E4D
:100E6000672022002200656E717565696E67202219
:100E700000FFFFFF0000A0400000A0400000004075
:100E800000005643000046431FC5484300000000D1
:100E9000000000001F856B3E0000564300004643E3
:100EA0000000494300000000000000001F856B3E69
:100EB0006563686F3A004572726F723A00436172FF
:100EC000642072656D6F76656400436172642069A9
:100ED0006E73657274656400473120453430204676
:100EE0003130300047312045373020463430300033
:100EF0004D383300473120452D38302046343030CE
:100F0000004D3833002D2D3A2D2D002D2D2D005361
:100F1000440001200001200041646A757374696E09
:100F200067205A004D6F646520202020205B736984
:100F30006C656E745D004D6F6465205B6869676801
:100F400020706F7765725D004C6976652061646A18
:100F5000757374205A004D363030004368616E67F7
:100F6000652066696C616D656E7400466C6F770014
:100F7000466C6F770046616E20737065656400464D
:100F8000616E20737065656400426564004265644B
:100F9000004E6F7A7A6C65004E6F7A7A6C650053FA
:100FA00070656564005370656564004D61696E002D
:100FB000436F6F6C646F776E00464C4558202D2050
:100FC000203233302F35300050502020202D20206B
:100FD0003235342F3130300048495053202D2020F5
:100FE0003232302F3130300050455420202D202017
:100FF0003234302F393000504C4120202D20203207
:1010000031302F35300041425320202D2020323501
:10101000352F313030004D61696E004D3834004D50
:10102000383420582059205A2045004D3234004D84
:10103000323320257300052E2E004D61696E004667
:10104000616E2073706565640046616E2073706523
:1010500065640042656400426564004E6F7A7A6C94
:1010600065004E6F7A7A6C650053657474696E67BB
:101070007300580059005A0045787472756465729F
:10108000004578747275646572004D6F7665205AFC
:10109000004D6F76652059004D6F766520580053DE
:1010A000657474696E6773004D6F6465202020203D
:1010B000205B73696C656E745D004D6F6465205BC9
:1010C0006869676820706F7765725D004732380025
:1010D0004175746F20686F6D65004D383400446948
:1010E0007361626C6520737465707065727300471C
:1010F0003238205A0043616C696272617465205A0B
:10110000004D6F766520617869730054656D706578
:10111000726174757265004D61696E005265763A50
:10112000203137352D316100686F77746F2E707202
:1011300075736133642E636F6D00666F72756D2E0B
:10114000707275736133642E636F6D0070727573A6
:101150006133642E636F6D004669726D77617265ED
:10116000202D20322E322E3362004D61696E0053E5
:101170007570706F72740053657474696E67730074
:10118000556E6C6F61642066696C616D656E74008C
:101190004C6F61642066696C616D656E74004E6FA2
:1011A0002053442063617264005072696E7420663B
:1011B000726F6D2053440053746F70207072696EAB
:1011C0007400526573756D65207072696E7400509D
:1011D00061757365207072696E7400507265686520
:1011E00061740054756E6500496E666F207363729A
:1011F00065656E0048617264636F64656420446570
:101200006661756C742053657474696E6773204CE5
:101210006F616465640046696C616D656E7420730E
:10122000657474696E67733A2044697361626C65B2
:1012300064002020204D32303020440046696C612B
:101240006D656E742073657474696E67733A0020FF
:1012500020204D3230392053004175746F2D526576
:1012600074726163743A20533D3020746F20646956
:101270007361626C652C203120746F20696E746517
:10128000727072657420657874727564652D6F6E06
:101290006C79206D6F76657320617320726574724E
:1012A00061637473206F72207265636F7665726913
:1012B0006573002046002020204D32303820530036
:1012C0005265636F7665723A20533D45787472615A
:1012D000206C656E67746820286D6D2920463A532E
:1012E0007065656420286D6D2F6D2900205A0020DF
:1012F00046002020204D3230372053005265747252
:101300006163743A20533D4C656E67746820286DA4
:101310006D2920463A537065656420286D6D2F6DE8
:1013200029205A3A205A4C69667420286D6D29008C
:101330002044002049002020204D3330312050002F
:101340005049442073657474696E67733A00205A7B
:101350000020590020204D323036205800486F6D53
:1013600065206F666673657420286D6D293A0020CC
:101370004500205A00205800204200205400202020
:101380004D323035205300416476616E63656420D0
:101390007661726961626C65733A20533D4D696E86
:1013A00020666565647261746520286D6D2F7329F0
:1013B0002C20543D4D696E2074726176656C2066F8
:1013C0006565647261746520286D6D2F73292C200A
:1013D000423D6D696E696D756D207365676D656EF3
:1013E000742074696D6520286D73292C20583D6D1B
:1013F0006178696D756D205859206A65726B202877
:101400006D6D2F73292C20205A3D6D6178696D75A3
:101410006D205A206A65726B20286D6D2F73292C00
:101420002020453D6D6178696D756D2045206A65A8
:10143000726B20286D6D2F73290020540020204DE1
:10144000323034205300416363656C6572617469A6
:101450006F6E3A20533D616363656C6572617469B8
:101460006F6E2C20543D72657472616374206163E9
:1014700063656C65726174696F6E00204500205A67
:101480000020590020204D3230312058004D617825
:10149000696D756D20416363656C65726174696F18
:1014A0006E20286D6D2F7332293A00204500205A96
:1014B0000020590020204D3230332058004D6178F3
:1014C000696D756D20666565647261746573202849
:1014D0006D6D2F73293A00204500205A00205900D5
:1014E00020204D3932205800537465707320706588
:1014F0007220756E69743A0045303A20005A3A20DD
:1015000000593A2000583A20004D53312C4D5332A7
:101510002050696E730A00656E6473746F70732077
:101520006869743A205A00205A3A00656E647374F0
:101530006F7073206869743A20590020593A006529
:101540006E6473746F7073206869743A2058002059
:10155000583A00656E6473746F7073206869743AEA
:10156000200024F4D43050C38E20C2A24017828BB6
:101570007011127A910D816CD90AA861E108C758DF
:101580006607615143061E4B5D05C145A7041A411C
:101590001104093D9803713931034036DB0265338C
:1015A0009102D4305402802E1D02632CEE01752A64
:1015B000C501B028A001102781018F2564012B24CB
:1015C0004B01E0223401AC211F018D200D01801F51
:1015D000FC00841EED00971DDF00B81CD200E61B46
:1015E000C600201BBC00641AB200B219A8000A1978
:1015F000A0006A189900D117910040178B00B5160A
:10160000840031167E00B31579003A157300C714B3
:101610006F0058146A00EE136600881363002513E8
:101620005E00C7125B006C12570015125400C11106
:10163000510070114F0021114B00D61049008D1040
:1016400047004610440002104200C00F4000800FC7
:101650003E00420F3C00060F3B00CB0E3800930EBD
:1016600037005C0E3500270E3400F30D3200C10D3B
:101670003100900D3000600D2E00320D2D00050D53
:101680002C00D90C2B00AE0C2900850C29005C0C19
:101690002700350C27000E0C2600E80B2400C40B95
:1016A0002400A00B23007D0B23005A0B2100390BD3
:1016B0002100180B2000F80A1F00D90A1E00BB0ADF
:1016C0001E009D0A1D00800A1D00630A1C00470AB7
:1016D0001B002C0A1B00110A1A00F7091A00DD0969
:1016E0001900C4091900AB091900920917007B09F8
:1016F0001800630917004C09160036091600200966
:1017000016000A091500F5081500E0081400CC08B9
:101710001400B8081400A4081400900813007D08F1
:1017200012006B0813005808120046081200340813
:101730001100230811001208110001081100F00720
:101740001000E0071000D0071000C0071000B0071D
:101750000F00A107100091070E0083070F00740708
:101760000F0065070E0057070E0049070E003B07E4
:101770000D002E070E0020070D0013070D000607B1
:101780000D00F9060C00ED060D00E0060C00D40675
:101790000C00C8060C00BC060C00B0060C00A40629
:1017A0000B0099060C008D060B0082060B007706D5
:1017B0000B006C060B0061060A0057060B004C0676
:1017C0000A0042060A0038060A002E060A0024060D
:1017D0000A001A060A001006090007060A00FD059D
:1017E0000900F4050900EB050900E2050900D90527
:1017F0000900D0050900C7050900BE050900B505A7
:101800000800AD050800A50509009C050800940521
:1018100008008C050800840508007C050800740594
:1018200008006C050700650508005D050700560502
:1018300008004E0507004705070040050800380569
:101840000700310507002A050700230507001C05CE
:101850000600160507000F0507000805060002052B
:101860000700FB040600F5040700EE040600E80488
:101870000600E2040700DB040600D5040600CF04DE
:101880000600C9040600C3040600BD040600B70430
:101890000600B1040500AC040600A6040600A0047E
:1018A00005009B04060095040500900406008A04C8
:1018B000050085040500800406007A04050075040F
:1018C0000500700405006B04050066040500610452
:1018D00005005C04050057040500520405004D0492
:1018E000050048040500430405003E0404003A04D2
:1018F000050035040500300404002C04050027040D
:101900000400230405001E0404001A040400160445
:101910000500110404000D0404000904050004047A
:10192000040000040400FC030400F8030400F403B2
:101930000400F0030400EC030400E8030400E403E3
:101940000400E0030400DC030400D8030400D40313
:101950000400D0030400CC030400C8030300C50343
:10196000030024F404D9201BC40C5C0E9804C409A1
:101970005F0265077101F405F900FB04B300480438
:101980008700C10369005803550003034500BE02E8
:101990003A008402310053022A0029022500040281
:1019A0002000E4011C00C8011900AF0117009801D4
:1019B0001400840113007101100061011000510135
:1019C0000E0043010D0036010B002B010B0020011E
:1019D0000B00150109000C01090003010800FB00C0
:1019E0000800F3000800EB000700E4000600DE003A
:1019F0000600D8000600D2000600CC000500C70093
:101A00000500C2000500BD000400B9000400B500D7
:101A10000400B1000400AD000400A9000400A5000A
:101A20000300A20003009F0004009B000300980035
:101A300003009500020093000300900003008D0056
:101A400002008B0003008800020086000200840070
:101A50000300810002007F0002007D0002007B0085
:101A60000200790002007700010076000200740095
:101A7000020072000100710002006F0002006D00A0
:101A800001006C0002006A000100690002006700AA
:101A900001006600010065000100640002006200B0
:101AA000010061000100600001005F0002005D00B4
:101AB00001005C0001005B0001005A0001005900B8
:101AC00001005800010057000100560001005500B8
:101AD00001005400010053000000530001005200B7
:101AE000010051000100500001004F0001004E00B4
:101AF00000004E0001004D0001004C0001004B00B1
:101B000000004B0001004A000100490001004800AC
:101B100000004800010047000100460000004600A8
:101B200001004500000045000100440001004300A1
:101B3000000043000100420000004200010041009B
:101B4000000041000100400001003F0000003F0094
:101B500001003E0000003E0001003D0000003D008D
:101B600001003C0000003C0000003C0001003B0084
:101B700000003B0001003A0000003A00010039007B
:101B80000000390001003800000038000000380073
:101B90000100370000003700010036000000360069
:101BA000000036000100350000003500000035005F
:101BB0000100340000003400000034000100330054
:101BC000000033000000330001003200000032004A
:101BD000000032000100310000003100000031003F
:101BE00001003000000030000000300001002F0034
:101BF00000002F0000002F0000002F0001002E0029
:101C000000002E0000002E0001002D0000002D001D
:101C100000002D0000002D0001002C0000002C0011
:101C200000002C0000002C0001002B0000002B0005
:101C300000002B0000002B0001002A0000002A00F9
:101C400000002A0000002A000100290000002900ED
:101C500000002900000029000000290001002800E0
:101C600000002800000028000000280000002800D4
:101C700001002700000027000000270000002700C7
:101C800000002700010026000000260000002600BA
:101C900000002600000026000100250000002500AD
:101CA00000002500000025000000250000002500A0
:101CB0000100240000002400000024000000240093
:101CC0000000240001002300000023000000230086
:101CD0000000230000002300000023000000230078
:101CE000010022000000220000002200000022006B
:101CF000000022000000220001002100000021005D
:101D0000000021000000210000002100000021004F
:101D10000000210001002000000020000000200041
:101D20000000200000002000000020000000200033
:101D30000000200001001F0000001F0000001F0025
:101D400000001F0000001F0000001F0000001F0017
:101D500001001E0000001E0000001E0000001E000A
:101D6000000020746F6F206C6F6E6720657874724E
:101D70007573696F6E2070726576656E7465640048
:101D800020636F6C6420657874727573696F6E2060
:101D900070726576656E746564000000090A020859
:101DA0000B0C0D07060304010000000000000000FA
:101DB0000000000000000000000000000000000023
:101DC00000000000000011100F00000000000000E3
:101DD0000000000000000000000000000000000003
:101DE00000000000000000000000000000000000F3
:101DF000010210202008081020401020408002011D
:101E00000201080402010102040810204080804001
:101E10002010080402018004020180402010080400
:101E2000020108040201010204081020408001029E
:101E3000040810204080100804088010204004404E
:101E400080102040048005050505070508080808DE
:101E5000020202020A0A0808040404040101010142
:101E6000010101010303030303030303040707073D
:101E70000C0C0C0C0C0C0C0C0202020206060606E2
:101E8000060606060B0B0B0B0B0B0B0B07070A0AC0
:101E90000A0A0A0A050505040404080800002000CF
:101EA0002300260029002C002F0032000001000032
:101EB00003010601090100002200250028002B0073
:101EC0002E003100340002010000050108010B0161
:101ED00000002100240027002A002D0030003300DC
:101EE00001010000040107010A01024E414E494E62
:101EF000495459494E46CDCCCC3D0AD7233C17B75F
:101F0000D13877CC2B329595E6241FB14F0A0000CB
:101F100020410000C84200401C4620BCBE4CCA1BE9
:101F20000E5AAEC59D74AE64DE80CAA9B264112497
:101F30001FBECFEFD1E2DEBFCDBF00E00CBF16E089
:101F4000A0E0B2E0E8E4FAE701E00BBF02C00790CE
:101F50000D92A230B107D9F724E1A2E0B6E001C0AA
:101F60001D92AB3EB207E1F71FE1CCE2DFE100E0FA
:101F700006C022970109FE010BBF0E94B5B6C6320A
:101F8000D10780E00807A9F70E94CEAD0C9413BDDD
:101F90000C940000CF93DF93EC019C012C5F3F4F2A
:101FA00041E050E060E070E0898D9A8D0E946C1AEB
:101FB000882399F04D895E896F89788D452B462B52
:101FC000472B59F44C815D816E817F814D8B5E8BF7
:101FD0006F8B788F998190689983DF91CF91089565
:101FE000CF92DF92EF92FF920F931F93CF93DF93E5
:101FF000EC0189899A89AB89BC89803E9F4FAF41AA
:10200000B10510F080E06BC0CE01C4DF8823D1F3AE
:102010000E948018182F8823A9F3E98DFA8DCC80AF
:10202000DD80EE80FF8032E0C31AD108E108F108BC
:10203000058404C0CC0CDD1CEE1CFF1C0A94D2F7F6
:1020400086859785A089B189C80ED91EEA1EFB1E18
:1020500081E080930806C0920B08D0920C08E092B1
:102060000D08F0920E0880E092E0EBE0F6E0DF0170
:102070009C011D9221503040E1F701E0E98DFA8D7D
:102080008481081790F42BE036E0B701A601400FD9
:10209000511D611D711D8091090690910A060E94D3
:1020A000063D8823E1F00F5FE9CFC12C82E0D82EF6
:1020B000E12CF12C058404C0CC0CDD1CEE1CFF1CB3
:1020C0000A94D2F749895A896B897C894C0D5D1D28
:1020D0006E1D7F1D498B5A8B6B8B7C8B812FDF9103
:1020E000CF911F910F91FF90EF90DF90CF900895C7
:1020F000CF93DF93EC0141E0611101C040E06C85BA
:102100007D858E859F850E94C018882341F088892F
:1021100020E2829FC0011124855F994F02C080E0B8
:1021200090E0DF91CF91089530E020E04EE2DC01B5
:102130005C91503271F0383029F4FB01E20FF11D4F
:1021400040832F5FFB01E20FF11DDC015C915083A6
:102150002F5F3F5F01963B3051F7FB01E20FF11D0E
:1021600010820895CF93DF93EB01FC0123812111AD
:1021700002C080E00EC02250223020F48FE288831B
:10218000198206C060E0B4DF009799F3BE01CCDF8E
:1021900081E0DF91CF910895FB012BE030E2319394
:1021A0002150E9F7DC0190E027E03A2FEB2F8D91E9
:1021B00081110AC0DA013C931196EC9381E0FB0196
:1021C0009081903239F525C08F32A1F38E3219F00B
:1021D000EAE8F1E008C02A30E1F098E02AE0E5CF33
:1021E00031963817B1F034913111FACF291788F0B0
:1021F0003FED380F3E3568F431E0390FFB01E90F50
:10220000F11D9FE9980F9A3108F480528083932F33
:10221000CCCF80E008950F931F93CF93DF93EC0111
:102220008B018B81882311F080E042C0FB018789FC
:10223000803139F18032C1F783E08B83F801428D20
:10224000538D648D758D4D8B5E8B6F8B788F9E015A
:102250002F5E3F4FC8010E947719882329F31A8FF8
:10226000098F81E089831C821D821E821F8218864D
:1022700019861A861B861C861D861E861F86188A4E
:1022800017C082E08B831D8A1E8A1F8A188EFB016D
:10229000408D518D60E070E095E0440F551F661F42
:1022A000771F9A95D1F7498B5A8B6B8B7C8BD7CF45
:1022B000DF91CF911F910F9108952F923F924F92EE
:1022C0005F926F927F928F929F92AF92BF92CF92C6
:1022D000DF92EF92FF920F931F93CF93DF93EC0166
:1022E0005B016A018B81811103C08FEF9FEFC7C033
:1022F000898180FFFACF49895A896B897C898885D1
:102300009985AA85BB852601612C712C8A019B01C8
:10231000081B190B2A0B3B0B40165106620673066D
:1023200018F06A01C81AD90A76013E0124E0620E4B
:10233000711CE114F10409F476C0488559856A8559
:102340007B854A0181E098222B811A012B01E9E06B
:102350005694479437942794EA95D1F7898D9A8DAE
:10236000FC01223049F4628D738D848D958D620D50
:10237000731D841D951D3CC01481115012218114C0
:102380009104C1F4111116C0452B462B472B49F47B
:102390008D899E89AF89B88D8C839D83AE83BF83E1
:1023A00009C04C815D816E817F81930121D7882393
:1023B00009F49BCFE98DFA8D6C817D818E819F819F
:1023C0006250710981099109058404C0660F771F65
:1023D000881F991F0A94D2F726853785408951892D
:1023E000620F731F841F951F610F711D811D911D49
:1023F00020E032E02819390987012E153F0508F43D
:1024000089010115F2E01F0769F520910B08309151
:102410000C0840910D0850910E086217730784074D
:10242000950719F41FC0C6012AC09501AB01BC0174
:102430008091090690910A060E94913C882309F434
:1024400054CFA00EB11E88859985AA85BB85800FC3
:10245000911FA11DB11D88879987AA87BB87E01AA4
:10246000F10A67CF40E08CD6882309F43ECFB4014F
:10247000655F794FA801C5010E94D2B9E2CFDF9113
:10248000CF911F910F91FF90EF90DF90CF90BF9071
:10249000AF909F908F907F906F905F904F903F9004
:1024A0002F900895CF93DF931F92CDB7DEB741E011
:1024B00050E0BE016F5F7F4F00DF019719F4898103
:1024C00090E002C08FEF9FEF0F90DF91CF910895C2
:1024D000CF92DF92EF92FF920F931F93CF93DF93F0
:1024E0006C01EB017A01FC018381823060F0008590
:1024F0001185228533850F71112722273327012B60
:10250000022B032B11F08FEF5CC04115510511F028
:10251000F70110821DE040E250E0BE01C601CDDEB1
:102520008032910539F021E0892B09F420E0822FD7
:10253000819547C028812223C1F0253E61F32E32C8
:1025400051F33B853F733F3061F4E114F10449F0EE
:102550004A8D5B8D452B29F42F713FEF320F3430BC
:1025600030F02B8523FDD7CF2CC080E02AC030E08F
:1025700021503109129FC001139F900D1124F701C2
:10258000E80FF91F298120832B8121832D8122834C
:102590002F812383298524832E85258328892683DB
:1025A0002A8927832C8920872E892187288D2287B5
:1025B0002C8D23872E8D2487288126FFD2CF158648
:1025C000D0CFDF91CF911F910F91FF90EF90DF90CF
:1025D000CF9008951F93CF93DF93EC018B818230CE
:1025E00018F480E090E023C0488559856A857B8592
:1025F000A5E07695679557954795AA95D1F7142F3D
:102600001F70CE014FDF97FDECCF488559856A8555
:102610007B85415E5F4F6F4F7F4F488759876A8741
:102620007B8720E2129FC0011124855F994FDF91C3
:10263000CF911F9108954F925F926F927F92AF92C8
:10264000BF92CF92DF92EF92FF920F931F93CF939F
:10265000DF93EC016A017B012B81222349F08989F8
:102660009A89AB89BC8984179507A607B70710F428
:1026700080E06BC0223009F463C0C114D104E104CE
:10268000F10449F41C821D821E821F82188619865D
:102690001A861B8659C088859985AA85BB85E98DD0
:1026A000FA8DE585F0E03996AC01BD014150510944
:1026B000610971090E2E04C0769567955795479567
:1026C0000A94D2F7970186010150110921093109B5
:1026D00004C03695279517950795EA95D2F7041704
:1026E00015072607370720F0892B8A2B8B2B49F4F7
:1026F0008D899E89AF89B88D8C839D83AE83BF837E
:1027000004C0041B150B260B370B280139015E0191
:1027100084E0A80EB11C411451046104710481F0DD
:102720004C815D816E817F819501898D9A8D60D507
:1027300091E0491A5108610871088111ECCF05C078
:10274000C886D986EA86FB8681E0DF91CF911F910A
:102750000F91FF90EF90DF90CF90BF90AF907F9060
:102760006F905F904F9008950F931F93CF93DF93D7
:10277000EC018B818823D1F1898187FF32C061E030
:10278000CE01B6DC8C01009789F1FC018081853E89
:1027900069F18B81823040F449895A896B897C893F
:1027A000448F558F668F778F4D895E896F89788DBD
:1027B000F801538F428F758B648BE0910206F09184
:1027C0000306309759F0B8016A5E7F4FC8014896FA
:1027D0001995F801808D918D938B828B89818F77EC
:1027E0008983DF91CF911F910F918AC481E0888303
:1027F00080E0DF91CF911F910F910895CF93DF93E8
:10280000EC01B2DF1B82DF91CF910895FC0123819F
:102810002111F4CF08954F925F926F927F92AF9201
:10282000BF92CF92DF92EF92FF920F931F93CF93BD
:10283000DF9300D01F92CDB7DEB75C016A017B0148
:10284000FC0183818130E9F4818181FF1AC0F501A7
:1028500081899289A389B48984179507A607B70748
:1028600080F0892B8A2B8B2B09F472C0F5014084F0
:10287000518462847384B701A601C501DCDE811135
:1028800002C080E066C0F501818D928DC114D10433
:10289000E104F10469F4458956896789708D25D76B
:1028A000882379F3F501158A168A178A108E37C0A6
:1028B000F50144815581668177819E012F5F3F4FED
:1028C00097D48823F1F249815A816B817C81F5018B
:1028D000818D928DFC012789203139F4483FFFEF2B
:1028E0005F0761057105D8F407C0483F2FEF520715
:1028F00062072FE0720798F4F8D6882309F4C1CF55
:10290000F50144815581668177810FEF1FEF2FEF2D
:102910003FE0818D928D51D5882309F4B2CFF50126
:10292000C18AD28AE38AF48A818180688183C50161
:102930001BDF882309F4A5CFB701A6014C145D0461
:102940006E047F0410F4B301A201C50174DE01C05E
:1029500081E00F900F900F900F90DF91CF911F911A
:102960000F91FF90EF90DF90CF90BF90AF907F904E
:102970006F905F904F900895FF920F931F93CF93A6
:10298000DF93EC01F42E80E2689FF0011124E55FF3
:10299000F94F8385817121F0842F827109F04EC037
:1029A00080910B0890910C08A0910D08B0910E0831
:1029B0008C879D87AE87BF87688B4489558960E087
:1029C00070E0BA0155274427028D138D20E030E0D6
:1029D000402B512B622B732B4D8B5E8B6F8B788F23
:1029E0008385887151F4048D158D268D378D098B63
:1029F0001A8B2B8B3C8B81E00BC08031F9F49E014C
:102A00002F5E3F4F898D9A8D72D48823B9F084E070
:102A10008B838F2D8F7089831C821D821E821F8263
:102A2000188619861A861B86F4FE0BC040E050E01B
:102A3000BA01CE01F0DE811104C011C01B8280E01A
:102A40000EC0F5FE0BC049895A896B897C89CE017D
:102A5000DF91CF911F910F91FF90EDCD81E0DF913C
:102A6000CF911F910F91FF900895AF92BF92CF9297
:102A7000DF92EF92FF920F931F93CF93DF937C012E
:102A8000EB016A01B22E898D9A8DF701928F818FA9
:102A900040E050E0BA01CE01CEDDA12C08851985B9
:102AA0002A853B8589899A89AB89BC8908171907CA
:102AB0002A073B07A0F585E03695279517950795DA
:102AC0008A95D1F70F70CE0185DD009709F481C09A
:102AD000FC012081222311F0253EB9F4A1100EC083
:102AE00040910B0850910C0860910D0870910E08F0
:102AF000F7014487558766877787008BFC018081C3
:102B0000AA24A3948111CACF0AC04BE050E0BC01B3
:102B1000C6010E94C5B9892B09F0C0CF58C08B2DC2
:102B20008274823409F055C0AA2049F0F701008967
:102B300061E0C701DDDAEC01009769F44AC08B81DE
:102B4000823009F446C0CE014BDA882309F441C033
:102B5000CBE0D6E000E080E2FE0111928A95E9F731
:102B60008BE0F601DE0101900D928A95E1F7E0918C
:102B70000206F0910306309739F0BE01625F7F4F85
:102B8000CE014096199508C081E298E2998B888B16
:102B900080E098E09F878E87888999899B8B8A8BB4
:102BA000998F888F8E859F859F8B8E8BA9D2882346
:102BB00081F04B2D602FC701DF91CF911F910F91B5
:102BC000FF90EF90DF90CF90BF90AF90D5CEB7FE43
:102BD000F0CF80E0DF91CF911F910F91FF90EF90A8
:102BE000DF90CF90BF90AF9008953F924F925F9249
:102BF0006F927F928F929F92AF92BF92CF92DF920D
:102C0000EF92FF920F931F93CF93DF93CDB7DEB771
:102C1000C354D1090FB6F894DEBF0FBECDBF5C011F
:102C20006B0124965FAF4EAF2497522E1C8E1F8EE1
:102C300019821C826115710511F410E073C0FC014A
:102C400083818111FACF2496EEADFFAD2497808168
:102C50008F3211F076011DC02496EEADFFAD2497A2
:102C600080818F3231F431962496FFAFEEAF2497F6
:102C7000F3CFF60183818250823060F3F601618DDB
:102C8000728DCE010196C7DA8823B9F2CE01019682
:102C90007C018E01045E1F4F3801FE0131964F0109
:102CA000402E312E19C08823A9F121E0AE01495CE4
:102CB0005F4FB701C801D9DE882309F4BECFEC14F9
:102CC000FD0411F0C7019ADD0615170501F1942DD9
:102CD000832D7801092F182FAE014E5B5F4FBE0187
:102CE000695C7F4F24968EAD9FAD249755DA88237B
:102CF00009F4A3CF2496EEADFFAD249780818F32E7
:102D000091F631962496FFAFEEAF2497F3CF982D2E
:102D1000892DDFCF252DAE01495C5F4FB701C5017D
:102D2000A4DE182FCE01019671DDCE014C966EDD2A
:102D3000812FCD5BDF4F0FB6F894DEBF0FBECDBF46
:102D4000DF91CF911F910F91FF90EF90DF90CF9087
:102D5000BF90AF909F908F907F906F905F904F90BB
:102D60003F900895CF93DF93EC0140E050E0BA012B
:102D700052DD882361F061E0CE01BAD9009739F0C5
:102D800025EEFC0120831B82DF91CF91B9C180E049
:102D9000DF91CF9108951F93CF93DF93CDB7DEB727
:102DA0006B970FB6F894DEBF0FBECDBFAB01198293
:102DB0001C8222E0BC01CE01019617DF182F882368
:102DC00021F0CE010196CEDF182FCE0101961EDD37
:102DD000812F6B960FB6F894DEBF0FBECDBFDF918B
:102DE000CF911F9108952F923F924F925F926F92D1
:102DF0007F928F929F92AF92BF92CF92DF92EF928B
:102E0000FF920F931F93CF93DF9300D01F921F92D7
:102E1000CDB7DEB78C015B013A01DC0113968C91D2
:102E200013978130C1F411968C9181FF14C082FFF9
:102E300018C0F80141895289638974898085918518
:102E4000A285B38584179507A607B70751F0C80177
:102E5000F2DB811106C081E0F80180838FEF9FEFE4
:102E600037C1630183C0D80159968D919C915A97BF
:102E7000FC01F481F1501A012B0169E0569447944A
:102E8000379427946A95D1F7F221FD834A0121E016
:102E90009222FF2309F476C080E092E08819990914
:102EA00076018C159D0508F47C01D8015996ED91A9
:102EB000FC915A9714962D903D904D905C901797E9
:102EC000B2E02B1A310841085108058404C0220CD5
:102ED000331C441C551C0A94D2F786859785A0891B
:102EE000B189280E391E4A1E5B1EED812E0E311C43
:102EF000411C511CE114F2E0FF0609F089C08091E9
:102F00000B0890910C08A0910D08B0910E08821545
:102F10009305A405B50569F4109208068FEF9FEF9D
:102F2000DC0180930B0890930C08A0930D08B093DC
:102F30000E089501B201A1018091090690910A063F
:102F40000E94063D882309F486CFF801808591858B
:102F5000A285B3858E0D9F1DA11DB11D8087918710
:102F6000A287B387AE0CBF1CCE18DF08D801189615
:102F70004D915D916D917C911B97C114D10409F025
:102F800072CF7AC08114910409F086CF14964D91C6
:102F90005D916D917C911797411551056105710502
:102FA00059F455968D919D910D90BC91A02D00974F
:102FB000A105B10539F520C09E012F5F3F4F18D103
:102FC000882309F448CF89819A81AB81BC81F801BB
:102FD000218D328DF9012789203139F4883FFFEFA7
:102FE0009F07A105B10540F40DC0883F2FEF920760
:102FF000A2072FE0B20730F0C8010E94CA0F81116A
:103000004BCF29CFF80184839583A683B78344CF20
:103010008114910411F5D80118964D915D916D912F
:103020007C911B9751968D919D910D90BC91A02DF7
:10303000481759076A077B0780F062D0882309F494
:103040000ACF81E08093080620920B0830920C088A
:1030500040920D0850920E0807C041E0C201B10134
:103060008FD0882309F4F7CEA701B501C401855F8D
:10307000994F0E94D2B969CF51968D919D910D9033
:10308000BC91A02DF801218184179507A607B707E9
:1030900038F4418B528B638B748B206821830CC076
:1030A0008091020690910306892B31F0611471041E
:1030B00019F02068F8012183D80111968C9183FDC5
:1030C00002C0C30105C0C8014FDB8111FACFC3CED6
:1030D0000F900F900F900F900F90DF91CF911F9155
:1030E0000F91FF90EF90DF90CF90BF90AF909F90A7
:1030F0008F907F906F905F904F903F902F900895AA
:10310000CF93809108068823B9F140910B08509124
:103110000C0860910D0870910E082BE036E080914C
:10312000090690910A060E94063DC82F811102C02F
:10313000C0E023C040910406509105066091060648
:1031400070910706411551056105710591F02BE05D
:1031500036E08091090690910A060E94063D882378
:1031600039F310920406109205061092060610928A
:1031700007061092080601C0C1E08C2FCF91089578
:10318000CF92DF92EF92FF92CF936B017C01C42F1D
:1031900080910B0890910C08A0910D08B0910E0839
:1031A0008C159D05AE05BF05C9F0AADF811102C0CF
:1031B00080E018C02BE036E0B701A6018091090637
:1031C00090910A060E94913C882391F3C0920B08CB
:1031D000D0920C08E0920D08F0920E0881E0C11127
:1031E00080930806CF91FF90EF90DF90CF900895E5
:1031F0008F929F92AF92BF92CF92DF92EF92FF9207
:103200000F931F93CF93DF93EC016A017B01890138
:1032100089859A85AB85BC850196A11DB11D841752
:103220009507A607B70710F480E054C08F89803156
:1032300029F49927872F762F652F0BC08032A1F7AD
:10324000CB01BA0127E096958795779567952A95E2
:10325000D1F78B889C88AD88BE88680D791D8A1D42
:103260009B1D80900B0890900C08A0900D08B090CA
:103270000E08681579058A059B0581F48F898031D0
:1032800091F4DD24EE24FF24F601EE0FFF1FE55F2D
:10329000F94F80819181A0E0B0E016C040E070DF7E
:1032A0008111ECCFC1CFE894C7F8DD24EE24FF24D0
:1032B000F601EE0FFF1FEE0FFF1FE55FF94F808154
:1032C0009181A281B381BF70F80180839183A28331
:1032D000B38381E0DF91CF911F910F91FF90EF9029
:1032E000DF90CF90BF90AF909F908F9008954F92B6
:1032F0005F926F927F92AF92BF92CF92DF92EF92E6
:10330000FF920F931F93CF93DF9300D01F92CDB7FF
:10331000DEB78C0149835A836B837C835901C12CAE
:10332000D12C7601412C42E0542E612C712C498124
:103330005A816B817C819E012F5F3F4FC80158DF0E
:10334000882341F1D301C201F801058404C0880F2C
:10335000991FAA1FBB1F0A94D2F7C80ED91EEA1ED6
:10336000FB1E49815A816B817C818789803139F4C8
:1033700081E0483F5F4F6105710538F4D8CF81E0A7
:10338000483F5F4F6F4F7F4090F2F501C082D1827E
:10339000E282F3820F900F900F900F90DF91CF9108
:1033A0001F910F91FF90EF90DF90CF90BF90AF9063
:1033B0007F906F905F904F9008954F925F926F92C1
:1033C0007F928F929F92AF92BF92CF92DF92EF92B5
:1033D000FF920F931F93CF93DF93EC014A015B01A0
:1033E00028013901423051056105710508F462C0B8
:1033F00049855A856B857C854F5F5F4F6F4F7F4F47
:10340000481559056A057B0508F454C08F89803139
:1034100029F4FF24EB2CDA2CC92C0CC0803209F0E3
:1034200049C07501640177E0F694E794D794C79496
:103430007A95D1F74B895C896D897E89C40ED51E3A
:10344000E61EF71E41E0C701B6019ADE882391F11E
:103450009F89903159F49924AA24BB24F401EE0FDA
:10346000FF1FE55FF94F5182408210C0E89487F852
:103470009924AA24BB24F401EE0FFF1FEE0FFF1FB7
:10348000E55FF94F40825182628273829A8992305D
:1034900090F04D815E816F8178854C0D5D1D6E1DB4
:1034A0007F1D4093040650930506609306067093B3
:1034B000070601C080E0DF91CF911F910F91FF902F
:1034C000EF90DF90CF90BF90AF909F908F907F90C4
:1034D0006F905F904F9008952F923F924F925F921E
:1034E0006F927F928F929F92AF92BF92CF92DF9214
:1034F000EF92FF920F931F93CF93DF93CDB7DEB779
:103500002F970FB6F894DEBF0FBECDBF1C014C87BE
:103510005D876E877F873B872A87DC0119960D912F
:103520001D912D913C911C970F5F1F4F2F4F3F4FC7
:103530000D831E832F833887EA85FB8580809180E9
:10354000A280B38081149104A104B10431F0FFEF93
:103550008F1A9F0AAF0ABF0A10C0DC018D909D90A0
:10356000AD90BC90B1E0B9870C851D852E853F8557
:10357000013011052105310509F019867501640135
:10358000412C512C3201F10181859285A385B485AE
:10359000481659066A067B0608F04EC00D811E814A
:1035A0002F8138850C151D052E053F0550F4F2E0DE
:1035B000CF2ED12CE12CF12CA2E08A2E912CA12C23
:1035C000B12C9E012F5F3F4FB701A601C10110DE54
:1035D000882391F149815A816B817C81D701C60191
:1035E0000196A11DB11D452B462B472B19F04C010F
:1035F0005D010FC0AC01BD01481959096A097B0979
:103600000C851D852E853F8540175107620773077E
:1036100041F01FEF411A510A610A710A6C017D01E4
:10362000B2CF0FEF1FEF2FEF3FE0B701A601C101AF
:10363000C4DE8D83811113C01D823DC02601370178
:1036400021E0421A51086108710897018601B3010F
:10365000A201C101B2DE882379F3730162018C14E7
:103660009D04AE04BF0450F3AA85BB854D915D91C6
:103670006D917C914115510561057105A9F4EA85AB
:10368000FB8580829182A282B382F985FF2399F023
:103690000FEF801A900AA00AB00AD1018D929D9274
:1036A000AD92BC92139707C095018401C10185DEDC
:1036B0008111E5CFC1CF8D812F960FB6F894DEBF73
:1036C0000FBECDBFDF91CF911F910F91FF90EF9073
:1036D000DF90CF90BF90AF909F908F907F906F9032
:1036E0005F904F903F902F900895AF92BF92CF92EE
:1036F000DF92EF92FF920F931F93CF93DF9300D04F
:103700001F92CDB7DEB75C016A017B0182E090E0D9
:10371000A0E0B0E0F50180839183A283B3839E0192
:103720002F5F3F4FB701A601C50162DD811102C0C5
:1037300080E023C000E010E09801B701A601C501B8
:103740003CDE8823A9F3C980DA80EB80FC80F50198
:103750008789803149F481E0F8EFCF16FFEFDF066B
:10376000E104F10450F4DBCF81E098EFC9169FEF3C
:10377000D906E9069FE0F90690F20F900F900F909E
:103780000F90DF91CF911F910F91FF90EF90DF90FD
:10379000CF90BF90AF9008957F928F929F92AF92FB
:1037A000BF92CF92DF92EF92FF920F931F93CF932E
:1037B000DF93EC01142F70930A06609309061F8AA9
:1037C00082E090E0A0E0B0E088839983AA83BB8385
:1037D0001092080610920406109205061092060632
:1037E000109207068FEF9FEFDC0180930B089093F8
:1037F0000C08A0930D08B0930E08442349F14530FE
:1038000008F0DEC040E060E070E0CB01B9DC882366
:1038100009F4D6C020E1129FF0011124E754F84FBB
:1038200080818F7709F0CCC084859585A685B78582
:1038300084369105A105B10508F4C2C0C084D184C5
:10384000E284F384C114D104E104F10421F4B8C08A
:10385000C12CD12C760140E0C701B60191DC782E55
:10386000882309F4ADC08091160690911706811542
:10387000924009F0A5C030911B06332309F4A0C083
:103880008091190690911A06892B09F499C020910C
:103890001806222309F494C03A8B2C831D8630E04D
:1038A00041E050E06D85062FCA01062E02C0880F48
:1038B000991F0A94E2F72817390731F081E0860F43
:1038C0008D87683078F37CC02091210630912206E4
:1038D0002115310519F040E050E008C020912F0675
:1038E0003091300640913106509132062D833E834F
:1038F0004F8358878091190690911A064601570107
:10390000880E991EA11CB11C8B8A9C8AAD8ABE8A26
:10391000E0911C06F0911D06F98FE88FA0911B061F
:10392000B0E00E94A5B6680D791D8A1D9B1D6A8FA7
:103930007B8F8C8F9D8FB5E0EE0FFF1FBA95E1F75F
:10394000E150FE4FEF2FFF27E695DC01CB018E0FF4
:103950009F1FA11DB11D8E879F87A88BB98B80905B
:103960001E0690901F068114910419F0A12CB12C11
:1039700008C080902B0690902C06A0902D06B09049
:103980002E06A7019601281B390B4A0B5B0BDA01A7
:10399000C901880D991DAA1DBB1D04C0B695A79528
:1039A000979587950A95D2F789879A87AB87BC87C1
:1039B000853F3FE09307A105B10520F48CE08F8B94
:1039C000712C15C0853F9F4FA105B10510F480E112
:1039D0000DC08091370690913806A0913906B091BC
:1039E0003A068A8F9B8FAC8FBD8F80E28F8B872D9D
:1039F000DF91CF911F910F91FF90EF90DF90CF90CB
:103A0000BF90AF909F908F907F9008954F925F925C
:103A10006F927F928F929F92AF92BF92CF92DF92DE
:103A2000EF92FF920F931F93CF93DF932C0124EF1C
:103A300033E081E090E0F901459154914416550638
:103A40000CF062C0AC0141505109DA01AA0FBB1F52
:103A5000AA0FBB1FAE50BC4FFD0165917491440F7E
:103A6000551F440F551F40515C4FFA0165907490EB
:103A7000FC01EE0FFF1FEE0FFF1FEE50FC4FA59055
:103A8000B490FD0105911491F901C591D491FA0109
:103A900085909490882777FD8095982F0E941FB37A
:103AA0006B017C01B20166197709882777FD809543
:103AB000982F0E941FB32B013C01B501601B710BB5
:103AC000882777FD8095982F0E941FB39B01AC013A
:103AD000C301B2010E9452B52B013C01BE0168191D
:103AE0007909882777FD8095982F0E941FB39B0145
:103AF000AC01C301B2010E9484B29B01AC01C701B9
:103B0000B6010E94A4B111C001962C5F3F4F8D33C6
:103B1000910509F090CFE2EEF4E065917491882769
:103B200077FD8095982F0E941FB3DF91CF911F9151
:103B30000F91FF90EF90DF90CF90BF90AF909F904C
:103B40008F907F906F905F904F9008954F925F920B
:103B50006F927F928F929F92AF92BF92CF92DF929D
:103B6000EF92FF920F931F93CF93DF932C01662365
:103B700071F1E6EBFEE08491882341F09091C00062
:103B800095FFFCCF8093C6003196F5CF70E04AE0F8
:103B900050E089EC9DE00E94DE8DE9E5F2E0849141
:103BA000882341F09091C00095FFFCCF8093C60020
:103BB0003196F5CF8091C00085FFFCCF8AE08093DD
:103BC000C6000E94414660E070E0CB017EC024E761
:103BD00033E081E090E0F901459154914416550697
:103BE0000CF062C0AC0141505109DA01AA0FBB1FB1
:103BF000AA0FBB1FAE58BC4FFD0165917491440FD5
:103C0000551F440F551F40595C4FFA016590749041
:103C1000FC01EE0FFF1FEE0FFF1FEE58FC4FA590AB
:103C2000B490FD0105911491F901C591D491FA0167
:103C300085909490882777FD8095982F0E941FB3D8
:103C40006B017C01B20166197709882777FD8095A1
:103C5000982F0E941FB32B013C01B501601B710B13
:103C6000882777FD8095982F0E941FB39B01AC0198
:103C7000C301B2010E9452B52B013C01BE0168197B
:103C80007909882777FD8095982F0E941FB39B01A3
:103C9000AC01C301B2010E9484B29B01AC01C70117
:103CA000B6010E94A4B111C001962C5F3F4F803233
:103CB000910509F090CFEEEEF3E0659174918827BD
:103CC00077FD8095982F0E941FB3DF91CF911F91B0
:103CD0000F91FF90EF90DF90CF90BF90AF909F90AB
:103CE0008F907F906F905F904F90089560E08091EB
:103CF0006408909165082ADF6093600870936108FA
:103D0000809362089093630880915E0890915F08A9
:103D10007DDE60935A0870935B0880935C089093F3
:103D20005D088FB7F894109252088FBF08952091C4
:103D3000140230911502409116025091170260E072
:103D400070E08FE793E40E9484B26093320870932E
:103D500033088093340890933508089597FF03C083
:103D60008091590804C0FC01E45DF74F808190E028
:103D70000895CF93DF93D82FC62FC19561E00E949D
:103D80002EAC6C2F8D2F0E9467AC6C2F70E08D2FA6
:103D9000DF91CF910C9424ABCF93C1E020E030E0D1
:103DA00048E452E460916008709161088091620873
:103DB000909163080E9480B418160CF0C0E06C2F3C
:103DC00088E090E0CF91D5CF2F923F924F925F92B3
:103DD0006F927F928F929F92AF92BF92CF92DF921B
:103DE000EF92FF920F931F93CF93DF93CDB7DEB780
:103DF00028970FB6F894DEBF0FBECDBF8091520852
:103E0000882309F4F8C172DF8090600890906108FF
:103E1000A0906208B090630800916808109169084A
:103E2000B801882777FD8095982F0E941FB3A501C0
:103E300094010E94A3B16B017C0160933A087093D6
:103E40003B0880933C0890933D0820E030E040E23E
:103E500051E40E9480B4181624F481E08093310864
:103E6000F7C020E030E040E251ECC701B6010E940B
:103E70007DB287FD02C0012B21F481E080933108DF
:103E80000CC180913108882351F010924E08109295
:103E90004F0810925008109251081092310820914A
:103EA00018023091190240911A0250911B02C70169
:103EB000B6010E9452B569837A838B839C83609399
:103EC00046087093470880934808909349082091CA
:103ED0004E0830914F084091500850915108C70149
:103EE000B6010E94A4B12B013C012090360830900D
:103EF000370810913808009139089101412F502F4F
:103F00000E947DB287FD14C02090320830903308A3
:103F100010913408009135089101412F502FB201C2
:103F2000C3010E9480B418161CF01201162D072D33
:103F3000C101A12FB02F80934E0890934F08A093FA
:103F40005008B0935108209114023091150240910D
:103F5000160250911702B101812F902F0E9452B585
:103F60006D837E838F8398876093420870934308A4
:103F7000809344089093450820914A0830914B085B
:103F800040914C0850914D08C501B4010E94A3B165
:103F900020911002309111024091120250911302AF
:103FA0000E9452B520ED3CEC4CE45DE30E9452B51A
:103FB0002B013C0123E333E343E75FE360913E08D9
:103FC00070913F0880914008909141080E9452B53D
:103FD0009B01AC01C301B2010E94A4B12B013C01C1
:103FE00060933E0870933F08809340089093410887
:103FF0002D813E814F81588569817A818B819C8199
:104000000E94A4B1A30192010E94A3B12B013C0123
:1040100020E030E04FE753E40E9480B420E030E03D
:10402000A9011816E4F4C701B6010E9480B418165D
:104030007CF4A7019601B101812F902F0E94A3B1BA
:1040400060934E0870934F088093500890935108E6
:10405000412C512C9FE7692E93E4792E21C0C30196
:10406000B2010E947DB287FF1BC020E030E0A901B1
:10407000C701B6010E947DB287FF0FC0A70196015C
:10408000B101812F902F0E94A3B160934E087093CD
:104090004F088093500890935108412C512C3201C5
:1040A00080924A0890924B08A0924C08B0924D081A
:1040B0006091240870912508882777FD8095982FB6
:1040C0000E941FB39B01AC01C501B4010E9480B4E2
:1040D0001816DCF46091080270910902882777FDB8
:1040E0008095982F0E941FB39B01AC01C501B401BC
:1040F0000E947DB287FF09C0C301B2010E94ECB2E9
:104100007595679560932C0802C010922C080E9448
:104110000EAD009128081091290820912A083091AD
:104120002B08601B710B820B930B653C794081055A
:10413000910558F031DE0E940EAD6093280870930F
:10414000290880932A0890932B080E940EAD0091B5
:104150002D0810912E0820912F0830913008601BF7
:10416000710B820B930B683873418105910508F43C
:1041700042C00E940EAD60932D0870932E0880936C
:104180002F0890933008C0905A08D0905B08E090B8
:104190005C08F0905D0820E030E040E751E4C701A2
:1041A000B6010E9480B418161CF520E030E046E10C
:1041B00053E4C701B6010E947DB287FF19C0609128
:1041C000660870916708882777FD8095982F0E9470
:1041D0001FB39B01AC01C701B6010E9480B487FDEB
:1041E00003C01092590807C08FE78093590803C095
:1041F00010925908A59828960FB6F894DEBF0FBE06
:10420000CDBFDF91CF911F910F91FF90EF90DF9085
:10421000CF90BF90AF909F908F907F906F905F9066
:104220004F903F902F900895CF93DF9310923608D0
:104230001092370810923808109239082091140211
:1042400030911502409116025091170260E070E023
:104250008FE793E40E9484B260933208709333082E
:1042600080933408909335086D9A809101018061A4
:10427000809301019D9A80910101886080930101E2
:1042800087ED80937A0010927E0010927D008091DD
:104290007E00816080937E0080917E0082608093AA
:1042A0007E0080917E00846080937E0080E888BDDF
:1042B00080916E00846080936E006AEF70E080E011
:1042C00090E00E943DAD8FE090E0909325088093B0
:1042D000240860E080910A0290910B0237DC20E014
:1042E00030E040E751E40E947DB287FF0AC0809130
:1042F0000A0290910B02409790930B0280930A025E
:10430000E8CF83E091E0909309028093080260E097
:10431000809126089091270819DC20E030E841E8D8
:1043200053E40E9480B4181654F4809126089091AA
:10433000270840969093270880932608E8CFC091DD
:104340002208D0912308CE0161DB20E030E046E175
:1043500053E40E9480B4181634F46096D093230876
:10436000C0932208ECCFDF91CF9108950895109269
:1043700069081092680810926708109266081092F7
:104380002C087598109267081092660810925908C8
:10439000A59808952F923F924F925F926F927F92CD
:1043A0008F929F92AF92BF92CF92DF92EF92FF9245
:1043B0000F931F93CF93DF93CDB7DEB7AE970FB6B2
:1043C000F894DEBF0FBECDBF6B8F7C8F8D8F292EF3
:1043D0005A8749873CA72BA70E940EAD6F8F78A301
:1043E00089A39AA30E940EAD6FA378A789A79AA765
:1043F00029853A85121613061CF0E0E3F3E017C096
:10440000E3E4F3E08191882339F09091C00095FFB7
:10441000FCCF8093C600F6CF8091C00085FFFCCF13
:104420001BC29091C00095FFFCCF8093C600819184
:104430008111F7CF8091C00085FFFCCF8AE0809387
:10444000C60095DF49855A858FE7452B99F1809302
:1044500059088F8D98A1A9A1BAA1898B9A8BAB8B92
:10446000BC8B8D879E87AF87B88B1D8290E4988F19
:10447000ACE1A98FB6E4BA8F1DA61D8A1E8A1F8AD9
:104480002FE730E040E050E029833A834B835C83A0
:10449000EFE74E2E512C612C712C1BA21CA21DA2E9
:1044A0001EA231E03E8F1C861B86312C00E010E0FE
:1044B0001EA605C080932C08CCCF0E949F778091C8
:1044C0005208882309F4F6C011DC49855A85452B2A
:1044D00051F030905A0800915B0810915C0850919F
:1044E0005D085EA709C030906008009161081091D6
:1044F0006208809163088EA7232D302F412F5EA57F
:104500006DA57D898E899F890E9480B418162CF034
:104510003DA60D8B1E8B9EA59F8B232D302F412FEB
:104520005EA56D81788D898D9A8D0E947DB287FD03
:1045300005C03D82088F198FAEA5AA8F0E940EADCF
:104540002FA138A549A55AA5621B730B840B950BA7
:10455000653C79408105910538F01EDC0E940EAD66
:104560006FA378A789A79AA74E8D442309F44FC05B
:104570002B8D3C8D4D8D522D632D702F812F9EA53F
:104580000E9480B418160CF095C00E940EAD2989C7
:104590003A894B895C89621B730B840B950B6938D4
:1045A00073418105910508F485C0D301C2012981B9
:1045B0003A814B815C81821B930BA40BB50B49851F
:1045C0005A85B595A79597958795452B19F08093B2
:1045D000590802C080932C080E940EAD6D877E871B
:1045E0008F87988BDC01CB0129893A894B895C89BB
:1045F000821B930BA40BB50B8BA39CA3ADA3BEA3F3
:104600003B8D3DA74C8D4D8B5D8D5E8B2F8A2B8D09
:104610003C8D4D8D522D632D702F812F9EA50E94B4
:104620007DB287FFEEC20E940EAD2D853E854F857F
:104630005889621B730B840B950B69387341810594
:10464000910508F4DEC20E940EAD698B7A8B8B8BCC
:104650009C8BDC01CB012D853E854F855889821BC3
:10466000930BA40BB50B4B855C85452B09F010C152
:1046700089819A81AB81BC81840D951DA61DB71DD2
:1046800029853A85B595A79597958795232B09F4A4
:10469000B5C2809359084B855C854F5F5F4F5C873F
:1046A0004B875B8D5D838C8D888F9D8D998F2A8E36
:1046B000A1E0AE8F20E030E040EA51E46B8D7C8DCC
:1046C0008D8D922D0E94A4B19B01AC01632D702FA2
:1046D000812F9EA50E9480B4181694F4EFEFF2E0AB
:1046E0008491882341F09091C00095FFFCCF809386
:1046F000C6003196F5CF8091C00085FFFCCFACC0DD
:104700000E940EAD2F8D38A149A15AA1621B730BD7
:10471000840B950B613D77408105910508F44FC0EE
:1047200049855A85452B81F0E0905908F12CE9EF35
:10473000F2E084918823C1F09091C00095FFFCCFF6
:104740008093C6003196F5CFE0902C08F12CE3EF72
:10475000F2E08491882341F09091C00095FFFCCF56
:104760008093C6003196F5CF22E030E0432D502FE4
:10477000612F7EA589EC9DE00E94B48EEFEEF2E001
:104780008491882341F09091C00095FFFCCF8093E5
:10479000C6003196F5CF4AE050E0B70189EC9DE0C4
:1047A0000E94DE8D8091C00085FFFCCF8AE080935F
:1047B000C6000E940EAD6F8F78A389A39AA30E94B2
:1047C0000EAD6B017C010E940EAD89889A88AB8882
:1047D000BC882D853E854F855889820E931EA41E68
:1047E000B51EC818D908EA08FB08C60ED71EE81E71
:1047F000F91E31E8C3163FE4D30632E1E306F104C3
:1048000090F0E2EDF2E08491882341F09091C000B5
:1048100095FFFCCF8093C6003196F5CF8091C00004
:1048200085FFFCCF19C04B855C858BA59CA58417A3
:1048300095070CF042CEE6E7F2E08491882341F040
:104840009091C00095FFFCCF8093C6003196F5CFC4
:104850008091C00085FFFCCF8AE08093C600AE96B1
:104860000FB6F894DEBF0FBECDBFDF91CF911F9181
:104870000F91FF90EF90DF90CF90BF90AF909F90FF
:104880008F907F906F905F904F903F902F90089502
:104890008BA09CA0ADA0BEA0880E991EAA1EBB1E18
:1048A0002BA13CA14DA15EA1281B390B4A0B5B0B30
:1048B000CA01B90129813A814B815C810E9418B6F5
:1048C000A50194010E947DB6240D351D461D571D7E
:1048D000243131054105510504F129013A013CEE2D
:1048E00043165104610471042CF06BEE462E512CDA
:1048F000612C712C40E84416510461047104DCF011
:104900008EEF90E0A0E0B0E084199509A609B70900
:1049100089839A83AB83BC8312C054E1452E512C0A
:10492000612C712C24E130E040E050E029833A838F
:104930004B835C8304C049825A826B827C82E8E6A6
:10494000F3E08491882341F09091C00095FFFCCF63
:104950008093C6003196F5CF2AE030E0B301A20182
:1049600089EC9DE00E94B38DE3E6F3E08491882317
:1049700041F09091C00095FFFCCF8093C600319626
:10498000F5CF2AE030E049815A816B817C8189EC46
:104990009DE00E94B38DECE5F3E08491882341F023
:1049A0009091C00095FFFCCF8093C6003196F5CF63
:1049B00022E030E04D81588D698D7A8D89EC9DE043
:1049C0000E94B48EE5E5F3E08491882341F0909154
:1049D000C00095FFFCCF8093C6003196F5CF22E052
:1049E00030E04DA55D896E897F8989EC9DE00E944C
:1049F000B48E8091C00085FFFCCF8AE08093C60012
:104A00002B853C85233031050CF432CE69817A81C7
:104A10008B819C810E941FB320E030E040E850E48D
:104A20000E9452B56B017C012D81388D498D5A8DC4
:104A30006DA57D898E899F890E94A3B120ED3FE0FD
:104A400049E450E40E9452B520E030E040E05FE3EA
:104A50000E9452B59B01AC01C701B6010E9484B20D
:104A60006B017C01C501B4010E941FB320E030E05E
:104A70004AE754E40E9484B24B015C01EFE4F3E0A6
:104A80008491882341F09091C00095FFFCCF8093E2
:104A9000C6003196F5CF22E030E0B701A60189ECDF
:104AA0009DE00E94B48EE9E4F3E08491882341F014
:104AB0009091C00095FFFCCF8093C6003196F5CF52
:104AC00022E030E0B501A40189EC9DE00E94B48EA3
:104AD0008091C00085FFFCCF8AE08093C6002AE960
:104AE00039E949E15FE3C701B6010E9452B56B01A4
:104AF0007C019B01AC010E94A4B1A50194010E941C
:104B000084B26D837E838F839887A5019401C7014A
:104B1000B6010E9452B520E030E040E05EE30E9422
:104B200052B54B015C01EBE3F3E08491882341F043
:104B30009091C00095FFFCCF8093C6003196F5CFD1
:104B40008091C00085FFFCCF8AE08093C600E5E33A
:104B5000F3E08491882341F09091C00095FFFCCF51
:104B60008093C6003196F5CF22E030E0B701A60170
:104B700089EC9DE00E94B48E8091C00085FFFCCF3F
:104B80008AE08093C600EFE2F3E08491882341F04D
:104B90009091C00095FFFCCF8093C6003196F5CF71
:104BA00022E030E04D815E816F81788589EC9DE067
:104BB0000E94B48E8091C00085FFFCCF8AE0809374
:104BC000C600E9E2F3E08491882341F09091C000AF
:104BD00095FFFCCF8093C6003196F5CF22E030E000
:104BE000B501A40189EC9DE00E94B48E8091C000C3
:104BF00085FFFCCF8AE08093C6003ACD80932C08D5
:104C00004ACD1E8E57CDCF93C82FB1DB0E94084BE3
:104C1000811134C0E6EBFEE09491992341F080913C
:104C2000C00085FFFCCF9093C6003196F5CF6C2F66
:104C300070E04AE050E089EC9DE00E94DE8D8091BA
:104C4000C00085FFFCCF8AE08093C600ECE2F2E072
:104C50008491882341F09091C00095FFFCCF809310
:104C6000C6003196F5CF8091C00085FFFCCF8AE069
:104C70008093C6008FE192E00E941077CF910C9450
:104C8000C94ACF93C82F73DB0E94084B811134C0EF
:104C9000E6EBFEE09491992341F08091C00085FFFE
:104CA000FCCF9093C6003196F5CF6C2F70E04AE0B0
:104CB00050E089EC9DE00E94DE8D8091C00085FF70
:104CC000FCCF8AE08093C600E2EFF1E08491882374
:104CD00041F09091C00095FFFCCF8093C6003196C3
:104CE000F5CF8091C00085FFFCCF8AE08093C6009D
:104CF00085EE91E00E941077CF910C94C94AA59857
:104D00000E94084B811125C0E6EBFEE084918823C8
:104D100041F09091C00095FFFCCF8093C600319682
:104D2000F5CFEBEAF1E08491882341F09091C00047
:104D300095FFFCCF8093C6003196F5CF8091C000DF
:104D400085FFFCCF8AE08093C6008AE991E00E944B
:104D500010770C94C94A1F920F920FB60F9211242C
:104D60000BB60F920F931F932F933F934F935F9325
:104D70006F937F938F939F93AF93BF93CF93DF9363
:104D8000EF93FF9380910702811112C080912C084C
:104D900080932108882311F0759A01C0759880913D
:104DA000590880932008882311F0A59A01C0A5987E
:104DB0009091210880910702981708F475989091B6
:104DC000200880910702981708F4A598809107029F
:104DD0008F5F8F77809307028091060290E08B307F
:104DE000910508F093C0FC01EE58FF4F0C9499B662
:104DF00010927B0080E480937C0080917A00806434
:104E000080937A000E94197781E019C02091780080
:104E10003091790080911C0890911D08A0911E0886
:104E2000B0911F08820F931FA11DB11D80931C0814
:104E300090931D08A0931E08B0931F0882E08093F2
:104E4000060264C010927B0082E480937C00809113
:104E50007A00806480937A000E94197783E0EFCF14
:104E6000209178003091790080911808909119086C
:104E7000A0911A08B0911B08820F931FA11DB11DAC
:104E80008093180890931908A0931A08B0931B08F0
:104E900084E0D5CF10927B0081E480937C008091E8
:104EA0007A00806480937A000E94197785E0C7CFEA
:104EB0002091780030917900809114089091150824
:104EC000A0911608B0911708820F931FA11DB11D64
:104ED0008093140890931508A0931608B0931708B0
:104EE00086E0ADCF0E94197787E0A9CF88E0A7CFF1
:104EF0000E94197789E0A3CF1092060280911308CF
:104F00008F5F8093130802C01092060280911308ED
:104F1000803108F463C080915208811110C08091E3
:104F20001C0890911D0890936508809364088091F7
:104F300018089091190890935F0880935E0881E0AB
:104F4000809352081092130810921C0810921D08AA
:104F500010921E0810921F08109214081092150843
:104F6000109216081092170810920F08109210084D
:104F70001092110810921208109218081092190835
:104F800010921A0810921B0820916408309165084D
:104F900080912608909127088217930714F080E0EB
:104FA00032DE209164083091650880910A02909168
:104FB0000B022817390714F080E063DE20915E08A9
:104FC00030915F08809122089091230882179307FF
:104FD0002CF0109267081092660891DE00E010E055
:104FE000E801CC0FDD1FCD5AD74F88819981181663
:104FF000190644F461E0802F0E94599788819981B5
:10500000019709C0892B49F060E0802F0E945997D1
:10501000888199810196998388830F5F1F4F0330A0
:105020001105F1F6FF91EF91DF91CF91BF91AF9113
:105030009F918F917F916F915F914F913F912F91B0
:105040001F910F910F900BBE0F900FBE0F901F90EE
:1050500018952CEA35EC47E25EE30C9452B52CEA45
:1050600035EC47E25EE30C9484B22CEA35EC47E27F
:105070005EE30C9484B22CEA35EC47E25EE30C94D8
:1050800052B5CF93DF93EC0160E08E810E9467AC54
:1050900081E090E00E9461AD61E08E810E9467AC8A
:1050A00081E090E00E9461AD60E08E810E9467AC7B
:1050B00084E690E0DF91CF910C9461ADCF92DF92C6
:1050C000EF92FF920F931F93CF93DF937C01C0E089
:1050D000D0E0C62ED12C87010C0F1D1F61E0F80116
:1050E00087810E942EACB6010C2E02C07595679583
:1050F0000A94E2F76170F80187810E9467AC2196FB
:10510000C430D10541F7C701DF91CF911F910F91B5
:10511000FF90EF90DF90CF90B4CFCF92DF92EF92DD
:10512000FF920F931F93CF93DF937C01C0E0D0E0F9
:10513000C62ED12C87010C0F1D1F61E0F80187815D
:105140000E942EACB6010C2E02C0759567950A948C
:10515000E2F76170F80187810E9467AC2196C83040
:10516000D10541F7C701DF91CF911F910F91FF90BA
:10517000EF90DF90CF9085CF1F93CF93DF93EC011B
:10518000162F642F8C810E9467AC8D818F3F19F0A0
:1051900060E00E9467AC8F85612F84FF05C0CE015F
:1051A000DF91CF911F91B9CF70E084E0759567953D
:1051B0008A95E1F7CE0182DF612FCE01DF91CF9199
:1051C0001F917CCF40E0D8CF61E0FCDF80E496E027
:1051D0000C9461AD62E0F6DF80E496E00C9461AD82
:1051E000CF93DF93CDB7DEB728970FB6F894DEBF25
:1051F0000FBECDBF28E0E3EBF2E0DE011196019097
:105200000D922A95E1F7FC012389421710F04FEF28
:10521000420FFE013196E40FF11DE40FF11D2081D4
:10522000260F2068622F28960FB6F894DEBF0FBEB7
:10523000CDBFDF91CF91C6CFFC016089262F2460BE
:10524000208B6C60BFCFCF93DF93EC01423018F01E
:105250008F8588608F874B8B1C8A222329F04130F1
:1052600019F48F8584608F8780E593EC0E9461AD8F
:1052700060E08C810E9467AC60E08E810E9467AC28
:105280008D818F3F19F060E00E9467AC6F8564FDEF
:1052900019C063E0CE0112DF84E991E10E9461ADA3
:1052A00063E0CE010BDF84E991E10E9461AD63E030
:1052B000CE0104DF86E990E00E9461AD62E0CE019C
:1052C000FDDE13C06062CE017DDF84E991E10E94C2
:1052D00061AD6F856062CE0175DF86E990E00E9466
:1052E00061AD6F856062CE016DDF6F856062CE015A
:1052F00069DF8CE390E00E9461AD84E0888BCE0191
:105300009BDF8CE390E00E9461ADCE015DDF88EB16
:105310009BE00E9461AD82E0898B66E0CE0152DFA6
:105320008CE390E0DF91CF910C9461AD6F927F920E
:105330008F92AF92CF92EF920F931F93CF93DF9301
:10534000CDB7DEB73C01162F842F5E854F85388997
:105350009989F301848325830683E782C086A18629
:105360008286538744873587968761E00E942EACFA
:10537000F30185818F3F19F061E00E942EAC61E05E
:10538000F30186810E942EAC112319F0F3011786D8
:1053900003C080E1F301878720E041E060E1C301C1
:1053A000DF91CF911F910F91EF90CF90AF908F90A1
:1053B0007F906F9048CF8F92AF92CF92EF920F93E2
:1053C000DC0113961C921E921297E1E7F3E0ED9335
:1053D000FC931F921F921F921F928C2CAE2CC02EFA
:1053E000E22E042F2FEF462F61E0A0DF0F900F90E9
:1053F0000F900F900F91EF90CF90AF908F900895F6
:10540000CF93DF93EC01423018F08F8588608F874F
:105410004B8B1C8A222329F0413019F48F8584603C
:105420008F8780E593EC0E9461AD60E08C810E94E3
:1054300067AC60E08E810E9467AC8D818F3F19F070
:1054400060E00E9467AC6F8564FD19C063E0CE0127
:1054500035DE84E991E10E9461AD63E0CE012EDE8C
:1054600084E991E10E9461AD63E0CE0127DE86E927
:1054700090E00E9461AD62E0CE0120DE13C0606268
:10548000CE01A0DE84E991E10E9461AD6F8560628A
:10549000CE0198DE86E990E00E9461AD6F85606282
:1054A000CE0190DE6F856062CE018CDE8CE390E0F1
:1054B0000E9461AD84E0888BCE01BEDE8CE390E07B
:1054C0000E9461ADCE0186DE80E496E00E9461AD6F
:1054D00082E0898B66E0CE0175DE8CE390E00E946D
:1054E00061AD40E068E0CE017BDE6AE973E0CE01A9
:1054F0000E949BB141E068E0CE0172DE6AE973E090
:10550000CE010E949BB142E066E0CE0169DE68E90F
:1055100073E0CE01DF91CF910C949BB1CF92DF92DB
:10552000EF92FF920F931F93CF93DF931F921F92DF
:10553000CDB7DEB78C01677088E0689FB001112499
:105540006064C80149835A833DDE4981C42E5A8173
:10555000D52EE12CF12CD6016D916D01D801ED9184
:10556000FC910190F081E02DC8011995BFEFEB1A75
:10557000FB0AE8E0EE16F10471F70F900F90DF914F
:10558000CF911F910F91FF90EF90DF90CF900895F2
:1055900041E0F2DD81E090E008952F923F924F923A
:1055A0005F926F927F928F929F92AF92BF92CF92B3
:1055B000DF92EF92FF920F931F93CF93DF93CDB7BC
:1055C000DEB7CF54D1090FB6F894DEBF0FBECDBF02
:1055D0001C017E8F6D8F4A012FAB09AF2896EFAE6D
:1055E00028972C96ACAEBDAECEAEDFAE2C9734E095
:1055F000239F50011124FC01EA0DFB1D8081918144
:10560000A281B381898F9A8FAB8FBC8FDA01AA0DEB
:10561000BB1DBCAFABAF4D905D906D907C90A30176
:105620009201698D7A8D8B8D9C8D0E94A4B12196FB
:105630006CAF7DAF8EAF9FAF2197B4E00B9F800121
:105640001124F101E00FF11F20813181428153814A
:105650002F8F38A349A35AA3A401400F511F2396AB
:105660005FAF4EAF2397DA01CD90DD90ED90FC90C7
:10567000A70196016F8D78A189A19AA10E94A4B17A
:1056800027966CAF7DAF8EAF9FAF27972896EFAD73
:105690002897B4E0EB9FC0011124F101E80FF91F36
:1056A00020813181428153812BA33CA34DA35EA372
:1056B000ED8DFE8DE80FF91F6081718182819381EC
:1056C0000E94A3B16FA378A789A79AA7AD8DBE8DBD
:1056D0001C968D919D910D90BC91A02D60968CAFE4
:1056E0009DAFAEAFBFAF6097D1011C962D913D919C
:1056F0004D915C911F972BA73CA74DA75EA7A301D7
:10570000920150582D8B3E8B4F8B588FD701C6017D
:10571000B058898B9A8BAB8BBC8BED8DFE8DEA0DCF
:10572000FB1D20813181428153812FA738AB49ABCA
:105730005AAB21962CAD3DAD4EAD5FAD21976FA517
:1057400078A989A99AA90E94A3B16B017C01ED8D6A
:10575000FE8DE00FF11F80819181A281B3818BAB1F
:105760009CABADABBEAB27962CAD3DAD4EAD5FADAA
:105770002797BC01CD010E94A3B14B015C01A70199
:1057800096016D897E898F89988D0E9452B52B0173
:105790003C01A501940169897A898B899C890E94C1
:1057A00052B59B01AC01C301B2010E94A4B12B010F
:1057B0003C01A50194016D897E898F89988D0E9495
:1057C00052B54B015C01A701960169897A898B89E1
:1057D0009C890E9452B59B01AC01C501B4010E9495
:1057E000A3B1A30192010E9417B26B017C0120E0DA
:1057F00030E0A9010E947DB287FF0AC02BED3FE097
:1058000049EC50E4C701B6010E94A4B16B017C01D0
:10581000AA968FADAA97882351F02BED3FE049EC73
:1058200050E4C701B6010E94A3B16B017C012FA512
:1058300038A949A95AA9698D7A8D8B8D9C8D0E94B2
:105840007DB281111FC02BA93CA94DA95EA96F8D06
:1058500078A189A19AA10E947DB2811113C020E094
:1058600030E0A901C701B6010E947DB281110AC0D2
:105870002BED3FE049EC50E4C701B6010E94A4B112
:105880006B017C01A9962CAD3DAD4EAD5FADA997E6
:10589000C701B6010E9452B52FA138A549A55AA546
:1058A0005F770E948DB44B015C012FE632E143E843
:1058B0005AE30E947DB287FDC8C1C501B4010E94B0
:1058C0005AB30E94F1B27A8F698FDB01AB2B21F4BE
:1058D000E1E0F0E0FA8FE98F298D3A8DB90180E09F
:1058E00090E00E941DB34B015C019B01AC01C7011C
:1058F000B6010E9484B22B013C01A50194016FA165
:1059000078A589A59AA50E9484B26FA778AB89ABC8
:105910009AAB2BA53CA54DA55EA560966CAD7DAD63
:105920008EAD9FAD60970E94A3B1A50194010E9426
:1059300084B26BAB7CAB8DAB9EAB20E030E040E043
:105940005FE3C301B2010E9452B5A30192010E941C
:1059500052B59B01AC0160E070E080E89FE30E94DB
:10596000A3B16FA378A789A79AA7CE010196FC01DE
:1059700028964FAD289734E0439FE00DF11D112488
:105980002BA13CA14DA15EA120833183428353838F
:105990002BA53CA54DA55EA52D873E874F87588B2F
:1059A000B12C41E050E058A34F8F1C01BFA9A4E0E7
:1059B000BA9F800D911D112498AF8FAB910159AD05
:1059C00044E0549F200D311D11243AAF29AFFCA7AC
:1059D000EBA74F8D58A1898D9A8D4817590708F06C
:1059E0001AC188E18B150CF444C02FA138A549A534
:1059F0005AA569897A898B899C890E9452B56B0165
:105A00007C01A30192016D897E898F89988D0E9406
:105A100052B5A70196010E94A4B1A62E172F982E69
:105A2000892E2FA138A549A55AA56D897E898F8910
:105A3000988D0E9452B56B017C01A3019201698986
:105A40007A898B899C890E9452B59B01AC01C70160
:105A5000B6010E94A3B16D8B7E8B8F8B988FB39410
:105A60008A2D912FA92DB82D898B9A8BAB8BBC8B4E
:105A70006CC0AF8DB8A1BD0180E090E00E941DB365
:105A8000A30192010E9452B56B017C010E9481B278
:105A9000698B7A8B8B8B9C8BC701B6010E94B5B545
:105AA0004B015C01EBADFCADC080D180E280F380A6
:105AB000F7FAF094F7F8F0942396AEADBFAD2397C4
:105AC0002D913D914D915C912BA33CA34DA35EA3E1
:105AD00029893A894B895C89C701B6010E9452B570
:105AE0006D8B7E8B8F8B988FA50194016BA17CA110
:105AF0008DA19EA10E9452B59B01AC016D897E894A
:105B00008F89988D0E94A4B16D8B7E8B8F8B988F1F
:105B1000A5019401C701B6010E9452B56B017C0139
:105B200029893A894B895C896BA17CA18DA19EA1B1
:105B30000E9452B59B01AC01C701B6010E94A3B1FE
:105B4000698B7A8B8B8B9C8BB12C2D893E894F89ED
:105B5000588D21966CAD7DAD8EAD9FAD21970E9485
:105B6000A4B1EFA9F8AD60837183828393832989FF
:105B70003A894B895C8927966CAD7DAD8EAD9FAD22
:105B800027970E94A4B1A9ADBAAD6D937D938D9373
:105B90009C9313972FA538A949A95AA9EBA5FCA551
:105BA00060817181828193810E94A4B1ABA5BCA563
:105BB0006D937D938D939C9313972BA93CA94DA92D
:105BC0005EA96D857E858F8598890E94A4B16D87B9
:105BD0007E878F87988BC1010E948942FE01E6591A
:105BE000FF4F6F012C96ECACFDAC0EAD1FAD2C97AA
:105BF0009E01235F3F4FAE01475F5F4FBE016B5F6A
:105C00007F4FC1010E94549E2F8D38A12F5F3F4FBF
:105C100038A32F8FDECE2D8D3E8D245F3F4F4D8DCF
:105C20005E8D485F5F4F6D8D7E8D6C5F7F4FDE01B7
:105C3000A659BF4F6D012C96ECACFDAC0EAD1FAD5F
:105C40002C978D8D9E8D0E94549EC15BDF4F0FB6A9
:105C5000F894DEBF0FBECDBFDF91CF911F910F91A2
:105C6000FF90EF90DF90CF90BF90AF909F908F907C
:105C70007F906F905F904F903F902F900895FC0120
:105C800014821782138212828AED95E091838083B9
:105C900008952AED35E0FC013183208327812223FA
:105CA00019F004960C94FE130895CF92DF92EF92B0
:105CB000FF920F931F93CF93DF93EC01875B9F4F6E
:105CC000DEDFCE0186599F4FDADF7E0129E8E20E42
:105CD000F11C87016E0131E4C31A3EEFD30AC801FB
:105CE000CEDF015E1F4F0C151D05C9F7FE01EF53F6
:105CF000FE4F89E1818314823596178ACE018C513B
:105D00009E4FBDDFFE01EB56FD4F108211821282C5
:105D10001382389610821182128213821A821B8299
:105D2000188219826E0187E6C81A8DEFD80AF6012B
:105D30001082118212821382F80111821082FE01F8
:105D4000ED5FFD4F108286E391E0F7019C01119217
:105D500021503040E1F7FE01EF55FD4F81E0808397
:105D6000C95BDF4F198218820E940EAD68577C4EC6
:105D70008F4F9F4FF6016083718382839383DF91FE
:105D8000CF911F910F91FF90EF90DF90CF900895EA
:105D9000FC0120E03EE2DB014C91403241F0283032
:105DA00011F430833196DB014C91408331962F5FA3
:105DB0006F5F7F4F2B3079F7108208952F923F92BB
:105DC0004F925F926F927F928F929F92AF92BF920B
:105DD000CF92DF92EF92FF920F931F93CF93DF93B7
:105DE000CDB7DEB7CA58D1090FB6F894DEBF0FBEE3
:105DF000CDBF8C016B017A014901CA57DF4F188270
:105E0000C658D04084E0E80EF11C180191E1290E3B
:105E1000311CF801EA5BFF4FC957DF4FF983E88374
:105E2000C758D0403801FEE56F1AFDEF7F0A5801D0
:105E30008CE5A81A8DEFB80A80E4482E512C4C0E40
:105E40005D1E94E0490E511CA101BE016F5F7F4FA2
:105E5000C7010E94681218160CF03CC12C85322F25
:105E60003871303109F09EC0F30180819181019732
:105E7000029708F497C0BE016F5F7F4FCE0187582D
:105E80009F4F86DFA0961FAEA097F60180818111FB
:105E900007C065E773E0CE01815A9F4F0E94F5B9B4
:105EA000B601CE01815A9F4F0E94F5B9BE016758D5
:105EB0007F4FCE01815A9F4F0E94F5B965E773E08D
:105EC000CE01815A9F4F0E94F5B9CE01805C9F4F51
:105ED000D6DE21E0AE0147585F4FB701C2010E94F4
:105EE000F515811139C0F30180819181892BA1F5CC
:105EF000E0EBFEE08491882341F09091C00095FF93
:105F0000FCCF8093C6003196F5CFE7E7F3E08191AF
:105F1000882339F09091C00095FFFCCF8093C60094
:105F2000F6CF8091C00085FFFCCF8AE08093C60049
:105F3000FE01E758FF4F8191882339F09091C0000E
:105F400095FFFCCF8093C600F6CF8091C00085FFFF
:105F5000FCCF8AE08093C6008BE1FE01EC5BFF4F33
:105F6000DE01959601900D928A95E1F724968EAD0B
:105F70009FAD24979CA38BA38AED95E09AA389A358
:105F800020E030E0AE014F5D5F4FBE01615A7F4FB0
:105F9000C80114DFCE0181967CDECE01805C9F4F6C
:105FA00078DE52CF8981882309F494C08E3209F4B7
:105FB0004BCF8F3509F448CFF80181898E3209F42F
:105FC00043CF8F3509F440CF23FD3ECF81E0303100
:105FD00009F080E0C957DF4FE881F981C758D04008
:105FE0008083811108C08985873409F02DCF8A8587
:105FF0008E3709F429CF98012C5F3F4FBE016F5FA8
:106000007F4FC901C757DF4F2883C958D040C657B3
:10601000DF4F3883CA58D040BBDEF30180819181C5
:10602000C757DF4F2881C958D040C657DF4F388146
:10603000CA58D0400097F1F4F6018191882339F0D5
:106040009091C00095FFFCCF8093C600F6CFF90178
:106050008191882339F09091C00095FFFCCF809307
:10606000C600F6CF8091C00085FFFCCF8AE0809308
:10607000C600EACE8130910539F4F5018081918125
:10608000019691838083E0CE029709F0DDCE8114E2
:10609000910439F0B901C4010E94E2B9892B71F46D
:1060A00019C0CA57DF4FF881C658D0402F2F30E0B3
:1060B000F501808191812817390761F0CA57DF4FB8
:1060C000F881C658D040FF5FCA57DF4FF883C658E3
:1060D000D040BACEC657DF4F0FB6F894DEBF0FBE22
:1060E000CDBFDF91CF911F910F91FF90EF90DF9087
:1060F000CF90BF90AF909F908F907F906F905F9068
:106100004F903F902F9008950F931F93CF93DF935D
:10611000CDB7DEB76F970FB6F894DEBF0FBECDBF19
:106120008C01FC01EE55FD4F1182108240E050E0E1
:10613000BA01835B9F4F0E941B13C801875B9F4F6F
:106140002BE1FC013496DE01159601900D922A9503
:10615000E1F7FC01828193819C838B838AED95E03A
:106160009A83898320E030E0AE014F5F5F4F6EE994
:1061700073E0C80123DECE0101968BDD6F960FB66A
:10618000F894DEBF0FBECDBFDF91CF911F910F916D
:1061900008952BE1FB013496DC01149601900D92D9
:1061A0002A95E1F7FB0122813381FC0133832283AD
:1061B0000895EF92FF920F931F93CF93DF93EC011B
:1061C0001B82FC01E05BFF4F8081882329F0CE0118
:1061D000835B9F4F0E94FE137E018FE3E81A8EEFD0
:1061E000F80A45E360E0C7010E94DE3B81111FC051
:1061F000E0EBFEE08491882341F09091C00095FF90
:10620000FCCF8093C6003196F5CFE8ECF6E08491A0
:10621000882341F09091C00095FFFCCF8093C60089
:106220003196F5CF8091C00085FFFCCF77C08E01FD
:106230000A531E4F41E0B701C8010E94CC1B8111D7
:1062400026C040E0B701C8010E94CC1B81111FC0CD
:10625000E6EBFEE08491882341F09091C00095FF29
:10626000FCCF8093C6003196F5CFE5EBF6E0849144
:10627000882341F09091C00095FFFCCF8093C60029
:106280003196F5CF8091C00085FFFCCF47C0B801A3
:10629000CE01835B9F4F0E940B1181111FC0E6EB63
:1062A000FEE08491882341F09091C00095FFFCCFDF
:1062B0008093C6003196F5CFE5EAF6E08491882315
:1062C00041F09091C00095FFFCCF8093C6003196BD
:1062D000F5CF8091C00085FFFCCF20C081E08B838B
:1062E000E0EBFEE08491882341F09091C00095FF9F
:1062F000FCCF8093C6003196F5CFEAE9F6E08491B1
:10630000882341F09091C00095FFFCCF8093C60098
:106310003196F5CF8091C00085FFFCCF8AE0809355
:10632000C6008E01075B1F4FB801CE0186599F4FF3
:1063300030DFC859DF4F19830883DF91CF911F9158
:106340000F91FF90EF900895FC011282138208953F
:10635000FC012381222311F021E022830895FC0116
:106360002281211112820895AF92BF92CF92DF92C3
:10637000EF92FF920F931F93CF93DF931F92CDB7AE
:10638000DEB78C018FE2FB0181935F01D12C41E0EC
:106390007801F1E4EF1AFEEFFF0A9FE1C92E2D2DDF
:1063A00030E0F7018081918128173907D8F4C29E27
:1063B000C001C39E900D112483579F4FB501800FDC
:1063C000911F49830E94B210C50149815C01019669
:1063D000F5012081222321F04D3810F44F5FF6CFD4
:1063E000D394DDCF47FD11C0B501C80188519E4F40
:1063F0000F90DF91CF911F910F91FF90EF90DF9061
:10640000CF90BF90AF900C94B210F50110820F9016
:10641000DF91CF911F910F91FF90EF90DF90CF9080
:10642000BF90AF9008953F924F925F926F927F928C
:106430008F929F92AF92BF92CF92DF92EF92FF9294
:106440000F931F93CF93DF93CDB7DEB7AC970FB603
:10645000F894DEBF0FBECDBF7C015B01FC018381E0
:10646000882309F408C1C70188519E4F0E94FE137A
:10647000F7011282CE0101966C0101DC270198E63A
:10648000490E511CC701875B9F4FF20191838083A6
:10649000F50180818F3209F084C06FE270E0C501A0
:1064A0000E9400BA8C010F5F1F4F2AE0322E0115A7
:1064B000110509F47CC06FE270E0C8010E9400BAC7
:1064C0004C01009709F474C00817190708F070C050
:1064D0003C01601A710AA301B801CE0180960E94A6
:1064E00029BAE0E2F0E0EC0FFD1FE60DF71D108287
:1064F000FE01B0968191882339F09091C00095FFFC
:10650000FCCF8093C600F6CF8091C00085FFFCCF02
:106510003092C600F201608171816115710519F038
:106520006C5F7F4F02C060E070E021E0AE01405E32
:106530005F4FCE0105960E94F51581112BC0EFE744
:10654000F5E08491882341F09091C00095FFFCCF45
:106550008093C6003196F5CFFE01B09681918823D5
:1065600039F09091C00095FFFCCF8093C600F6CF24
:10657000EDE7F5E08491882341F09091C00095FF0C
:10658000FCCF8093C6003196F5CF8091C00085FF87
:10659000FCCF6CC0F201D182C08284010F5F1F4F1B
:1065A00086CFC70186599F4FF20191838083850171
:1065B000F20180819181009711F0049602C080E081
:1065C00090E0B8010E94CB16882339F1EFE6F5E0A0
:1065D0008491882341F09091C00095FFFCCF809377
:1065E000C6003196F5CFF8018191882339F090915A
:1065F000C00095FFFCCF8093C600F6CF8091C0000D
:1066000085FFFCCF8AE08093C600F701E356FD4F7B
:1066100010821182128213822CC0E7E5F5E084918A
:10662000882341F09091C00095FFFCCF8093C60075
:106630003196F5CFF8018191882339F09091C0000F
:1066400095FFFCCF8093C600F6CFE5E5F5E0849199
:10665000882341F09091C00095FFFCCF8093C60045
:106660003196F5CF8091C00085FFFCCF8AE0809302
:10667000C600C6010EDBAC960FB6F894DEBF0FBEA7
:10668000CDBFDF91CF911F910F91FF90EF90DF90E1
:10669000CF90BF90AF909F908F907F906F905F90C2
:1066A0004F903F9008958F929F92AF92BF92CF925A
:1066B000DF92EF92FF92CF93DF931F92CDB7DEB7B9
:1066C0007C01FC018281882309F4AFC0719681911D
:1066D000882339F09091C00095FFFCCF8093C600CD
:1066E000F6CFE3E5F5E08491882341F09091C00076
:1066F00095FFFCCF8093C6003196F5CFE1E4F5E03D
:106700008491882341F09091C00095FFFCCF809345
:10671000C6003196F5CFF701E356FD4F4081518118
:10672000628173812AE030E089EC9DE00E940A8E4C
:10673000EFE3F5E08491882341F09091C00095FF4C
:10674000FCCF8093C6003196F5CFF701EB56FD4F95
:1067500040815181628173812AE030E089EC9DE0C3
:106760000E940A8E8091C00085FFFCCF8AE0809352
:10677000C6000E940EAD30E6C32E3AEED32EE12CB9
:10678000F12CA70196010E945BB649015A01609164
:106790007208709173088091740890917508A70130
:1067A00096010E945BB6821A930AC4016CE370E002
:1067B0000E9434B66983CE0101960E94227AFC01C0
:1067C0002191CF01222339F03091C00035FFFCCF59
:1067D0002093C600F4CF40E050E06AE389EC9DE0EE
:1067E0000E94C28DC4016CE370E00E9434B68983BC
:1067F000CE0101960E94227AFC012191CF01222331
:1068000039F03091C00035FFFCCF2093C600F4CFA3
:10681000EDE3F5E084918823E1F09091C00095FFCD
:10682000FCCF8093C6003196F5CFE0E3F5E084918C
:10683000882341F09091C00095FFFCCF8093C60063
:106840003196F5CF8091C00085FFFCCF8AE0809320
:10685000C6000F90DF91CF91FF90EF90DF90CF9027
:10686000BF90AF909F908F900895AF92BF92CF92BC
:10687000DF92EF92FF920F931F93CF93DF935C0110
:10688000EB01FB0101900020E9F78F010150110994
:10689000061B170B6C01F8E1CF1AFEEFDF0AF601B9
:1068A00010826EE470E0CE010E9400BA7C01009775
:1068B00029F4F8013197EC0FFD1F0DC060E270E084
:1068C0000E9400BAEC0121966AE270E0C7010E94C2
:1068D00000BAFC0131978DE081838AE082831382C4
:1068E000BE01C5018C519E4F0E94C78EF60180816A
:1068F000882309F1E6EBFEE08491882341F0909132
:10690000C00095FFFCCF8093C6003196F5CFEAE139
:10691000F5E08491882341F09091C00095FFFCCF71
:106920008093C6003196F5CF8091C00085FFFCCFE3
:106930008AE08093C600DF91CF911F910F91FF9065
:10694000EF90DF90CF90BF90AF9008952F923F923D
:106950004F925F926F927F928F929F92AF92BF926F
:10696000CF92DF92EF92FF920F931F93CF93DF931B
:10697000CDB7DEB7CC55D1090FB6F894DEBF0FBE48
:10698000CDBF4C018C010F551D4F662339F0F80126
:106990001082F401838181111DC015C0F80180812E
:1069A000882309F4AFC0F401E756FD4FC080D180C1
:1069B000E280F3800E940EADC616D706E806F906FF
:1069C00008F4A0C0E4CFC401F4DBF4018381882380
:1069D00009F498C07401F7E4EF0EF11CF70181810E
:1069E0008F9380818F9381E195E09F938F938E01A8
:1069F000015C1F4F1F930F930E9438BA0F900F90A6
:106A00000F900F900F900F90B12CF8010190002083
:106A1000E9F73197E01BF10BBE1684F46801CB0C4B
:106A2000D11CB7FCDA94F6018081992787FD9095F7
:106A30000E9475B9F6018083B394E7CFFDE48F0E11
:106A4000911C40E050E0BA01C4010E941B13512C7C
:106A5000CE0101966C014AE0642E45E0742E5E0181
:106A600091E2A90EB11C40E050E0B601C4010E94C1
:106A700068121816DCF5412CF60101900020E9F7A8
:106A80003197EC19FD094E1674F41601240C311CD3
:106A900047FC3A94F101808190E00E9475B9F101C0
:106AA00080834394E9CF8A858E37E9F245E050E050
:106AB000B801C6010E941BBA892BA9F61F930F9338
:106AC0007F926F92BF92AF920E9438BAC5010E9426
:106AD000DF3E86E095E00E94523F0F900F900F90AE
:106AE0000F900F900F9055245394BDCF511004C0B8
:106AF0008FEF9FEFF70104C0F7018081918101962C
:106B000091838083C45ADF4F0FB6F894DEBF0FBE67
:106B1000CDBFDF91CF911F910F91FF90EF90DF904C
:106B2000CF90BF90AF909F908F907F906F905F902D
:106B30004F903F902F9008950F931F93CF93DF9323
:106B4000EC018C0108511E4FC8010E94B413C8010A
:106B50000E94FE1318821982DF91CF911F910F912D
:106B60000895CF92DF92EF92FF920F931F93CF93EE
:106B7000DF93CDB7DEB76F970FB6F894DEBF0FBEC9
:106B8000CDBF8C016A017C0188E6E80EF11CC801CA
:106B900086599F4FF70191838083E65CFD4F22E089
:106BA00030E03183208332967183608340E050E08F
:106BB000BA0104960E941B13F701808191812BE199
:106BC000FC013496DE01159601900D922A95E1F7AD
:106BD000FC01828193819C838B838AED95E09A836B
:106BE00089839601AE014F5F5F4F6EE973E0C80184
:106BF000E5D8CE0101964DD86F960FB6F894DEBF5A
:106C00000FBECDBFDF91CF911F910F91FF90EF90FD
:106C1000DF90CF9008952F923F924F925F926F92A4
:106C20007F928F929F92AF92BF92CF92DF92EF921C
:106C3000FF920F931F93CF93DF93CDB7DEB7AC973F
:106C40000FB6F894DEBF0FBECDBF8C016B01342EA2
:106C5000DC0113968C91882309F4EEC2F801E5510A
:106C6000FE4F8081882309F4F5C02111C1C078014D
:106C7000BDEFEB1AFB0AF7018081882361F1E6EB97
:106C8000FEE08491882341F09091C00095FFFCCFF5
:106C90008093C6003196F5CFE7E5F6E0849188232E
:106CA00041F09091C00095FFFCCF8093C6003196D3
:106CB000F5CF4AE050E061E070E089EC9DE00E9491
:106CC000DE8D8091C00085FFFCCF8AE08093C600F6
:106CD0000E944146B1C2E0EBFEE08491882341F07E
:106CE0009091C00095FFFCCF8093C6003196F5CF00
:106CF000EEE3F6E08491882341F09091C00095FF87
:106D0000FCCF8093C6003196F5CFF60181918823A0
:106D100039F09091C00095FFFCCF8093C600F6CF6C
:106D2000E3E3F6E08491882341F09091C00095FF61
:106D3000FCCF8093C6003196F5CFD7018C916DE8DA
:106D4000B62EB801B89E600D711D1124685F7D4F8D
:106D5000C8010ADBF7018081F801B89EE00DF11D42
:106D60001124E85FFD4F8191882339F09091C00094
:106D700095FFFCCF8093C600F6CFEDE2F6E084915C
:106D8000882341F09091C00095FFFCCF8093C6000E
:106D90003196F5CF5801F3E6AF1AFDEFBF0AD501E2
:106DA0004D915D916D917C912AE030E089EC9DE000
:106DB0000E940A8E8091C00085FFFCCF8AE08093FC
:106DC000C600F7012081F80184E0289FE00DF11D45
:106DD0001124EC5FFD4FD5014D915D916D917C913A
:106DE00040835183628373832F5FF70120832CC01C
:106DF000E0EBFEE08491882341F09091C00095FF84
:106E0000FCCF8093C6003196F5CFECE1F6E084919B
:106E1000882341F09091C00095FFFCCF8093C6007D
:106E20003196F5CFF6018191882339F09091C00019
:106E300095FFFCCF8093C600F6CF8091C00085FF00
:106E4000FCCF8AE08093C600C80188519E4F0E9403
:106E5000FE1330C0F801ED5FFD4F1082E0EBFEE065
:106E60008491882341F09091C00095FFFCCF8093DE
:106E7000C6003196F5CFEBE0F6E08491882341F02F
:106E80009091C00095FFFCCF8093C6003196F5CF5E
:106E9000F6018191882339F09091C00095FFFCCFD5
:106EA0008093C600F6CF8091C00085FFFCCF8AE0BA
:106EB0008093C600D80112961C92FE0131965F01A4
:106EC000CF010E943F2E2801F8E64F0E511CC80149
:106ED000875B9F4FD2018D939C93F60180818F3207
:106EE00009F084C06FE270E0C6010E9400BA01960A
:106EF0007C015AE0252EE114F10409F47DC06FE213
:106F000070E0C7010E9400BA4C01009709F475C0F7
:106F1000E816F90608F071C03C016E187F08A3015D
:106F2000B701CE0180960E9429BAE0E2F0E0EC0FB2
:106F3000FD1FE60DF71D1082FE01B096819188239A
:106F400039F09091C00095FFFCCF8093C600F6CF3A
:106F50008091C00085FFFCCF2092C600D2016D91C8
:106F60007C916115710519F06C5F7F4F02C060E084
:106F700070E021E0AE01405E5F4FCE0105960E94B9
:106F8000F51581112BC0E7EFF5E08491882341F0DE
:106F90009091C00095FFFCCF8093C6003196F5CF4D
:106FA000FE01B0968191882339F09091C00095FF41
:106FB000FCCF8093C600F6CFE5EFF5E084918823FF
:106FC00041F09091C00095FFFCCF8093C6003196B0
:106FD000F5CF8091C00085FFFCCF02C1F201B182E4
:106FE000A0827401FFEFEF1AFF0A85CFC80186590E
:106FF0009F4FD2018D939C937601F801E851FE4F8B
:107000004F01332009F4B1C0D2016D917C9161151B
:10701000710519F06C5F7F4F02C060E070E021E005
:10702000A701C4010E94F515882309F474C0F40176
:1070300081899289A389B489F801EB56FD4F808339
:107040009183A283B383E7EEF5E08491D801AB5638
:10705000BD4F882349F09091C00095FFFCCF8093ED
:10706000C60031968491F5CFF7018191882339F0DC
:107070009091C00095FFFCCF8093C600F6CFEFED56
:10708000F5E08491882341F09091C00095FFFCCFFA
:107090008093C6003196F5CF4D915D916D917C91B5
:1070A0002AE030E089EC9DE00E940A8E8091C000C9
:1070B00085FFFCCF8AE08093C600F801E356FD4FC0
:1070C0001082118212821382E1EDF5E0849188230F
:1070D00041F09091C00095FFFCCF8093C60031969F
:1070E000F5CF8091C00085FFFCCF8AE08093C60079
:1070F000A70160E070E0C80134DDD80151968C91A1
:10710000882319F0C801419601C0C7010E945E732F
:107110008AE893E08CC0EDEBF5E08491882341F0A0
:107120009091C00095FFFCCF8093C6003196F5CFBB
:10713000F7018191882339F09091C00095FFFCCF31
:107140008093C600F6CFEBEBF5E08491882341F005
:107150009091C00095FFFCCF8093C6003196F5CF8B
:107160008091C00085FFFCCF3BC0F201608171813E
:107170006115710519F06C5F7F4F02C060E070E02F
:1071800026E5A701C4010E94F51581112DC0E7EA8B
:10719000F5E08491882341F09091C00095FFFCCFE9
:1071A0008093C6003196F5CFF7018191882339F09D
:1071B0009091C00095FFFCCF8093C600F6CFE5EA22
:1071C000F5E08491882341F09091C00095FFFCCFB9
:1071D0008093C6003196F5CF8091C00085FFFCCF2B
:1071E0008AE08093C60025C081E0D8018C93E3E952
:1071F000F5E08491882341F09091C00095FFFCCF89
:107200008093C6003196F5CFF6018191882339F03D
:107210009091C00095FFFCCF8093C600F6CF80917F
:10722000C00085FFFCCF8AE08093C600C7010E94A2
:107230005E73C5010E94492EAC960FB6F894DEBF6E
:107240000FBECDBFDF91CF911F910F91FF90EF90B7
:10725000DF90CF90BF90AF909F908F907F906F9076
:107260005F904F903F902F90089521E0FC01218383
:1072700040E0D1CCCF92DF92EF92FF920F931F9319
:10728000CF93DF93CDB7DEB76F970FB6F894DEBF1D
:107290000FBECDBF8C016C0128E6C20ED11C8659F1
:1072A0009F4FF60191838083E65CFD4F21E030E043
:1072B000318320837801FCE5EF1AFDEFFF0AF70127
:1072C0001182108240E050E0BA0104960E941B1324
:1072D000F601808191812BE1FC013496DE01159647
:1072E00001900D922A95E1F7FC01828193819C83A4
:1072F0008B838AED95E09A83898320E030E0AE01AC
:107300004F5F5F4F6EE973E0C8010E94DE2ECE0131
:1073100001960E94492EF701808191816F960FB6E8
:10732000F894DEBF0FBECDBFDF91CF911F910F91BB
:10733000FF90EF90DF90CF900895AF92BF92CF92E1
:10734000DF92EF92FF920F931F93CF93DF93CDB70E
:10735000DEB76F970FB6F894DEBF0FBECDBF8C01BE
:107360007B01CE0101960E943F2EF801EF58FF4F9E
:1073700080816801811104C029E4C20ED11C03C0C0
:107380008AE6C80ED11C21E0A701B6016C5F7F4FD1
:10739000CE0105960E94F51581112DC0E0EBFEE0AF
:1073A0008491882341F09091C00095FFFCCF809399
:1073B000C6003196F5CFE0EFF4E08491882341F0E8
:1073C0009091C00095FFFCCF8093C6003196F5CF19
:1073D000F7018191882339F09091C00095FFFCCF8F
:1073E0008093C600F6CF8091C00085FFFCCF8AE075
:1073F0008093C60036C0F801E154FE4F8081918130
:107400008A30910530F59C012F5F3F4F31832083F7
:107410002FE1289F7001299FF00C112429E8E20E2A
:10742000F11CE00EF11E5C01B701C7014F960E94EE
:10743000C93081E0A81AB1082FE1E21AF1088FEFF4
:10744000A816B80689F7B601C80187579F4F0E9452
:10745000C930BE016F5F7F4FC80186599F4F0E94A0
:10746000C930CE0101960E94492E6F960FB6F8944E
:10747000DEBF0FBECDBFDF91CF911F910F91FF9067
:10748000EF90DF90CF90BF90AF900895EF92FF9272
:107490000F931F93CF93DF93EC01C154DE4F2881EC
:1074A000398121153105F9F02150310939832883BB
:1074B0008C0107571F4FB80186599F4F0E94C93052
:1074C000C80100E010E07C012FE1E20EF11C2881F0
:1074D00039810217130738F40F5F1F4FB7010E945D
:1074E000C930C701F0CFDF91CF911F910F91FF906D
:1074F000EF900895EF92FF920F931F93CF93DF9336
:10750000EC010E94C1968E010D5F1D4FF801808134
:107510009E0128513E4F79018823A1F1C9010E94A3
:10752000FE13F801808181508083BE01FDE88F9FAA
:10753000600D711D1124685F7D4F21E041E0CE0197
:107540006ADBF8018081FE0124E0829FE00DF11DDD
:107550001124EC5FFD4F4081518162817381FE01F6
:10756000E356FD4F4083518362837383C7010E94BA
:107570001B13CE01DF91CF911F910F91FF90EF90E0
:107580000C94A8310E943797C7010E94FE131A82FB
:1075900084EE94E0DF91CF911F910F91FF90EF90D7
:1075A00081C48FEF8EBD0DB407FEFDCF8EB508955B
:1075B0008EBD0DB407FEFDCF089561E0FC01808112
:1075C0000C9467ACFC012281322F306A36953CBDA9
:1075D00020FD06C031E0263009F430E0232F01C041
:1075E00020E02DBD60E0FC0180810C9467ACCF925F
:1075F000DF92EF92FF920F931F93CF93DF93EC01F3
:107600008B017A010E940EAD6B01CBDF8B838F3F24
:1076100049F40E940EAD6C197D096D327140A8F3DA
:1076200081E144C08E3F11F08FE040C0E114F104CD
:10763000D9F0C70101972FEF2EBDF8014FEF9F0141
:10764000201B310B2817390738F40DB407FEFDCF86
:107650002EB521934EBDF3CF0DB407FEFDCF2EB551
:10766000F801E80FF91F2083D801E00EF11EC12CAC
:10767000D12CAE15BF0579F08D91ED2DFF27E827B0
:10768000EE0FFF1FEB52F94F85919491DC2CCC2427
:10769000C826D926EECF85DF082F10E0102F00274F
:1076A00080DF082BC016D10631F080E28983CE013D
:1076B00084DF80E003C0CE0180DF81E0DF91CF91E5
:1076C0001F910F91FF90EF90DF90CF9008950F934F
:1076D0001F93CF93DF93EB010E940EAD8B0161DF0F
:1076E0008F3F49F00E940EAD601B710B6C177D0738
:1076F000B0F380E001C081E0DF91CF911F910F9145
:107700000895CF92DF92FF920F931F93CF93DF9351
:1077100000D01F92CDB7DEB76C01F62E29833A83D5
:107720004B835C834FDF6CE271E0C601D0DF8F2DAD
:1077300080643EDF08E110E05C814B813A81298161
:10774000DA01C901002E04C0B695A79597958795D3
:107750000A94D2F729833A834B835C8329DF08504C
:10776000110929813A814B815C81083F8FEF18070D
:1077700039F7FF2029F0E8E0FE1621F08FEF03C073
:1077800085E901C087E814DFFCE0FF1201C009DFD2
:1077900010E007DFF601838387FF04C01F3F11F06D
:1077A0001F5FF7CF0F900F900F900F90DF91CF9149
:1077B0001F910F91FF90DF90CF900895BF92CF92CD
:1077C000DF92EF92FF920F931F93CF93DF93EC0121
:1077D000B62E1C82198248830E940EAD8B0161E097
:1077E00088810E942EACCE01E8DE60E082E30E9438
:1077F0002EAC61E083E30E942EAC61E084E30E9442
:107800002EAC61E085E30E942EAC61E085E30E942E
:1078100067AC85E08A8382E58CBD1DBC6AE0F62EEC
:107820008FEFC6DEFA94E1F720E030E0A90160E0D6
:10783000CE0167DFF82E8B8381E0F81649F00E94B5
:107840000EAD601B710B613D774070F381E046C067
:107850002AEA31E040E050E068E0CE0152DF82FFEA
:1078600002C0FC820CC054E0F52E9BDE8B83FA94A0
:10787000E1F78A3A11F082E031C082E08C838C819A
:10788000823031F4C12CD12CE12C40E4F42E03C021
:10789000C12CD12C760120E030E0A90167E3CE01B4
:1078A00030DFA701960169E2CE012BDF8B838823AD
:1078B00049F00E940EAD601B710B613D774058F39B
:1078C0008AE00CC08C818230B1F420E030E0A90164
:1078D0006AE3CE0116DF882329F088E08983CE0190
:1078E0006CDE14C05EDE807C803C11F483E08C830F
:1078F00058DE57DE56DECE0160DE86E08B1518F4CA
:1079000088E1898303C0BA8281E001C080E0DF9111
:10791000CF911F910F91FF90EF90DF90CF90BF908C
:107920000895AF92BF92CF92DF92EF92FF920F93A2
:107930001F93CF93DF93EC016A017B0189018C8156
:10794000833039F0F9E0CC0CDD1CEE1CFF1CFA95FD
:10795000D1F773E0B72EE4E0AE2EBA94A7019601FA
:1079600061E1CE01CEDE882311F0A98207C040E09C
:1079700052E0B801CE013BDE81110EC0CE01BB202A
:1079800049F01BDE20E030E0A9016CE0CE01B9DE59
:107990001982E3CF12DE80E0DF91CF911F910F912A
:1079A000FF90EF90DF90CF90BF90AF900895CF936E
:1079B000DF93EC016EBD20E030E00DB407FEFDCF9B
:1079C000FA01E20FF31F80818EBD0DB407FEFDCFDB
:1079D00081818EBD2E5F3F4F211582E0380769F708
:1079E0000DB407FEFDCF8FEFE3DD8FEFE1DDD9DDD5
:1079F0008B838F71853031F083E18983CE01DDDDAA
:107A000080E001C081E0DF91CF9108950F931F9333
:107A1000CF93DF93EC0189018C81833039F0B9E099
:107A2000440F551F661F771FBA95D1F79A01AB0116
:107A300068E1CE0166DE882311F086E01EC0A80151
:107A40006EEFCE01B4DF8823C9F068E572E0CE01A5
:107A50003EDE182F811102C087E10FC020E030E028
:107A6000A9016DE0CE014DDE811106C09ADD8111C4
:107A700003C0CE01A2DD05C086E18983CE019DDD74
:107A800010E0812FDF91CF911F910F910895FC019C
:107A9000659175918591949108952F923F924F929F
:107AA0005F926F927F928F929F92AF92BF92CF928E
:107AB000DF92EF92FF920F931F93CF93DF9300D04B
:107AC00000D0CDB7DEB71C01FC01EF58F14F149187
:107AD0009C01220F331F220F331F3E832D832C590D
:107AE000354F4901F901108211821282138220E779
:107AF0003AE04CE65AE068E67AE084E69AE00E94D2
:107B00001BA88D819E818058914FC1DF6B017C0144
:107B1000612F772767FD7095872F972F0E941FB3DE
:107B20002B013C012D813E81215D354F590120E023
:107B300030E040EC5FE3C701B6010E9452B5A301FB
:107B400092010E9452B5F501608371838283938311
:107B50002D813E81215A3D4F3C832B83F901608169
:107B600071818281938160932102709322028093BC
:107B700023029093240220E030E040E752E40E9488
:107B800084B220E5C22E2AE0D22E7B018C012BE3A9
:107B90003AE047E35AE063E37AE08FE29AE00E943A
:107BA000549E0E94C196F4011082118212821382A7
:107BB00020E73AE04CE65AE068E67AE084E69AE0AC
:107BC0000E941BA82D813E812C58314F3A83298376
:107BD000C9015DDF9058A30192010E9452B5F501E1
:107BE000608371838283938320E030E040E752E436
:107BF00060912102709122028091230290912402CF
:107C00000E9484B27B018C012BE33AE047E35AE007
:107C100063E37AE08FE29AE00E94549E0E94C1964C
:107C200089819A8134DF9B01AC010E94A4B1A30138
:107C300092010E9452B5F501608371838283938320
:107C400020E030E040E05FE3EB81FC816081718106
:107C5000828193810E9452B5609321027093220227
:107C6000809323029093240220E030E040E752E426
:107C70000E9484B27B018C012BE33AE047E35AE097
:107C800063E37AE08FE29AE00E94549E0E94C196DC
:107C90008D819E818457914FFADE0D811E81085A95
:107CA000154FF80120813181428153810E94A4B196
:107CB000F40160837183828393838D819E818C55CF
:107CC000914FE5DE2D813E812D5B3D4F7901F8011D
:107CD00020813181428153810E94A4B1F7016083E8
:107CE0007183828393838D819E818856914FCFDEED
:107CF0002D813E81295C3D4F7901F8012081318140
:107D0000428153810E94A4B1F70160837183828311
:107D10009383F40180819181A281B381F5018083F5
:107D20009183A283B38310922102109222021092B7
:107D30002302109224020E946E8FF101EB5AF54F3C
:107D400081E0808326960FB6F894DEBF0FBECDBFCC
:107D5000DF91CF911F910F91FF90EF90DF90CF9027
:107D6000BF90AF909F908F907F906F905F904F905B
:107D70003F902F900895FC012491222341F03091EF
:107D8000C00035FFFCCF2093C6000196F4CF22E05F
:107D900030E089EC9DE00C94B48EFC012491222308
:107DA00041F03091C00035FFFCCF2093C600019612
:107DB000F4CF2AE030E089EC9DE00C940A8E20910B
:107DC000840830918508243031050CF06AC0409158
:107DD00086085091870860E6649F9001659F300D8A
:107DE0001124BC01C9018257974F0E9414BAE0EBDD
:107DF000FEE08491882341F09091C00095FFFCCF74
:107E00008093C6003196F5CFE6E6FEE084918823A4
:107E100041F09091C00095FFFCCF8093C600319651
:107E2000F5CF809186089091870820E6289FF00181
:107E3000299FF00D1124E257F74F8191882339F0E3
:107E40009091C00095FFFCCF8093C600F6CFE4E68A
:107E5000FEE08491882341F09091C00095FFFCCF13
:107E60008093C6003196F5CF8091C00085FFFCCF8E
:107E70008AE08093C60080918608909187080196D9
:107E800064E070E00E9448B690938708809386086B
:107E9000809184089091850801969093850880933D
:107EA0008408089520918408309185082430310594
:107EB0000CF06AC0409186085091870860E6649F84
:107EC0009001659F300D1124BC01C9018257974F65
:107ED0000E947DB9E0EBFEE08491882341F090910F
:107EE000C00095FFFCCF8093C6003196F5CFE9E541
:107EF000FEE08491882341F09091C00095FFFCCF73
:107F00008093C6003196F5CF8091860890918708BE
:107F100020E6289FF001299FF00D1124E257F74F2A
:107F20008191882339F09091C00095FFFCCF809318
:107F3000C600F6CFE7E5FEE08491882341F09091FA
:107F4000C00095FFFCCF8093C6003196F5CF80919D
:107F5000C00085FFFCCF8AE08093C6008091860830
:107F600090918708019664E070E00E9448B6909373
:107F700087088093860880918408909185080196EF
:107F8000909385088093840808959B9AA3980895F8
:107F9000FCDF40E052EC61E070E089EC9DE00E9483
:107FA000C28CE1E5FEE08491882341F09091C0000D
:107FB00095FFFCCF8093C6003196F5CF8091C0002D
:107FC00085FFFCCF8AE08093C60080EB9EE0FC0139
:107FD0002491222341F03091C00035FFFCCF209343
:107FE000C6003196F5CF24B720FF14C0E9E4FEE0C7
:107FF0003491332341F04091C00045FFFCCF3093D2
:10800000C6003196F5CF3091C00035FFFCCF3AE085
:108010003093C60021FF14C0E9E3FEE0349133231E
:1080200041F04091C00045FFFCCF3093C60031962F
:10803000F5CF3091C00035FFFCCF3AE03093C60059
:1080400022FF14C0E8E2FEE03491332341F0409176
:10805000C00045FFFCCF3093C6003196F5CF30917C
:10806000C00035FFFCCF3AE03093C60023FF14C0B8
:10807000E8E1FEE03491332341F04091C00045FF38
:10808000FCCF3093C6003196F5CF3091C00035FF5C
:10809000FCCF3AE03093C60025FF14C0E8E0FEE0D4
:1080A0002491222341F03091C00035FFFCCF209372
:1080B000C6003196F5CF2091C00025FFFCCF2AE005
:1080C0002093C60014BEE1E0FEE02491222341F09B
:1080D0003091C00035FFFCCF2093C6003196F5CF1C
:1080E000EBEFFDE02491222341F03091C00035FFF9
:1080F000FCCF2093C6003196F5CF2091C00025FF1C
:10810000FCCF2AE02093C600FC012491E0EBFEE0C6
:10811000222349F03091C00035FFFCCF2093C600E8
:1081200031962491F5CFEBEEFDE02491222341F02E
:108130003091C00035FFFCCF2093C6003196F5CFBB
:10814000E6EDFDE02491222341F03091C00035FF9F
:10815000FCCF2093C6003196F5CFEAECFDE02491E8
:10816000222341F03091C00035FFFCCF2093C600A0
:108170003196F5CFE3EBFDE02491222341F03091DD
:10818000C00035FFFCCF2093C6003196F5CF20917B
:10819000C00025FFFCCF2AE02093C600E8EAFDE0FE
:1081A0002491222341F03091C00035FFFCCF209371
:1081B000C6003196F5CFECE9FDE02491222341F091
:1081C0003091C00035FFFCCF2093C6003196F5CF2B
:1081D0002091C00025FFFCCF2AE02093C600FC01BF
:1081E0008491E0EBFEE0882349F09091C00095FF78
:1081F000FCCF8093C60031968491F5CFEDE8FDE089
:108200008491882341F09091C00095FFFCCF80932A
:10821000C6003196F5CF0E94359A4AE050E0BC0185
:1082200089EC9DE00E94DE8DE6E7FDE084918823E5
:1082300041F09091C00095FFFCCF8093C60031962D
:10824000F5CF4AE050E060ED74E089EC9DE00E94DB
:10825000DE8D8091C00085FFFCCF8AE08093C60050
:1082600010928A0810928B0810928C0810928D0838
:108270000E94E58A0E94B7860E9414210E94049EF3
:108280000E9423990E947377FFEF23ED80E3F15062
:1082900020408040E1F700C00000089580917E08F2
:1082A00090917F0860E070E001960C94D4B68091C4
:1082B0007E0890917F084AE050E060E070E001960F
:1082C0000C943CB8682F772767FD7095209188083B
:1082D0003091890840E6429FC001439F900D1124D0
:1082E0008257974F0E9400BA90937F0880937E0830
:1082F00021E0892B09F420E0822F08950E940EAD21
:1083000060937A0870937B0880937C0890937D0833
:1083100008950E940EAD60937A0870937B08809355
:108320007C0890937D08E0918808F0918908E657D1
:10833000F74F8081811114C0EDE7F9E08491882323
:1083400041F09091C00095FFFCCF8093C60031961C
:10835000F5CF8091C00085FFFCCF8AE08093C600F6
:10836000089589EC9DE00E94148DE0E8F9E0849185
:10837000882341F09091C00095FFFCCF8093C60008
:108380003196F5CF4091130A5091140A6091150A65
:108390007091160A4F5F5F4F6F4F7F4F2AE030E0BA
:1083A00089EC9DE00E94B38D8091C00085FFFCCFD9
:1083B0008AE08093C600ADCF8F929F92AF92BF921A
:1083C000CF92DF92EF92FF920F931F93CF93DF93A1
:1083D00034EDE32E34E0F32E04E61AE0CFE2DAE0E7
:1083E00049E7C42E4AE0D42EF70181917F016ADF6C
:1083F000882311F153DF4B015C01F601808181116B
:1084000003C060910E0A01C061E070E080E090E07E
:108410000E941FB3F80120813181428153810E9463
:1084200052B59B01AC01C501B4010E94A4B168839F
:1084300079838A839B8309C0F80180819181A2811D
:10844000B38188839983AA83BB830C5F1F4F2496D3
:10845000FFEFCF1ADF0A88EDE81684E0F80621F670
:1084600086E430DF8823D1F019DF6B017C01609353
:108470001F0A7093200A8093210A9093220A20E019
:1084800030E0A9010E9480B4181644F4C092210281
:10849000D0922202E0922302F0922402DF91CF9147
:1084A0001F910F91FF90EF90DF90CF90BF90AF9012
:1084B0009F908F90089580DF89E404DF882351F036
:1084C000EDDE6093230A7093240A8093250A90932B
:1084D000260A08C01092230A1092240A1092250A34
:1084E0001092260A8AE4EEDE882351F0D7DE6093EC
:1084F000270A7093280A8093290A90932A0A0895DC
:108500001092270A1092280A1092290A10922A0A19
:108510000895CF92DF92EF92FF92CF93DF93EC0119
:10852000C0904302D0904402E0904502F090460291
:10853000A7019601688179818A819B810E947DB221
:1085400087FF04C0C882D982EA82FB82C0904702BA
:10855000D0904802E0904902F0904A02A7019601AB
:108560006C817D818E819F810E947DB287FF04C0D6
:10857000CC82DD82EE82FF8220E030E0A9016091B2
:108580004B0270914C0280914D0290914E020E94DC
:10859000A4B16B017C019B01AC01688579858A855A
:1085A0009B850E947DB287FF04C0C886D986EA8673
:1085B000FB86C0903702D0903802E0903902F090EC
:1085C0003A02A7019601688179818A819B810E9484
:1085D00080B4181624F4C882D982EA82FB82C09043
:1085E0003B02D0903C02E0903D02F0903E02A70199
:1085F00096016C817D818E819F810E9480B41816C6
:1086000024F4CC82DD82EE82FF82C0903F02D090C3
:108610004002E0904102F0904202A7019601688575
:1086200079858A859B850E9480B4181624F4C886B3
:10863000D986EA86FB86DF91CF91FF90EF90DF909D
:10864000CF900895CF92DF92EF92FF920F931F93F6
:108650008FE29AE05EDF0E940EAD60937A0870931D
:108660007B0880937C0890937D0820912F0A30919D
:10867000300A4091310A5091320A6091640A709137
:10868000650A8091660A9091670A0E947DB2811105
:1086900079C02091330A3091340A4091350A5091C3
:1086A000360A6091680A7091690A80916A0A90910D
:1086B0006B0A0E947DB2811165C020E030E040E786
:1086C00052E46091210270912202809123029091E4
:1086D00024020E9484B250E5C52E5AE0D52E7B01BB
:1086E0008C012BE33AE047E35AE063E37AE08FE260
:1086F0009AE00E94549E80912F0A9091300AA09196
:10870000310AB091320A8093640A9093650AA0936B
:10871000660AB093670A8091330A9091340AA09157
:10872000350AB091360A8093680A9093690AA0933B
:108730006A0AB0936B0A8091370A9091380AA09127
:10874000390AB0913A0A80936C0A90936D0AA0930B
:108750006E0AB0936F0A80913B0A90913C0AA091F7
:108760003D0AB0913E0A8093700A9093710AA093DB
:10877000720AB093730A1F910F91FF90EF90DF90F0
:10878000CF90089560915D0270915E02882777FD19
:108790008095982F0E941FB32091210230912202D0
:1087A00040912302509124020E9452B520E030E013
:1087B00040E752E40E9484B220E030E048EC52E40A
:1087C00088CFCF92DF92EF92FF92CF93C62FE091A6
:1087D000500AF0E0882309F4C2C0DF01A45BB54F62
:1087E0008C91811196C18091640A9091650AA09143
:1087F000660AB091670A80932F0A9093300AA0937B
:10880000310AB093320A8091680A9091690AA09166
:108810006A0AB0916B0A8093330A9093340AA0934A
:10882000350AB093360A80916C0A90916D0AA09136
:108830006E0AB0916F0A8093370A9093380AA0931A
:10884000390AB0933A0AC090700AD090710AE09049
:10885000720AF090730AC0923B0AD0923C0AE092EE
:108860003D0AF0923E0AEE0FFF1FEE0FFF1FE15B85
:10887000FD4F2081318142815381CC2349F06091A9
:108880002F0270913002809131029091320208C023
:1088900060913302709134028091350290913602DA
:1088A0000E9484B29B01AC01C701B6010E94A4B131
:1088B0006093700A7093710A8093720A9093730A9E
:1088C00080E79AE00E94C0A8C0902102D0902202C6
:1088D000E0902302F090240220E030E040E752E4F0
:1088E00060912B0270912C0280912D0290912E02AA
:1088F0000E9452B56093210270932202809323025A
:1089000090932402E091500AF0E0E45BF54F81E09F
:10891000808398DE2091480A3091490A40914A0AA2
:1089200050914B0A60916C0A70916D0A80916E0AA9
:1089300090916F0A0E94A3B160936C0A70936D0AC4
:1089400080936E0A90936F0A20E73AE04CE65AE073
:1089500068E67AE084E69AE00E941BA8D1C0E45B56
:10896000F54F8081882309F4D4C08091640A9091E6
:10897000650AA091660AB091670A80932F0A9093C6
:10898000300AA093310AB093320A8091680A90911C
:10899000690AA0916A0AB0916B0A8093330A909396
:1089A000340AA093350AB093360A60916C0A70912C
:1089B0006D0A80916E0A90916F0A6093370A7093E6
:1089C000380A8093390A90933A0AC090700AD0907E
:1089D000710AE090720AF090730AC0923B0AD0923A
:1089E0003C0AE0923D0AF0923E0A2091480A3091FA
:1089F000490A40914A0A50914B0A0E94A4B16093DF
:108A00006C0A70936D0A80936E0A90936F0A20E748
:108A10003AE04CE65AE068E67AE084E69AE00E94A2
:108A20001BA8F090500ACC2389F02091400A309185
:108A3000410A4091420A5091430A60912F0270917D
:108A40003002809131029091320210C02091440A8C
:108A50003091450A4091460A5091470A609133028D
:108A60007091340280913502909136020E94A4B137
:108A700024E0F29EF0011124E15BFD4F2081318161
:108A8000428153810E9484B29B01AC016091700AC3
:108A90007091710A8091720A9091730A0E94A3B139
:108AA0006093700A7093710A8093720A9093730AAC
:108AB00080E79AE00E94C0A8C0902102D0902202D4
:108AC000E0902302F090240220E030E040E752E4FE
:108AD00060912702709128028091290290912A02C8
:108AE0000E9452B560932102709322028093230268
:108AF00090932402E091500AF0E0E45BF54F10827D
:108B0000A1DDC0922102D0922202E0922302F092D3
:108B10002402CF91FF90EF90DF90CF900895AF9215
:108B2000BF92CF92DF92EF92FF920F931F93CF935A
:108B3000DF93D82F2091270A3091280A4091290AE3
:108B400050912A0A6091230A7091240A8091250A83
:108B50009091260A0E948DB4C62F172F082FF92E48
:108B600060915D0270915E02882777FD8095982F55
:108B70000E941FB3209121023091220240912302D2
:108B8000509124020E9452B520E030E040E752E4C8
:108B90000E9484B220E030E048EC52E40E9484B2AB
:108BA0002091500A2F93DF93FF920F931F93CF933F
:108BB0005B016C0172E0E72E01E020E043E25AE045
:108BC0006FE27AE084E69AE00E94CD2A80912F0A33
:108BD0009091300AA091310AB091320A8093640AD0
:108BE0009093650AA093660AB093670A8091330A4E
:108BF0009091340AA091350AB091360A8093680AA0
:108C00009093690AA0936A0AB0936B0A8091370A1D
:108C10009091380AA091390AB0913A0A80936C0A6F
:108C200090936D0AA0936E0AB0936F0A80913B0AED
:108C300090913C0AA0913D0AB0913E0A8093700A3F
:108C40009093710AA093720AB093730A0E940EADBA
:108C500060937A0870937B0880937C0890937D08DA
:108C60000F900F900F900F900F900F90DF91CF917A
:108C70001F910F91FF90EF90DF90CF90BF90AF903A
:108C80000895F8940E94B721179A1092550A169ADF
:108C90001092560A159A1092570A149A60E087E4C7
:108CA0000E942EACE6EBFEE08491882341F0909187
:108CB000C00095FFFCCF8093C6003196F5CFEEE55E
:108CC000F9E08491882341F09091C00095FFFCCF9A
:108CD0008093C6003196F5CF8091C00085FFFCCF10
:108CE0008AE08093C60085E599E00E941077789429
:108CF000C6E0D0E02197209749F068EC70E080E072
:108D000090E00E943DAD0E949F77F4CFF894FFCF92
:108D10002F923F924F925F926F927F928F929F928B
:108D2000AF92BF92CF92DF92EF92FF920F931F9379
:108D3000CF93DF93CDB7DEB76E970FB6F894DEBF53
:108D40000FBECDBFB0E6BB2E14E0E12EF12C0CE33C
:108D5000C02E0CE0D02E8AE0A82E99249394809106
:108D60004A0E90914B0E20914C0E30914D0E821B6D
:108D7000930B8F779927892B09F41AC28091840865
:108D80009091850804970CF013C289EC9DE00E9435
:108D9000F88C8093830820918108309182088A3072
:108DA00061F08D3051F08A3321F49091800899233D
:108DB00021F02F3531050CF41DC12115310509F4C1
:108DC00037C18091860890918708B89E3001B99E7E
:108DD000700C1124F301E20FF31FE257F74F1082DA
:108DE00020918008211101C110928008FC01E657F2
:108DF000F74F108283010257174F6EE470E0C801ED
:108E00000E9400BA0097F1F190937F0880937E084A
:108E1000801B910B860D971D4AE050E060E070E0EA
:108E20008157974F0E943CB86093170A7093180AB5
:108E30008093190A90931A0A4090130A5090140ACA
:108E40006090150A7090160A2FEF421A520A620AB1
:108E5000720A0091860810918708641575058605C9
:108E6000970509F4E8C0B09EC001B19E900D112491
:108E700068E57DE08257974F0E94ABB9892B09F0D6
:108E8000DAC069C16AE270E0C8010E9400BA892BA9
:108E900009F444C0E6EBFEE08491882341F0909110
:108EA000C00095FFFCCF8093C6003196F5CFE2EB72
:108EB000FCE08491882341F09091C00095FFFCCFA5
:108EC0008093C6003196F5CF4091130A5091140A51
:108ED0006091150A7091160A2AE030E089EC9DE055
:108EE0000E94B38D8091C00085FFFCCF8AE0809303
:108EF000C6001092820810928108C0C28091170AA1
:108F00009091180AA091190AB0911A0A8093130A35
:108F10009093140AA093150AB093160A80918608BC
:108F200090918708B89E8001B99E100D1124C80148
:108F30008257974F3C0167E470E00E9400BA0097A7
:108F400081F190937F0880937E0886199709800F9E
:108F5000911F60E070E08157974F0E94D4B60E9445
:108F6000ECB264307105E8F480916C088823C9F094
:108F7000F6018491ECE3FCE0882349F09091C00075
:108F800095FFFCCF8093C60031968491F5CF8091F8
:108F9000C00085FFFCCFA092C60082E39CE00E9447
:108FA00003770091860810918708B09EC001B19E9A
:108FB000900D11246FE973E08257974F0E940BBA0E
:108FC000892B09F45EDEC8010196B7010E9448B6FC
:108FD00090938708809386088091840890918508F3
:108FE00001969093850880938408109282081092CD
:108FF0008108B5CE8B3311F490928008909180084F
:109000009111ADCE4091860850918708B9016F5FEC
:109010007F4F7093820860938108B49EF001B59EE3
:10902000F00D1124E20FF31FE257F74F808397CE24
:109030001092800823C2B09E3001B19E700C1124A2
:10904000C3018257974F1C016AE270E00E9400BA88
:10905000009789F5E6EBFEE08491882341F090913A
:10906000C00095FFFCCF8093C6003196F5CFECEDA4
:10907000FCE08491882341F09091C00095FFFCCFE3
:109080008093C6003196F5CF4091130A5091140A8F
:109090006091150A7091160A2AE030E089EC9DE093
:1090A0000E94B38D8091C00085FFFCCF8AE0809341
:1090B000C60057D91ECF20E010E0F301E20FF11DEA
:1090C000E257F74F30813A3219F02F5F1327F5CF6F
:1090D00090937F0880937E0882199309860D971DCF
:1090E00060E070E08157974F0E94D4B60E94ECB2C6
:1090F000212F30E02617370709F400CFE6EBFEE01A
:109100008491882341F09091C00095FFFCCF80931B
:10911000C6003196F5CFE6E0FDE08491882341F06A
:109120009091C00095FFFCCF8093C6003196F5CF9B
:109130004091130A5091140A6091150A7091160A11
:109140002AE030E089EC9DE00E94B38D8091C00060
:1091500085FFFCCFABCFE6EBFEE08491882341F0A6
:109160009091C00095FFFCCF8093C6003196F5CF5B
:10917000E5E2FDE08491882341F09091C00095FFE5
:10918000FCCF8093C6003196F5CF4091130A5091E1
:10919000140A6091150A7091160A2AE030E089ECF1
:1091A0009DE00E94B38D8091C00085FFFCCF7ECFF3
:1091B0008091850A882309F461C18091810890918A
:1091C0008208892B09F05AC1809184089091850802
:1091D000892B11F410926A08F8EE2F2EF3E03F2E3F
:1091E000412C512CACE3CA2ED12CE12CF12C8E0158
:1091F0000F5F1F4FE0E66E2E772473944091200D91
:109200005091210D6091220D7091230D8091180DC8
:109210009091190DA0911A0DB0911B0D4817590787
:109220006A077B0708F02AC180918408909185081D
:1092300004970CF023C180916A0881111FC18091AD
:10924000730C9091740CA091750CB091760C809376
:10925000200D9093210DA093220DB093230D8BE64A
:109260009CE00E945212482F809383088A30B9F004
:109270004D30A9F0433229F420918008222379F05F
:1092800002C04A33C9F320918108309182082F35FA
:1092900031052CF48F3FFFEF9F0709F0D1C04091BB
:1092A000200D5091210D6091220D7091230D809120
:1092B000180D9091190DA0911A0DB0911B0D481722
:1092C00059076A077B0708F481C0EFE1FCE084914D
:1092D000882341F09091C00095FFFCCF8093C60099
:1092E0003196F5CF8091C00085FFFCCFFAE0F09376
:1092F000C6000E940EAD60936E0870936F08809355
:109300007008909371088090720890907308A090F4
:109310007408B0907508681979098A099B09A20137
:1093200091010E945BB649015A01CA01B901A70126
:1093300096010E945BB6CA01B901A70196010E947D
:109340005BB67F936F93C501B40120E13EE040E03E
:1093500050E00E945BB63F932F93ABE0BCE0BF931D
:10936000AF931F930F930E9438BAE0EBFEE0849115
:109370000FB6F894DEBF0FBECDBF882349F09091A1
:10938000C00095FFFCCF8093C60031968491F5CF45
:10939000F8018191882339F09091C00095FFFCCFAE
:1093A0008093C600F6CF8091C00085FFFCCF3AE0E5
:1093B0003093C600C8010E945E7383E89AE00E9461
:1093C0007A3A61E083E89AE00E94A63480918308AB
:1093D000833211F470926A082091810830918208DA
:1093E0002115310509F424CE8091860890918708D3
:1093F000689EF001699EF00D1124E20FF31FE25701
:10940000F74F1082FC01E657F74F708220918408D5
:10941000309185082F5F3F4F309385082093840853
:10942000019664E070E00E9448B6909387088093AC
:109430008608109280081092820810928108DECE71
:109440004B3311F470928008409180084111D2CEC4
:109450004091860850918708B9016F5F7F4F7093E4
:10946000820860938108649EF001659EF00D1124CE
:10947000E20FF31FE257F74F8083C0CE6E960FB610
:10948000F894DEBF0FBECDBFDF91CF911F910F913A
:10949000FF90EF90DF90CF90BF90AF909F908F9014
:1094A0007F906F905F904F903F902F900895CF9254
:1094B000DF92EF92FF920F931F93CF93C82F80916B
:1094C00084089091850803970CF422DC0E940EAD6D
:1094D00000917608109177082091780830917908EA
:1094E000C0907A08D0907B08E0907C08F0907D08CE
:1094F0006C197D098E099F09061717072807390778
:1095000028F4012B022B032B09F0BBDB40911D0239
:1095100050911E0260911F0270912002452B462B34
:10952000472B19F10E940EAD00917A0810917B082B
:1095300020917C0830917D08601B710B820B930B8E
:1095400000911D0210911E0220911F0230912002F5
:10955000061717072807390740F490919B0E809152
:109560009A0E981302C0CC2349F0CF911F910F910E
:10957000FF90EF90DF90CF900C94389E179A109246
:10958000550A169A1092560A159A1092570A149A6A
:10959000ECCF0E94B72180916C08811138C081E026
:1095A00080936C088091130A9091140AA091150A77
:1095B000B091160A80930F0A9093100AA093110A93
:1095C000B093120AE6EBFEE08491882341F090917B
:1095D000C00095FFFCCF8093C6003196F5CFEFED2C
:1095E000F8E08491882341F09091C00095FFFCCF72
:1095F0008093C6003196F5CF8091C00085FFFCCFE7
:109600008AE08093C60085ED98E00C940377089576
:1096100080916C080895CF93DF93EC018091500AFC
:1096200080936D0884E50E946241811102C080E050
:1096300075C00E944E410E94F1B260936D0866238E
:10964000B1F3E0EBFEE08491882341F09091C000FB
:1096500095FFFCCF8093C6003196F5CFCD36D1056E
:10966000B9F054F4C836D105B1F0C936D10509F0C6
:1096700045C0E9EEF3E021C0CA3DD10531F0CD3D52
:10968000D105E1F5E4EAF3E036C0EBEBF3E029C005
:10969000E2EDF3E01CC0E0E0F4E08191882371F199
:1096A0009091C00095FFFCCF8093C600F6CF9091BB
:1096B000C00095FFFCCF8093C60081918111F7CF48
:1096C0001DC09091C00095FFFCCF8093C600819192
:1096D0008111F7CF13C09091C00095FFFCCF80930C
:1096E000C60081918111F7CF09C09091C00095FF0C
:1096F000FCCF8093C60081918111F7CF40E050E00C
:1097000060916D0889EC9DE00E94158E8091C000EB
:1097100085FFFCCF8AE08093C60081E0DF91CF9186
:109720000895CF92DF92EF92FF922091740A222344
:10973000F1F020E030E040E05FE30E9452B56B01C1
:109740007C0120E030E0A9010E947DB2882379F0FD
:10975000A7019601C701B6010E9452B52BED3FE06B
:1097600049E450E40E9452B59B01AC0104C020E0E2
:1097700030E040E85FE360E070E080E89FE30E9453
:1097800084B2FF90EF90DF90CF90089560915302E4
:10979000709154028091550290915602C2DF6093FD
:1097A0004F02709350028093510290935202089599
:1097B0003F924F925F926F927F928F929F92AF9261
:1097C000BF92CF92DF92EF92FF920F931F93CF93AE
:1097D000DF93CDB7DEB7E9970FB6F894DEBF0FBEC3
:1097E000CDBF81E40E9462418823B1F182E70E94EB
:1097F00062418823A9F0E6E2F4E08191882339F000
:109800009091C00095FFFCCF8093C600F6CF809169
:10981000C00085FFFCCF8AE08093C6000C940562EF
:1098200086E70E946241882311F40C940562EDE200
:10983000F4E08191882339F09091C00095FFFCCF2E
:109840008093C600F6CF8091C00085FFFCCF8AE0F0
:109850008093C6000C94056287E40E9462418823CD
:1098600009F462C20E944E410E94ECB26A30710556
:1098700009F4AFC09CF46230710509F44CC024F4C3
:1098800077FF25C00C9405626330710509F44EC062
:109890006430710509F455C00C9405626A35710590
:1098A00009F4EEC154F46B30710509F498C06C31C1
:1098B000710509F49AC00C9405626B35710509F4C1
:1098C000E3C16C35710509F4E4C10C940562809123
:1098D0006C0881110C9405620E94DC4180914D0A54
:1098E0008823A9F088E50E946241811110C089E5B2
:1098F0000E94624181110BC08AE50E946241811180
:1099000006C085E40E94624181110C9408620E94A5
:1099100022430C94056280916C0881110C940562BD
:109920000E945B4281E0FBD80C94056280916C0838
:1099300081110C9405620E945B4280E0F0D80C9487
:10994000056282E09CE00E94037780E50E9462410C
:10995000882339F00E944E410E94F1B24B015C0114
:1099600003C0812C912C540183E50E94624188231D
:1099700061F00E944E4120E030E04AE754E40E944A
:1099800052B50E94F1B24B015C010E94C1960E9447
:109990000EAD6B017C01C80CD91CEA1CFB1C0E949B
:1099A0000EAD60937A0870937B0880937C08909347
:1099B0007D080E940EAD6C157D058E059F0510F08B
:1099C0000C9405620E94E41E80E071DD0E949F7786
:1099D000F0CF60E081E00E94E1430C94056260E01A
:1099E00080E00E94E1430C940562809121029091F5
:1099F0002202A0912302B091240280931B0A90932B
:109A00001C0AA0931D0AB0931E0A80915D029091DA
:109A10005E029093780A8093770A84E690E09093B0
:109A20005E0280935D020E940EAD60937A0870938F
:109A30007B0880937C0890937D0881E00E94758F5D
:109A40008091640A9091650AA091660AB091670AB4
:109A500080932F0A9093300AA093310AB093320A70
:109A60008091680A9091690AA0916A0AB0916B0A84
:109A70008093330A9093340AA093350AB093360A40
:109A800080916C0A90916D0AA0916E0AB0916F0A54
:109A90008093370A9093380AA093390AB0933A0A10
:109AA0008091700A9091710AA091720AB091730A24
:109AB00080933B0A90933C0AA0933D0AB0933E0AE0
:109AC000109221021092220210922302109224027C
:109AD00088E50E946241882311F090E00AC089E580
:109AE0000E9462418111F9CF8AE50E94624191E0B2
:109AF00098279093250291110C94376288E50E9473
:109B0000624181110C9437628091250281110C947D
:109B10003D6289E50E94624181110C943D6288E5B5
:109B20000E9462418823D1F00E945741672B682B25
:109B3000692BA1F00E944E412091580A3091590A98
:109B400040915A0A50915B0A0E94A4B16093640A42
:109B50007093650A8093660A9093670A89E50E946C
:109B600062418823D1F00E945741672B682B692BF3
:109B7000A1F00E944E4120915C0A30915D0A409113
:109B80005E0A50915F0A0E94A4B16093680A7093C4
:109B9000690A80936A0A90936B0A80912502811169
:109BA0000C9443628AE50E94624181110C944362E5
:109BB0008AE50E9462418823D1F00E945741672BB9
:109BC000682B692BA1F00E944E412091600A3091D0
:109BD000610A4091620A5091630A0E94A4B16093A5
:109BE0006C0A70936D0A80936E0A90936F0A20E757
:109BF0003AE04CE65AE068E67AE084E69AE00E94B1
:109C00001BA880E00E94758F80911B0A90911C0A0E
:109C1000A0911D0AB0911E0A809321029093220206
:109C2000A0932302B09324028091770A9091780A3E
:109C300090935E0280935D020E940EAD60937A085D
:109C400070937B0880937C0890937D080E946E8FB0
:109C50008091850A882311F40C94056261E87AE00A
:109C600089EF9FE00E9497708091810A9091820A0B
:109C7000892B11F40C9405620E9442790C940562C0
:109C800010920E0A0C94056281E080930E0A0C94E7
:109C9000056285E40E946241811102C00E94C19662
:109CA00054EDC52E54E0D52E68E5E62E6AE0F62E7A
:109CB00004E61AE0B12CF60181916F010E94624125
:109CC000882339F1F3E0BF120CC00E944E41F80125
:109CD000608371838283938380E79AE00E94C0A8A7
:109CE00018C00E944E41F701208131814281538189
:109CF0000E94A4B1F801608371838283938320E77B
:109D00003AE04CE65AE068E67AE084E69AE00E949F
:109D10001BA8B394F4E0EF0EF11C0C5F1F4F24E07E
:109D2000B212C9CF0C9405628DE40E94624188236F
:109D300011F40C9434610E944E410E94ECB26537DC
:109D4000710511F40C94FF560CF0A6C06032710539
:109D500009F4F0C20CF056C06731710509F445C230
:109D600054F56231710509F469C7BCF477FF02C08C
:109D70000C940562623071050CF461C161317105AA
:109D800011F00C94056289EC9BE00E940377179810
:109D90001698159814980C9405626531710509F4AC
:109DA00018C20CF01CC26431710511F00C940562EC
:109DB000E9EBFBE0EAC16B31710509F442C2B4F48E
:109DC0006931710509F429C20CF02DC283E89AE0CB
:109DD0000E94A8310E940EAD6093720870937308C0
:109DE00080937408909375080C9405626E31710528
:109DF00009F462C20CF03AC36C31710509F427C250
:109E00000C9405626C35710509F46BC7ECF462358E
:109E1000710509F40AC764F46035710509F4DBC6FD
:109E20000CF0E6C66A32710509F47EC30C94056233
:109E30006435710509F402C70CF4FBC6653571057C
:109E400009F434C70C9405626B36710509F4BDC67C
:109E500064F46936710509F4DEC30CF086C6683611
:109E6000710509F4A8C30C9405626037710509F403
:109E7000BFC334F46D36710509F4DAC40C9405627D
:109E80006237710509F4CFC76337710511F00C947F
:109E90000562EFE3FAE0AEC76D3D710511F40C9475
:109EA000075B0CF04DC06B3C710511F40C948359A9
:109EB00044F56C38710509F49DC39CF4683771054D
:109EC00011F40C94F3576937710511F40C94F85799
:109ED0006737710511F00C940562E4E3F4E00C942B
:109EE0000358683C710511F40C94ED58693C7105F8
:109EF00011F40C9462596E3B710511F00C940562DB
:109F000021C56F3C710511F40C943D5A54F46D3C1D
:109F1000710511F40C94C25914F40C94A0590C94CA
:109F2000205A613D710511F40C94985A14F40C9464
:109F3000725A6C3D710511F40C94F85A0C94056238
:109F4000603931E0730711F40C94CA5C54F56E3239
:109F500091E0790711F40C94845C84F46C32F1E0A4
:109F60007F0711F40C94885B14F00C94BE5B623E86
:109F7000710511F40C942D5B0C9405626E3531E083
:109F8000730711F40C94A1606F3581E0780711F428
:109F90000C94D8606F32714011F00C9405620C94EF
:109FA000925C6835E2E07E0711F40C94A85DBCF485
:109FB000663F21E0720711F40C94CD5C673F31E0FD
:109FC000730711F40C94D05C653F714011F00C9450
:109FD00005620E94E58A0E94B7860C9405626B3880
:109FE00093E0790711F40C947B603CF46335734083
:109FF00011F40C94D35C0C940562603A23E0720770
:10A0000009F401C2673E734011F00C94056210928E
:10A010006C080E94167780910F0A9091100AA09107
:10A02000110AB091120A8093130A9093140AA09314
:10A03000150AB093160A0E94B1410C940562009172
:10A040007E0810917F080E5F1F4F80E50E946241DD
:10A05000882379F00E944E410E94F1B26B017C018D
:10A06000BB24B394611571058105910531F4B12CC0
:10A0700004C0B12CC12CD12C760183E50E94624131
:10A08000882399F00E944E4120E030E04AE754E4F2
:10A090000E9452B50E94F1B26B017C01AA24A394E4
:10A0A000611571058105910509F4A12C6AE270E042
:10A0B000C8010E9400BA009711F0FC011082F8015B
:10A0C000CF0121912032E1F3B11007C0A11005C0EA
:10A0D000222319F00E945E7304C081EF9BE00E946E
:10A0E000037781E00E943E730E94C1960E940EADEC
:10A0F00060937A0870937B0880937C0890937D0826
:10A10000C114D104E104F104A9F00E940EAD4B0189
:10A110005C018C0C9D1CAE1CBF1C0E940EAD681512
:10A1200079058A059B05B8F40E947378811113C0E4
:10A130000C9449620E947178882311F40C94056292
:10A140000E94737881110AC00E94E41E80E0AFD99A
:10A150000E949F77F5CF80E00E943E738091850A30
:10A16000882331F082EE9BE00E9403770C94056215
:10A1700082ED9BE00E9403770C9405629091C000F1
:10A1800095FFFCCF8093C600319684918111F6CF64
:10A190008091C00085FFFCCF8AE08093C60083E8F1
:10A1A0009AE00E948430EBEAFBE08491882341F03E
:10A1B0009091C00095FFFCCF8093C6003196F5CFFB
:10A1C0008091C00085FFFCCF8AE08093C6000C948C
:10A1D000056283E89AE00E94D9300C94056283E816
:10A1E0009AE00E94A4310C94056200917E081091BF
:10A1F0007F080C5F1F4F6AE270E0C8010E9400BA3E
:10A20000009711F0FC01108221E041E0B80183E8E1
:10A210009AE00E940B360C94056283E89AE00E9453
:10A22000AF310C9405628091860A882311F40C9456
:10A23000056283E50E94624181110C9452620C9484
:10A24000056283E89AE00E9453330C940562809182
:10A250007E0890917F086AE270E004960E9400BA3E
:10A260008C010097D9F0209188083091890840E648
:10A27000429FC001439F900D11246EE470E082570D
:10A28000974F0E9400BA60E270E00E9400BA019607
:10A2900090937F0880937E08F801108260917E0879
:10A2A00070917F086C5F7F4F21E040E083E89AE087
:10A2B0000E940B360C9405628091860A882311F463
:10A2C0000C94056260E083E89AE00E949C358091DE
:10A2D0007E0890917F086AE270E004960E9400BABE
:10A2E0008C010097D9F0209188083091890840E6C8
:10A2F000429FC001439F900D11246EE470E082578D
:10A30000974F0E9400BA60E270E00E9400BA019686
:10A3100090937F0880937E08F801108260917E08F8
:10A3200070917F086C5F7F4F83E89AE00E94133240
:10A330000C9405628091850A81110E94C19600915A
:10A340007E0810917F080C5F1F4F6AE270E0C80121
:10A350000E9400BA7C0161E270E0C8010E9400BA6C
:10A36000009719F08C010F5F1F4FE114F10411F0F9
:10A37000F701108280E50E946241F82E20917E084C
:10A3800030917F080217130708F4F12C8091860A98
:10A39000882311F40C94056221E02F2541E0B801D7
:10A3A00083E89AE00E940B3683E50E94624188238D
:10A3B000B9F020917E0830917F082017310780F492
:10A3C0000E945741AB01BC014093200D5093210DD9
:10A3D0006093220D7093230D8BE69CE00E941B136B
:10A3E00083E89AE00E94A831F1100C9405620E9463
:10A3F0000EAD609372087093730880937408909305
:10A4000075080C94056280917E0890917F086AE23D
:10A4100070E005960E9400BA8C010097D9F0209157
:10A4200088083091890840E6429FC001439F900D03
:10A4300011246EE470E08257974F0E9400BA60E2E8
:10A4400070E00E9400BA019690937F0880937E0886
:10A45000F801108260917E0870917F086B5F7F4FDA
:10A4600083E89AE00E9435390C9405620E940EAD93
:10A4700060936E0870936F088093700890937108D2
:10A48000009172081091730820917408309175083A
:10A49000601B710B820B930B28EE33E040E050E021
:10A4A0000E945BB6CA01B9012CE330E040E050E005
:10A4B0000E945BB67F936F933F932F938CE99BE051
:10A4C0009F938F93CE0101969F938F930E9438BAEA
:10A4D000E0EBFEE084910FB6F894DEBF0FBECDBF77
:10A4E000882349F09091C00095FFFCCF8093C6006F
:10A4F00031968491F5CFFE0131968191882339F010
:10A500009091C00095FFFCCF8093C600F6CF80915C
:10A51000C00085FFFCCF8AE08093C600CE01019683
:10A520000E945E730C94056283E50E946241882359
:10A5300011F40C9405620E944E410E94ECB2F62E7A
:10A54000E72E862F9E2D8C0180E50E946241882394
:10A5500031F00F3F110509F010F40C9463620DE027
:10A5600010E0ECE9F4E0819191918017910711F4EA
:10A570000C94056234E0E43DF307A9F706301105B9
:10A5800039F48F2D9E2D90934F0A80934E0A04C06C
:10A5900017FF02C00C94056261E0802F0E942EAC70
:10A5A0006F2D802F0E9467AC6F2D7E2D802F0E9413
:10A5B00024AB0C94056288E690E02DD881110C94B0
:10A5C000056283E50E946241882371F000916D0865
:10A5D0000E944E4110E0000F111F0859174F0E94B2
:10A5E000ECB2F801718360830E94B6210C9405627D
:10A5F0000E94414683E50E946241882311F40C9435
:10A6000005620E944E410E94ECB27093670860930D
:10A6100066080C94056289E690E00E940B4B81115C
:10A620000C940562E6E9FBE08491882341F0909167
:10A63000C00095FFFCCF8093C6003196F5CFE09126
:10A640006D0824E0E29FF0011124E05AF74F4081A9
:10A6500051816281738121E030E089EC9DE00E94AC
:10A66000B48EE3E9FBE08491882341F09091C0002F
:10A6700095FFFCCF8093C6003196F5CFE0916D0831
:10A68000F0E0EE0FFF1FE859F74F608171818827D6
:10A6900077FD8095982F0E941FB3AB01BC0121E08C
:10A6A00030E089EC9DE00E94B48EEFE8FBE08491FD
:10A6B000882341F09091C00095FFFCCF8093C600A5
:10A6C0003196F5CF40915A0850915B0860915C0833
:10A6D00070915D0821E030E089EC9DE00E94B48E2D
:10A6E000ECE8FBE08491882341F09091C00095FF55
:10A6F000FCCF8093C6003196F5CF609166087091CB
:10A700006708882777FD8095982F0E941FB3AB01BB
:10A71000BC0121E030E089EC9DE00E94B48EE9E8C4
:10A72000FBE08491882341F09091C00095FFFCCF1D
:10A730008093C6003196F5CF4AE050E060E070E0CB
:10A7400089EC9DE00E94DE8DE7E8FBE084918823A0
:10A7500041F09091C00095FFFCCF8093C6003196E8
:10A76000F5CF409160085091610860916208709146
:10A77000630821E030E089EC9DE00E94B48EE4E8BB
:10A78000FBE08491882341F09091C00095FFFCCFBD
:10A790008093C6003196F5CF609168087091690882
:10A7A000882777FD8095982F0E941FB3AB01BC01CD
:10A7B00021E030E089EC9DE00E94B48EE0E8FBE00F
:10A7C0008491882341F09091C00095FFFCCF809345
:10A7D000C6003196F5CF80916D0890E00E94AE1EC4
:10A7E0004AE050E0BC0189EC9DE00E94DE8DEBE781
:10A7F000FBE08491882341F09091C00095FFFCCF4D
:10A800008093C6003196F5CF8FEF9FEF0E94AE1E6A
:10A810004AE050E0BC0189EC9DE00E94DE8D809111
:10A82000C00085FFFCCF8AE08093C6000C94C16312
:10A830008DE690E00E940B4B81110C94056280E73D
:10A840009BE00E94037783E50E946241882391F098
:10A8500000916D080E944E4110E0000F111F085931
:10A86000174F0E94ECB2F8017183608381E08093FE
:10A870001C0215C082E50E946241882381F000918C
:10A880006D080E944E4110E0000F111F0859174F2C
:10A890000E94ECB2F8017183608310921C020E9446
:10A8A000B6210E940EAD4B015C0100916D0810E0D5
:10A8B000F801EE0FFF1FE859F74F6081718188277B
:10A8C00077FD8095982F0E941FB3F801EE0FFF1FB0
:10A8D000EE0FFF1FE05AF74F11E0208131814281D6
:10A8E00053810E9480B418160CF010E010936B088E
:10A8F00010923F0ACC24CA94DC2C760148EE442EF8
:10A9000043E0542E612C712C5AE0352E80913F0A81
:10A9100081110C947E63FFEFCF16DF06EF06FF0672
:10A9200011F40C946A62F7FE02C00C947E630E94DC
:10A930000EAD6C197D09683B7B4010F40C946A6283
:10A940000C947E638AE49BE00E94037783E50E9477
:10A950006241882361F00E944E410E94ECB27093E4
:10A9600067086093660881E080931C020FC082E54F
:10A970000E946241882351F00E944E410E94ECB235
:10A98000709367086093660810921C020E940EADD7
:10A990004B015C0110923F0A609166087091670854
:10A9A000882777FD8095982F0E941FB311E0209192
:10A9B0005A0830915B0840915C0850915D080E94F4
:10A9C00080B418160CF010E010936B0807E41BE03D
:10A9D000E3E4EE2EEBE0FE2EFFE3CF2EFBE0DF2ED6
:10A9E000AAE07A2E80916B086091660870916708E2
:10A9F000882309F48BC080913F0A811187C0882782
:10AA000077FD8095982F0E941FB320915A083091AE
:10AA10005B0840915C0850915D080E9480B4181654
:10AA20000CF08BC00E940EAD681979098A099B0948
:10AA3000693E73408105910508F460C0E091500AB9
:10AA400084E0E89FF0011124E05AF74F40815181E2
:10AA500062817381F8018491E7E4FBE0882349F087
:10AA60009091C00095FFFCCF8093C60031968491F1
:10AA7000F5CF22E030E089EC9DE00E94B48EF70132
:10AA80008491E3E4FBE0882349F09091C00095FFB6
:10AA9000FCCF8093C60031968491F5CF6091500A27
:10AAA00070E04AE050E089EC9DE00E94DE8DF60106
:10AAB0008491EFE3FBE0882349F09091C00095FF7B
:10AAC000FCCF8093C60031968491F5CF40915A080F
:10AAD00050915B0860915C0870915D0821E030E066
:10AAE00089EC9DE00E94B48E8091C00085FFFCCF70
:10AAF0007092C6000E940EAD4B015C010E94E41EE4
:10AB000080E00E94574A0E949F776CCF882777FD8C
:10AB10008095982F0E941FB320915A0830915B08AE
:10AB200040915C0850915D080E947DB287FF05C08E
:10AB300080911C02882309F475CF85E39BE00E9475
:10AB400003778091850A882321F08AE893E00E94A8
:10AB50005E730E940EAD60937A0870937B088093B9
:10AB60007C0890937D080C94056283E50E94624105
:10AB7000882319F10E944E4120E030E0A9010E9493
:10AB80007DB287FD0FC00E944E4120E030E04FE7CC
:10AB900053E40E9480B4181644F00E944E410E9473
:10ABA000ECB205C060E070E002C06FEF70E070933F
:10ABB0004F0A60934E0A0C9405628FEF90E09093D9
:10ABC0004F0A80934E0A0C94056210924F0A10921D
:10ABD0004E0A0C9405629B9AA39881E0809326020A
:10ABE00085E29BE00E9403770E949F770C940562A8
:10ABF0000E94B7210E94C196149A0E942B9710922E
:10AC00004F0A10924E0A68EE73E080E090E00E94D6
:10AC10003DAD9B9AA39A1092260287E19BE00E9489
:10AC200003770E949F770C94056210927C0A0C9423
:10AC3000056281E080937C0A0C94056283E50E94A2
:10AC400062418823A1F00E944E4120E030E04AE7B3
:10AC500054E40E9452B50E94F1B260931D027093B9
:10AC60001E0280931F02909320020C94056288E5D7
:10AC70000E94624181110C949F6389E50E946241A8
:10AC800081110C949F638AE50E94624181110C94AA
:10AC90009F6385E40E94624181110C949F630E942E
:10ACA000C196149A0E942B970C94056283E50E942A
:10ACB0006241882311F40C9405620E944E4120E009
:10ACC00030E04AE754E40E9452B50E94F1B260932A
:10ACD00076087093770880937808909379080C949D
:10ACE000056224ED34E039AF28AF0FEC13E16FEDCE
:10ACF000862E63E1962E73E9A72E73E1B72E312CD1
:10AD0000E8ADF9AD8191F9AFE8AF0E9462418823C7
:10AD100009F45BC0F3E03F1251C00E944E416B0149
:10AD20007C0120E030E040EA51E40E947DB287FFE0
:10AD30003FC0A7019601F8016081718182819381F2
:10AD40000E9484B22B013C019B01AC016091A713CE
:10AD50007091A8138091A9139091AA130E9452B5E3
:10AD60006093A7137093A8138093A9139093AA13C9
:10AD7000A3019201F40160817181828193810E941B
:10AD800052B5F4016083718382839383F5016081FE
:10AD90007181828193810E941DB3A30192010E945F
:10ADA00052B50E94F1B2F50160837183828393836F
:10ADB000F801C082D182E282F38207C00E944E4134
:10ADC000F801608371838283938333940C5F1F4FF8
:10ADD000F4E08F0E911C24E0A20EB11C34E033127B
:10ADE0008FCF0C9405629091C00095FFFCCF8093AB
:10ADF000C600319684918111F6CF0C9405620091C2
:10AE00007E0810917F080B5F1F4F6AE270E0C80157
:10AE10000E9400BA009711F0FC011082C8010E9444
:10AE20005E730C940562ECE3FAE08491882341F0B0
:10AE30009091C00095FFFCCF8093C6003196F5CF6E
:10AE40004091640A5091650A6091660A7091670AA0
:10AE500022E030E089EC9DE00E94B48EE8E3FAE065
:10AE60008491882341F09091C00095FFFCCF80939E
:10AE7000C6003196F5CF4091680A5091690A6091F9
:10AE80006A0A70916B0A22E030E089EC9DE00E9432
:10AE9000B48EE4E3FAE08491882341F09091C000FD
:10AEA00095FFFCCF8093C6003196F5CF40916C0A98
:10AEB00050916D0A60916E0A70916F0A22E030E045
:10AEC00089EC9DE00E94B48EE0E3FAE0849188234F
:10AED00041F09091C00095FFFCCF8093C600319661
:10AEE000F5CF4091700A5091710A6091720A709189
:10AEF000730A22E030E089EC9DE00E94B48EE5E226
:10AF0000FAE08491882341F09091C00095FFFCCF36
:10AF10008093C6003196F5CF0E941D970E941FB303
:10AF20002091CF133091D0134091D1135091D2136F
:10AF30000E9484B2AB01BC0122E030E089EC9DE0CC
:10AF40000E94B48EE1E2FAE08491882341F090916E
:10AF5000C00095FFFCCF8093C6003196F5CF81E00D
:10AF60000E941D970E941FB32091D3133091D413D8
:10AF70004091D5135091D6130E9484B2AB01BC010D
:10AF800022E030E089EC9DE00E94B48EEDE1FAE031
:10AF90008491882341F09091C00095FFFCCF80936D
:10AFA000C6003196F5CF82E00E941D970E941FB324
:10AFB0002091D7133091D8134091D9135091DA13BF
:10AFC0000E9484B2AB01BC0122E030E089EC9DE03C
:10AFD0000E94B48E8091C00085FFFCCF8AE08093F0
:10AFE000C6000C94056280E00E94758F0C94056287
:10AFF00081E00E94758F0C9405629091C00095FFCE
:10B00000FCCF8093C60081918111F7CF8091C00061
:10B0100085FFFCCF8AE08093C600E5E1FAE08491E9
:10B02000882341F09091C00095FFFCCF8093C6002B
:10B030003196F5CF1E9B03C0E7E1F4E009C0E1E2E1
:10B04000F4E006C09091C00095FFFCCF8093C6004D
:10B0500081918111F7CF8091C00085FFFCCF8AE0FC
:10B060008093C600EDE0FAE08491882341F090914E
:10B07000C00095FFFCCF8093C6003196F5CF0299B2
:10B0800003C0E7E1F4E009C0E1E2F4E006C090911A
:10B09000C00095FFFCCF8093C60081918111F7CF4E
:10B0A0008091C00085FFFCCF8AE08093C600E5E078
:10B0B000FAE08491882341F09091C00095FFFCCF85
:10B0C0008093C6003196F5CF1D9B03C0E7E1F4E005
:10B0D00009C0E1E2F4E006C09091C00095FFFCCF0A
:10B0E0008093C60081918111F7CF8091C00085FFC8
:10B0F000FCCF8AE08093C600EDEFF9E084918823CD
:10B1000041F09091C00095FFFCCF8093C60031962E
:10B11000F5CF019903C0E7E1F4E009C0E1E2F4E012
:10B1200006C09091C00095FFFCCF8093C60081912E
:10B130008111F7CF8091C00085FFFCCF8AE080931A
:10B14000C600E5EFF9E08491882341F09091C000BA
:10B1500095FFFCCF8093C6003196F5CF1C9B03C0B2
:10B16000E7E1F4E009C0E1E2F4E006C09091C0003C
:10B1700095FFFCCF8093C60081918111F7CF80911C
:10B18000C00085FFFCCF8AE08093C600EDEEF9E0B9
:10B190008491882341F09091C00095FFFCCF80936B
:10B1A000C6003196F5CF379903C0E7E1F4E009C056
:10B1B000E1E2F4E006C09091C00095FFFCCF8093DF
:10B1C000C60081918111F7CF8091C00085FFFCCF2F
:10B1D0008AE08093C6000C9405628091500A8093A7
:10B1E0006D0884E50E946241882319F10E944E4156
:10B1F0000E94F1B260936D086623D9F0E0EBFEE0A7
:10B200008491882341F09091C00095FFFCCF8093FA
:10B21000C6003196F5CFEDE4F4E08191882311F476
:10B220000C9405629091C00095FFFCCF8093C600FE
:10B23000F4CF84E40E946241882311F40C940562E7
:10B240000E944E4120E030E0A9010E947DB28111B0
:10B2500003C01092740A32C000916D0810E00E9481
:10B260004E41F801EE0FFF1FEE0FFF1FED5AFD4F8D
:10B270006083718382839383E0905302F090540241
:10B28000009155021091560220E030E0A901B7016B
:10B29000C8010E947DB2811104C0E12CF12C00E4B0
:10B2A00010E4C701D8018093530290935402A093F5
:10B2B0005502B093560281E08093740A0E94C64BF7
:10B2C0000C94056204ED14E04FEBE42E43E1F42E00
:10B2D000F80181918F010E946241882349F00E9408
:10B2E0004E410E94F1B2F7016083718382839383A0
:10B2F000F4E0EF0EF11C24E0083D120749F70E942C
:10B30000EDA80C94056204ED14E03FEDE32E33E16B
:10B31000F32EF80181918F010E946241882339F058
:10B320000E944E41F7016083718382839383F4E02E
:10B33000EF0EF11C24E0083D120759F70C9405624A
:10B3400083E50E946241882351F00E944E41609340
:10B35000B7137093B8138093B9139093BA1384E51D
:10B360000E946241882311F40C9405620E944E41B0
:10B370006093B3137093B4138093B5139093B61383
:10B380000C94056283E50E946241882351F00E947B
:10B390004E416093BB137093BC138093BD13909385
:10B3A000BE1384E50E946241882351F00E944E4101
:10B3B0006093A3137093A4138093A5139093A61383
:10B3C00082E40E946241882361F00E944E410E9403
:10B3D000F1B26093EF137093F0138093F113909395
:10B3E000F21388E50E946241882351F00E944E4189
:10B3F0006093AF137093B0138093B1139093B21313
:10B400008AE50E946241882351F00E944E41609378
:10B41000AB137093AC138093AD139093AE1385E48C
:10B420000E946241882309F4F0C70E944E41609354
:10B43000A7137093A8138093A9139093AA13E5C739
:10B4400004ED14E028E5E22E2AE0F22EF8018191C5
:10B450008F010E946241882339F00E944E41F7011A
:10B460006083718382839383F4E0EF0EF11C24E008
:10B47000073D120709F4C9C7E9CF83E50E9462417D
:10B48000882351F00E944E4160933302709334023E
:10B49000809335029093360286E40E9462418823AD
:10B4A00081F00E944E4120E030E040E752E40E94EB
:10B4B00084B260932B0270932C0280932D029093A0
:10B4C0002E028AE50E946241882309F49EC70E94E9
:10B4D0004E416093480A7093490A80934A0A9093B8
:10B4E0004B0A93C783E50E946241882351F00E9472
:10B4F0004E416093440A7093450A8093460A9093A4
:10B50000470A86E40E946241882309F47EC70E94AC
:10B510004E4120E030E040E752E40E9484B2609364
:10B520002702709328028093290290932A026DC704
:10B5300083E50E946241882309F467C70E944E4157
:10B540000E94ECB26115710549F06130710559F442
:10B5500081E080934D0A10924C0A57C710924D0A11
:10B5600010924C0A52C7E0EBFEE08491882341F030
:10B570009091C00095FFFCCF8093C6003196F5CF27
:10B58000EAEDF9E08491882341F09091C00095FFA5
:10B59000FCCF8093C6003196F5CF809188089091BA
:10B5A000890820E6289FF001299FF00D1124E25719
:10B5B000F74F8191882339F09091C00095FFFCCF1F
:10B5C0008093C600F6CFE8EDF9E08491882341F03E
:10B5D0009091C00095FFFCCF8093C6003196F5CFC7
:10B5E0008091C00085FFFCCF8AE08093C6000DC724
:10B5F00083E50E946241882309F407C70E944E41F7
:10B600000E94ECB270935E0260935D02FEC683E519
:10B610000E946241882309F4F8C60E944E410E94AC
:10B62000ECB26B017C0184E50E946241882381F0C9
:10B630008DED90E00E940B4B8111E7C6E0916D0803
:10B64000F0E0EE0FFF1FE75AFD4FD182C082DDC64A
:10B65000D0925C02C0925B02D8C680E50E94624133
:10B66000882309F4D2C60E944E410E94ECB2D62E25
:10B67000062F172F83E50E946241882331F00E9434
:10B680004E410E94ECB27B0103C0EE24EA94FE2CF2
:10B69000C7010196039708F0B8C6ECE9F4E0819180
:10B6A00091918017910709F4B0C634E0E43DF307A7
:10B6B000B1F717FDAAC60E94C196CD2C60E08D2D72
:10B6C0000E942EAC8FEFE816F80631F0EA94EF28CE
:10B6D00071F000E010E00DC08D2D0E949CAC31E0B7
:10B6E00020E0892B09F030E0032F122F02C001E087
:10B6F00010E08C2D0E949CAC8017910709F485C640
:10B700000E94E41E80E00E94574A0E949F77F1CF7A
:10B7100083E50E946241882331F00E944E410E94DD
:10B72000ECB28B0102C00EE610E080E50E9462419F
:10B73000882331F00E944E410E94ECB2CB0102C03E
:10B7400088EE93E06C01EE24D7FCE094FE2C1016FA
:10B7500011067CF420E030E0A901B8018EE40E94DB
:10B76000DAADC701B6010E943DAD8EE40E94EBB098
:10B770004CC6C701B6010E943DAD47C680E50E9498
:10B780006241882351F00E944E41609318027093E9
:10B79000190280931A0290931B0289E40E9462416D
:10B7A000882361F00E944E410E9429286093140270
:10B7B00070931502809316029093170284E40E94FE
:10B7C0006241882361F00E944E410E9435286093B7
:10B7D000100270931102809312029093130283E47B
:10B7E0000E946241882351F00E944E4160930C02F6
:10B7F00070930D0280930E0290930F020E94971E89
:10B80000E4E6F4E08191882339F09091C00095FF3F
:10B81000FCCF8093C600F6CFE7E6F4E08191882361
:10B8200039F09091C00095FFFCCF8093C600F6CF11
:10B83000409118025091190260911A0270911B02F6
:10B8400022E030E089EC9DE00E94B48EEBE6F4E06B
:10B850008191882339F09091C00095FFFCCF8093AF
:10B86000C600F6CF60911402709115028091160205
:10B87000909117020E942F28AB01BC0122E030E01A
:10B8800089EC9DE00E94B48EEFE6F4E0819188237C
:10B8900039F09091C00095FFFCCF8093C600F6CFA1
:10B8A0006091100270911102809112029091130226
:10B8B0000E943B28AB01BC0122E030E089EC9DE016
:10B8C0000E94B48EE3E7F4E08191882339F09091EF
:10B8D000C00095FFFCCF8093C600F6CF40910C02CC
:10B8E00050910D0260910E0270910F0222E030E043
:10B8F00089EC9DE00E94B48E8091C00085FFFCCF52
:10B900008AE08093C60081C583E50E946241882356
:10B9100019F00E944E4103C060E070E0CB010E942C
:10B92000E4A873C585E40E946241882341F00E9427
:10B930004E410E94ECB28B0177FF03C009C000E0CA
:10B9400010E0C12CD12CB6E1EB2EB3E4FB2E06C0E7
:10B95000C12CD12CACE8EA2EA2E4FA2E83E50E9499
:10B960006241882321F00E944E416B017C0183E4F7
:10B970000E946241882331F00E944E410E94ECB245
:10B980009B0102C025E030E0A801C701B6010E947A
:10B99000CA213BC50E94C19638C50E94E58A35C5BB
:10B9A0000E94B78632C58AE50E946241882309F465
:10B9B00097C00E944E416B017C0120E030E040E7DF
:10B9C00051EC0E9480B487FD3FC020E030E040EAA7
:10B9D00050ECC701B6010E947DB21816ACF1F7FA1F
:10B9E000F094F7F8F094C092510AD092520AE09283
:10B9F000530AF092540AE0EBFEE08491882341F070
:10BA00009091C00095FFFCCF8093C6003196F5CF92
:10BA1000ECECF9E08491882341F09091C00095FF0F
:10BA2000FCCF8093C6003196F5CF8091C00085FF92
:10BA3000FCCF8AE08093C6008091C00085FFFCCFD8
:10BA40008AE08093C600E1C4E0EBFEE084918823A5
:10BA500041F09091C00095FFFCCF8093C6003196D5
:10BA6000F5CFE3ECF9E08491882341F09091C00098
:10BA700095FFFCCF8093C6003196F5CFEBEBF9E054
:10BA80008491882341F09091C00095FFFCCF809372
:10BA9000C6003196F5CF4AE050E061EF7FEF89ECC8
:10BAA0009DE00E94DE8DE3EBF9E08491882341F074
:10BAB0009091C00095FFFCCF8093C6003196F5CFE2
:10BAC0004AE050E06BEF7FEF89EC9DE00E94DE8D55
:10BAD0008091C00085FFFCCF8AE08093C60095C4AA
:10BAE000E0EBFEE08491882341F09091C00095FF47
:10BAF000FCCF8093C6003196F5CFE7EAF9E0849158
:10BB0000882341F09091C00095FFFCCF8093C60040
:10BB10003196F5CF8091C00085FFFCCF8AE08093FD
:10BB2000C6004091510A5091520A6091530A709197
:10BB3000540A705822E030E089EC9DE00E94B48EF7
:10BB40008091C00085FFFCCF8AE08093C6005DC471
:10BB500080915D0290915E0290935802809357020B
:10BB6000C090640AD090650AE090660AF090670A77
:10BB7000CF8ED8A2E9A2FAA20091680A1091690AB0
:10BB800020916A0A30916B0A0BA31CA32DA33EA33C
:10BB900040916C0A50916D0A60916E0A70916F0A23
:10BBA0004FA358A769A77AA78091700A9091710A4C
:10BBB000A091720AB091730A8BA79CA7ADA7BEA7EC
:10BBC000C982DA82EB82FC820D831E832F83388741
:10BBD00049875A876B877C878D879E87AF87B88B0D
:10BBE00085E40E946241882359F00E944E419B01E6
:10BBF000AC016BA57CA58DA59EA50E94A4B10AC031
:10BC000020E030E040E050E46BA57CA58DA59EA52A
:10BC10000E94A3B16BA77CA78DA79EA7E0E5CE2EBF
:10BC2000EAE0DE2EE12CF12C08EC13E49E01255D08
:10BC30003F4FAE01495D5F4FBE016D5D7F4FCE014D
:10BC40004F960E94549E8AE50E946241882349F0E3
:10BC50000E944E419B01AC016FA178A589A59AA5D0
:10BC60001EC020E030E040E050E46FA178A589A537
:10BC70009AA50E94A4B16B017C016FA378A789A744
:10BC80009AA720E030E040E251E40E947DB287FFB5
:10BC90000CC020E030E040E251E4C701B6010E9450
:10BCA000A4B16FA378A789A79AA760E5C62E6AE01A
:10BCB000D62EE12CF12C06E913E49E01255D3F4FC1
:10BCC000AE01495D5F4FBE016D5D7F4FCE014F9666
:10BCD0000E94549E88E50E946241882379F00E9468
:10BCE0004E419B01AC016F8D78A189A19AA10E9460
:10BCF000A4B16F8F78A389A39AA308C080E090E0D5
:10BD0000A3E5B3E48F8F98A3A9A3BAA389E50E9402
:10BD10006241882339F00E944E416BA37CA38DA31E
:10BD20009EA304C01BA21CA21DA21EA240E5C42EFD
:10BD30004AE0D42EE12CF12C0CE812E49E01255DA2
:10BD40003F4FAE01495D5F4FBE016D5D7F4FCE013C
:10BD50004F960E94549E8CE40E946241882359F0C1
:10BD60000E944E419B01AC016BA57CA58DA59EA5B3
:10BD70000E94A4B10AC020E030E040EA52E46BA582
:10BD80007CA58DA59EA50E94A3B16BA77CA78DA7BE
:10BD90009EA720E5C22E2AE0D22EE12CF12C08EC41
:10BDA00013E49E01255D3F4FAE01495D5F4FBE012B
:10BDB0006D5D7F4FCE014F960E94549E0E94C196AA
:10BDC000149A64E670E080E090E00E943DAD0E942D
:10BDD000E06F00E010E0F12C0E94737881111BC02D
:10BDE000F3940E94E41E81E00E94574AF110F4CFC0
:10BDF000043FE1E01E0711F400E010E06A9A01152B
:10BE0000110511F4729A04C00431110509F47298F5
:10BE10000F5F1F4FE1CF729820E030E04CE852E412
:10BE20006BA57CA58DA59EA50E94A4B16BA77CA740
:10BE30008DA79EA710E5C12E1AE0D12EE12CF12C82
:10BE400000EA11E49E01255D3F4FAE01495D5F4F61
:10BE5000BE016D5D7F4FCE014F960E94549E20E043
:10BE600030E048E452E46BA57CA58DA59EA50E9418
:10BE7000A4B16BA77CA78DA79EA7E12CF12C00E0B5
:10BE800010E49E01255D3F4FAE01495D5F4FBE014D
:10BE90006D5D7F4FCE014F960E94549E1092760AA0
:10BEA0001092750A0E9446708091750A9091760AE8
:10BEB000019709F47CC01092760A1092750A0E94CC
:10BEC00079788091750A9091760A8230910549F1CE
:10BED000039709F069C020E030E048E452E46BA524
:10BEE0007CA58DA59EA50E94A4B16BA77CA78DA75C
:10BEF0009EA770E5C72E7AE0D72EE12CF12C00E04A
:10BF000010E49E01255D3F4FAE01495D5F4FBE01CC
:10BF10006D5D7F4FCE014F960E94549E0E94067029
:10BF2000C3CF20E030E04CE852E46BA57CA58DA5A2
:10BF30009EA50E94A4B16BA77CA78DA79EA7F0E544
:10BF4000CF2EFAE0DF2EE12CF12C00EA11E49E0165
:10BF5000255D3F4FAE01495D5F4FBE016D5D7F4F77
:10BF6000CE014F960E94549E20E030E048E452E417
:10BF70006BA57CA58DA59EA50E94A4B16BA77CA7EF
:10BF80008DA79EA7E12CF12C00E010E49E01255D19
:10BF90003F4FAE01495D5F4FBE016D5D7F4FCE01EA
:10BFA0004F960E94549E7ECF0E94F96F7DCF20E075
:10BFB00030E040EA50E46BA57CA58DA59EA50E94CB
:10BFC000A4B16BA77CA78DA79EA790E5C92E9AE088
:10BFD000D92EE12CF12C00E010E49E01255D3F4FAD
:10BFE000AE01495D5F4FBE016D5D7F4FCE014F9643
:10BFF0000E94549EA80197016BA57CA58DA59EA5C6
:10C000000E94A3B16BA77CA78DA79EA7E12CF12C62
:10C0100008EC13E49E01255D3F4FAE01495D5F4F83
:10C02000BE016D5D7F4FCE014F960E94549EE12C64
:10C03000F12C0CE812E49E01255D3F4FAE01495DF5
:10C040005F4FBE016B5F7F4FCE0101960E94549EF1
:10C05000E12CF12C06E913E49E01255D3F4FAE0172
:10C06000475F5F4FBE016B5F7F4FCE0101960E941D
:10C07000549E20E030E040E050E46BA57CA58DA507
:10C080009EA50E94A4B16BA77CA78DA79EA7E12CBB
:10C09000F12C08EC13E49E01255D3F4FAE01475F94
:10C0A0005F4FBE016B5F7F4FCE0101960E94549E91
:10C0B000CE010D960E94C0A880915702909158021F
:10C0C00080935D0290935E029F938F938EE999E037
:10C0D0009F938F938E01015D1F4F1F930F930E94BB
:10C0E00038BAC8010E94DF3E0F900F900F900F905A
:10C0F0000F900F908AC188E50E946241882339F031
:10C100000E944E410E94ECB280E00E94EB978AE5CB
:10C110000E946241882339F00E944E410E94ECB295
:10C1200081E00E94EB9785E40E946241882309F434
:10C130006CC10E944E410E94ECB282E00E94EB97DB
:10C1400064C183E50E946241811104C004ED14E0E2
:10C15000F12C10C010E00E944E410E94F1B2812FDC
:10C160000E94C1981F5F1530B1F7F0CFF394F4E04F
:10C17000FF1679F0F80181918F010E9462418823B6
:10C18000A9F30E944E410E94F1B28F2D0E94C198E6
:10C19000EDCF82E40E946241882339F00E944E4133
:10C1A0000E94F1B284E00E94C1980E9487992DC13B
:10C1B00083E50E946241882309F453C00E944E41E6
:10C1C0000E94ECB26130710541F06230710509F0F6
:10C1D00048C004ED14E0F12C25C004ED14E0F12C6E
:10C1E000F80181918F010E946241882341F00E94F1
:10C1F0004E410E94ECB24FEF8F2D0E948398F39432
:10C20000F4E0FF12EDCF82E40E946241882349F1FD
:10C210000E944E410E94ECB24FEF20C0F394F4E034
:10C22000FF1689F0F80181918F010E9462418823F5
:10C23000A9F30E944E410E94ECB2462F6FEF8F2D62
:10C240000E948398EBCF82E40E946241882349F0E8
:10C250000E944E410E94ECB2462F6FEF84E00E9494
:10C2600083980E948799D1C084E50E946241882307
:10C2700009F487C00E944E410E94F1B260936D089C
:10C280006623A9F1E0EBFEE08491882341F09091D0
:10C29000C00095FFFCCF8093C6003196F5CFE7E74D
:10C2A000F4E08191882339F09091C00095FFFCCF94
:10C2B0008093C600F6CF40E050E060916D0889ECB5
:10C2C0009DE00E94158EE9E7F4E08191882339F022
:10C2D0009091C00095FFFCCF8093C600F6CF80916F
:10C2E000C00085FFFCCF8AE08093C6008EC086E444
:10C2F0000E9462418823D9F00E944E416B017C016B
:10C3000060931F0A7093200A8093210A9093220A57
:10C3100020E030E0A9010E9480B4181644F4C092D5
:10C320002102D0922202E0922302F0922402E0EB5A
:10C33000FEE08491882341F09091C00095FFFCCFEE
:10C340008093C6003196F5CFEAE8F4E08191882326
:10C3500039F09091C00095FFFCCF8093C600F6CFD6
:10C360006091500A70E04AE050E089EC9DE00E9444
:10C37000DE8D8091C00085FFFCCF8AE08093C600EF
:10C3800044C0E0EBFEE08491882341F09091C0002E
:10C3900095FFFCCF8093C6003196F5CFEBE8F9E02E
:10C3A0008491882341F09091C00095FFFCCF809349
:10C3B000C6003196F5CF809188089091890820E6D3
:10C3C000289FF001299FF00D1124E257F74F81912A
:10C3D000882339F09091C00095FFFCCF8093C60070
:10C3E000F6CFE9E8F9E08491882341F09091C0000C
:10C3F00095FFFCCF8093C6003196F5CF8091C000A9
:10C4000085FFFCCF8AE08093C6000E948941B9C1B4
:10C41000C0903B0AD0903C0AE0903D0AF0903E0A62
:10C420002091700A3091710A4091720A5091730AFA
:10C43000C701B6010E94A3B12DEC3CEC4CEC5DE3CE
:10C440000E9480B4181614F00C94874CC092700AA5
:10C45000D092710AE092720AF092730A80E79AE031
:10C460000E94C0A860E080E00E94E1438AC180E0B1
:10C4700090E00E944D3D0C94844D81E090E00E943C
:10C480004D3D0C948F4D82E090E00E944D3D0C9408
:10C49000D84D0E94E41E80E00E94574A0E949F7778
:10C4A0000C948D500E945741AB01BC014093200D6C
:10C4B0005093210D6093220D7093230D8BE69CE029
:10C4C0000E941B13A2CF0E944E410E94ECB28B012E
:10C4D0000C94B1520E940EAD681979098A099B0922
:10C4E000693E73408105910508F479C0EDE6FBE0F3
:10C4F0008491882341F09091C00095FFFCCF8093F8
:10C50000C6003196F5CFE0916D0824E0E29FF0017E
:10C510001124E05AF74F408151816281738121E0FB
:10C5200030E089EC9DE00E94B48EE9E6FBE0849166
:10C53000882341F09091C00095FFFCCF8093C60006
:10C540003196F5CF60916D0870E04AE050E089ECDB
:10C550009DE00E94DE8DE5E6FBE08491882341F0BA
:10C560009091C00095FFFCCF8093C6003196F5CF27
:10C57000F7FE03C0EDEBF5E025C00E940EAD8B0188
:10C580009C01C701B6016854744F8F4F9F4F601BC9
:10C59000710B820B930BA30192010E945BB6BA014F
:10C5A000A9012AE030E089EC9DE00E940A8E80918A
:10C5B000C00085FFFCCF0DC09091C00095FFFCCF5F
:10C5C0008093C60081918111F7CF8091C00085FFD3
:10C5D000FCCF3092C6000E940EAD4B015C010E9460
:10C5E000E41E80E00E94574A0E949F77FFEFCF161B
:10C5F000DF06EF06FF0609F046C080916B08E09168
:10C600006D08F0E08F01000F111F000F111F005A7D
:10C61000174FEE0FFF1FE859F74F60817181882394
:10C62000C9F0882777FD8095982F0E941FB320E0DE
:10C6300030E040E85FE30E94A3B19B01AC01F80148
:10C6400060817181828193810E9480B487FF50C094
:10C650000C948654882777FD8095982F0E941FB3ED
:10C6600020E030E040E85FE30E94A4B19B01AC0110
:10C67000F80160817181828193810E947DB21816D8
:10C68000BCF50C948654F7FE02C00C948654E091DD
:10C690006D08F0E08F01000F111F000F111F005AED
:10C6A000174FEE0FFF1FE859F74F60817181882700
:10C6B00077FD8095982F0E941FB39B01AC01F80174
:10C6C00060817181828193810E94A3B10E94ECB24A
:10C6D00097FF07C090958095709561957F4F8F4F1C
:10C6E0009F4F663071058105910514F40C948654B2
:10C6F0000E940EAD6B017C010C94865487E59BE093
:10C700000E9403778091850A882321F08AE893E0CC
:10C710000E945E730E940EAD60937208709373085E
:10C7200080937408909375080E940EAD60937A0808
:10C7300070937B0880937C0890937D0866CE0E945E
:10C74000C19688E50E946241882319F0179A1092D9
:10C75000550A89E50E946241882319F0169A1092C1
:10C76000560A8AE50E946241882319F0159A1092B0
:10C77000570A85E40E946241882309F446CE149A40
:10C7800044CEE9960FB6F894DEBF0FBECDBFDF9161
:10C79000CF911F910F91FF90EF90DF90CF90BF90BE
:10C7A000AF909F908F907F906F905F904F903F9051
:10C7B0000895CF93DF938091840890918508039723
:10C7C00014F40E94884660E083E89AE00E94A63450
:10C7D0008091840890918508892B09F464C0809128
:10C7E000830A8823E1F0809188089091890820E6E7
:10C7F000289FE001299FD00D1124C257D74F62E72F
:10C800007DE0CE010E94ABB9892BF1F4BE0183E833
:10C810009AE00E9435348091840A882319F00E949E
:10C82000D84B2BC0EFE6FDE08491882341F0909136
:10C83000C00095FFFCCF8093C6003196F5CF809164
:10C84000C00085FFFCCF16C060E083E89AE00E943C
:10C850009C35EDE5FDE08491882341F09091C00086
:10C8600095FFFCCF8093C6003196F5CF8091C00034
:10C8700085FFFCCF8AE08093C60080918408909168
:10C880008508019790938508809384088091880893
:10C8900090918908019664E070E00E9448B69093F8
:10C8A0008908809388080E94E41E80E00E94574A0D
:10C8B0000E94D38EDF91CF910C949F778F929F929D
:10C8C000AF92BF92CF92DF92EF92FF920F931F939E
:10C8D000CF93DF938C018C519E4F0E94492E6801AB
:10C8E00089E8C80ED11C21F1780181E4E81A8EEFA5
:10C8F000F80AE70157018FE1A81AB1087AED872EEF
:10C9000075E0972ECC15DD0599F0FE01EE19FF09B3
:10C91000EA0DFB1D91828082FE0178978081811152
:10C9200002C06F97EFCFCE014B970E94FE13F9CF55
:10C93000C80186599F4F0E94492EC801875B9F4FAF
:10C94000DF91CF911F910F91FF90EF90DF90CF90EB
:10C95000BF90AF909F908F900C94492E83E89AE0FF
:10C960000C94552E83E89AE0A9CFFB0160917002E8
:10C97000709171027093520D6093510D60915B0D37
:10C9800070915C0D7093500D60934F0D62E0609359
:10C990006F0263EA71E87093710260937002909382
:10C9A0004E0D80934D0DF0934C0DE0934B0D66278B
:10C9B00057FD6095762F4093470D5093480D609337
:10C9C000490D70934A0DC901AA2797FDA095BA2F6A
:10C9D000841B950BA60BB70B8093430D9093440DCE
:10C9E000A093450DB093460D80819181AA2797FDB4
:10C9F000A095BA2F841B950BA60BB70B80935B0DEC
:10CA000090935C0DA0935D0DB0935E0D08950F9310
:10CA10001F93CF93DF93EB01142F022F482F60E079
:10CA200086E69DE00E94F028612F86E69DE00E9448
:10CA30009CB111E1FE016491662311F0111117C040
:10CA4000112339F060E286E69DE00E949CB111500E
:10CA5000F7CF602F86E69DE00E949CB160E286E6FB
:10CA60009DE0DF91CF911F910F910C949CB186E6D0
:10CA70009DE00E949CB121961150DCCFEF92FF9275
:10CA80000F931F93CF93DF93EB01E42E8901F901FC
:10CA900001900020E9F7F22EFE1A92E1F90E482FDC
:10CAA00060E086E69DE00E94F0286E2D86E69DE01F
:10CAB0000E949CB1FE016491662311F0F11019C02F
:10CAC0006AE386E69DE00E949CB1FF2039F060E2B7
:10CAD00086E69DE00E949CB1FA94F7CFB80186E605
:10CAE0009DE0DF91CF911F910F91FF90EF900C94FB
:10CAF0009BB186E69DE00E949CB12196FA94DACF24
:10CB00001092C00D83E89AE00E94463A1092640D9C
:10CB1000089583E89AE00C94A83183E89AE00C9495
:10CB2000AF31CF93DF93CDB7DEB7C054D1090FB685
:10CB3000F894DEBF0FBECDBF88E0EBEBF2E0DE0184
:10CB4000D99601900D928A95E1F788E0E3ECF2E046
:10CB5000DE01D19601900D928A95E1F788E0EBEC29
:10CB6000F2E0DE01999601900D928A95E1F788E056
:10CB7000E3EDF2E0DE01919601900D928A95E1F7E6
:10CB800088E0EBEDF2E0DE01599601900D928A9576
:10CB9000E1F788E0E3EEF2E0DE01519601900D92BC
:10CBA0008A95E1F788E0EBEEF2E0DE01199601905C
:10CBB0000D928A95E1F788E0E3EFF2E0DE0111964D
:10CBC00001900D928A95E1F7AE01475C5F4F60E0FE
:10CBD00086E69DE00E948E2AAE014F5C5F4F61E0C9
:10CBE00086E69DE00E948E2AAE01475D5F4F62E0BF
:10CBF00086E69DE00E948E2AAE014F5D5F4F63E0A6
:10CC000086E69DE00E948E2AAE01475E5F4F64E09B
:10CC100086E69DE00E948E2AAE014F5E5F4F65E082
:10CC200086E69DE00E948E2AAE01475F5F4F66E078
:10CC300086E69DE00E948E2AAE014F5F5F4F67E05F
:10CC400086E69DE00E948E2AC05CDF4F0FB6F89406
:10CC5000DEBF0FBECDBFDF91CF910895CF9382E0AD
:10CC600080936F020E940EAD6C507E4F8F4F9F4F8E
:10CC70006093600D7093610D8093620D9093630DCE
:10CC80006A9ACAE0729A84E690E00E9461AD729856
:10CC900084E690E00E9461ADC150A1F7CF91089564
:10CCA000E0917002F0917102E817F90771F090932A
:10CCB00071028093700240935B0D50935C0D609302
:10CCC0005D0D70935E0D2111C9CF089521E040E004
:10CCD00050E0BA01E5CF21E040E050E0BA01E0CFFA
:10CCE000CF92DF92EF92FF920F931F93CF93DF9338
:10CCF00080915B0D90915C0DA0915D0DB0915E0DEA
:10CD000081309048A105B10540F010925B0D109262
:10CD10005C0D10925D0D10925E0D80915B0D9091F7
:10CD20005C0DA0915D0DB0915E0DB695A7959795A0
:10CD300087954091640D50E060E070E0841795079E
:10CD4000A607B70710F48093640DD091640D10917D
:10CD5000650D12FB112710F9C0E0FBE0CF2ED12C9E
:10CD6000E12CF12C01E040915B0D50915C0D609144
:10CD70005D0D70915E0DD1112DC080916F028823E1
:10CD800069F023E0423051056105710510F443E07C
:10CD900001C040E26AE671E18C2F39DE112309F40B
:10CDA000F1C080915B0D90915C0DA0915D0DB091F3
:10CDB0005E0D0297A105B10508F0E4C04FDF82E8DF
:10CDC00093E7DF91CF911F910F91FF90EF90DF904C
:10CDD000CF907CCFD13051F580916F02882389F0BC
:10CDE000769567955795479523E041305105610544
:10CDF000710511F443E001C040E268E571E18C2F58
:10CE000006DE112309F4BEC080915B0D90915C0D8C
:10CE1000A0915D0DB0915E0DB695A79597958795FC
:10CE20000197A105B10509F0ADC0C8CFD23051F5C9
:10CE300080916F02882389F076956795579547957D
:10CE400023E0423051056105710511F443E001C052
:10CE500040E26CE471E18C2FDADD112309F492C019
:10CE600080915B0D90915C0DA0915D0DB0915E0D78
:10CE7000B695A795979587950297A105B10509F0F5
:10CE800081C09CCFD33051F580916F02882389F007
:10CE9000769567955795479523E043305105610591
:10CEA000710511F443E001C040E26AE371E18C2FA7
:10CEB000AEDD112309F466C080915B0D90915C0D8D
:10CEC000A0915D0DB0915E0DB695A795979587954C
:10CED0000397A105B10509F055C070CFD43041F5D5
:10CEE00080916F02882389F07695679557954795CD
:10CEF00023E0443051056105710511F443E001C0A0
:10CF000040E268E271E18C2F82DD1123D9F180913A
:10CF10005B0D90915C0DA0915D0DB0915E0DB6958D
:10CF2000A795979587950497A105B10559F546CF23
:10CF3000D53041F580916F02882389F07695679509
:10CF40005795479523E0453051056105710511F46A
:10CF500043E001C040E26CE171E18C2F58DD112308
:10CF600089F080915B0D90915C0DA0915D0DB09169
:10CF70005E0DB695A795979587950597A105B1057F
:10CF800009F41CCF80915B0D90915C0DA0915D0D1B
:10CF9000B0915E0D0C97A105B10540F0C0925B0DFC
:10CFA000D0925C0DE0925D0DF0925E0D40915B0DB4
:10CFB00050915C0D60915D0D70915E0D7695679559
:10CFC000579547958091640D90E00396242F30E0AB
:10CFD000821793074CF48DEF840F8093640D0093B8
:10CFE0006F02DCEFD40FCFEFCF5FDF5FC43008F408
:10CFF000BACEDF91CF911F910F91FF90EF90DF900C
:10D00000CF9008950F931F93CF93DF9380915B0D83
:10D0100090915C0DA0915D0DB0915E0D81309048B6
:10D02000A105B10540F010925B0D10925C0D1092BD
:10D030005D0D10925E0D80915B0D90915C0DA09145
:10D040005D0DB0915E0DB695A7959795879540912A
:10D05000640D50E060E070E084179507A607B707FD
:10D0600010F48093640DD091640D1091650D12FB46
:10D07000112710F9C0E001E080915B0D90915C0DEB
:10D08000A0915D0DB0915E0DD11128C020916F026D
:10D09000222361F023E00297A105B10510F443E0DB
:10D0A00001C040E26FE970E18C2FB1DC112309F47B
:10D0B0006EC080915B0D90915C0DA0915D0DB09163
:10D0C0005E0D0297A105B10508F061C0C7DD81E2E0
:10D0D00091E7DF91CF911F910F91F8CDD13059F5A4
:10D0E00020916F02222381F0B695A7959795879599
:10D0F0002EE70197A105B10511F44EE301C040E20E
:10D1000068E970E18C2F83DC112309F440C0809121
:10D110005B0D90915C0DA0915D0DB0915E0DB6958B
:10D12000A795979587950197A105B10581F596DD9E
:10D130008FEE92E89FC0D23051F520916F022223EA
:10D1400081F0B695A795979587952EE70297A1054B
:10D15000B10511F44EE301C040E261E970E18C2FAA
:10D1600056DC1123A1F080915B0D90915C0DA09194
:10D170005D0DB0915E0DB695A79597958795029731
:10D18000A105B10521F46ADD86EF92E873C020E0C5
:10D1900030E040E251E46091370D7091380D80919C
:10D1A000390D90913A0D0E947DB287FF68C0809141
:10D1B0005B0D90915C0DA0915D0DB0915E0DD33033
:10D1C00061F520916F02222381F0B695A79597957E
:10D1D00087952EE70397A105B10511F44EE301C031
:10D1E00040E26AE870E18C2F12DC111102C025E0E8
:10D1F00047C080915B0D90915C0DA0915D0DB09149
:10D200005E0DB695A795979587950397A105B105EE
:10D2100071F724DD8DEF92E82DC0D43041F72091D5
:10D220006F02222381F0B695A795979587952EE7F3
:10D230000497A105B10511F44EE301C040E261E895
:10D2400070E18C2FE4DB112391F240915B0D509142
:10D250005C0D60915D0D70915E0D769567955795AB
:10D260004795443051056105710509F0C0CFF6DCE2
:10D270008AE291E8DF91CF911F910F912CCD23E0AD
:10D2800040915B0D50915C0D60915D0D70915E0D54
:10D290007695679557954795822F90E0A0E0B0E08E
:10D2A000481759076A077B0788F0822F90E0880F9C
:10D2B000991F0197AA2797FDA095BA2F80935B0D20
:10D2C00090935C0DA0935D0DB0935E0D40915B0D4E
:10D2D00050915C0D60915D0D70915E0D7695679536
:10D2E000579547958091640D90E00396242F30E088
:10D2F000821793074CF48DEF840F8093640D009395
:10D300006F02DCEFD40FCFEFCF5FDF5FC43008F4E4
:10D31000B3CEDF91CF911F910F91089580E090E0FF
:10D32000A0E8BFE38093370D9093380DA093390D9B
:10D33000B0933A0D67CE20E044E064E186E69DE0DC
:10D340000E942329EEDB86E69DE00C94E428F3DFBF
:10D3500020E040E050E0BA018FE993E8A1CC1092C0
:10D360006908109268081092670810926608109277
:10D370004F0A10924E0AEBCF86E69DE00C94E4280B
:10D3800020E030E04EE353E4609160087091610862
:10D3900080916208909163080E9480B418164CF442
:10D3A00081E09FE00E94523F84EF9EE00E94523F46
:10D3B00020C0E2DF40E060E086E69DE00E94F028C9
:10D3C00068ED74E086E69DE00E949BB142E060E07B
:10D3D00086E69DE00E94F0286FED74E086E69DE011
:10D3E0000E949BB160ED77E080E090E00E943DAD4F
:10D3F000C3DFADCF20E030E04EE353E4609160083E
:10D400007091610880916208909163080E9480B4D5
:10D4100018166CF480EF9EE00E94523F84EE9EE06E
:10D420000E94523F88ED9EE00E94523F20C0A4DF40
:10D4300040E060E086E69DE00E94F02868ED74E040
:10D4400086E69DE00E949BB142E060E086E69DE0BA
:10D450000E94F0286FED74E086E69DE00E949BB18B
:10D4600060ED77E080E090E00E943DAD85DF6FCF1A
:10D470008091BD0D9091BE0D9093690880936808CE
:10D480008091BB0D9091BC0D9093670880936608C6
:10D4900010924F0A10924E0A5ADF0C94B6218091D6
:10D4A000B70D9091B80D90936908809368088091AA
:10D4B000B50D9091B60D9093670880936608109211
:10D4C0004F0A10924E0A43DF0C94B62180919502C8
:10D4D00090919602909369088093680880919302D6
:10D4E00090919402909367088093660810924F0A77
:10D4F00010924E0A2CDF0C94B621809191029091EB
:10D500009202909369088093680880918F029091AD
:10D510009002909367088093660810924F0A1092C9
:10D520004E0A15DF0C94B62180918D0290918E02E7
:10D53000909369088093680880918B0290918C0287
:10D54000909367088093660810924F0A10924E0AD3
:10D55000FEDE0C94B6218091890290918A0290930C
:10D56000690880936808809187029091880290935F
:10D5700067088093660810924F0A10924E0AE7DE01
:10D580000C94B6212F923F924F925F926F927F92AE
:10D590008F929F92AF92BF92CF92DF92EF92FF92C3
:10D5A0000F931F93CF93DF93CDB7DEB7A2970FB63C
:10D5B000F894DEBF0FBECDBF80916F02811104C011
:10D5C0008091650D82FFA9C283E89AE00E943A39F2
:10D5D00040915B0D50915C0D60915D0D70915E0D01
:10D5E000413050486105710540F010925B0D10927A
:10D5F0005C0D10925D0D10925E0D40915B0D50918F
:10D600005C0D60915D0D70915E0D769567955795F7
:10D6100047950091640D10E020E030E0401751077D
:10D620006207730710F44093640D4090640D3090CE
:10D63000650D32FA332430F8512C9C012150310908
:10D6400039A328A341102BC080916F028823A1F039
:10D6500080915B0D90915C0DA0915D0DB0915E0D80
:10D6600023E00297A105B10510F443E001C040E2B8
:10D670006AE370E1852DCBD9332089F080915B0D71
:10D6800090915C0DA0915D0DB0915E0D0297A1058A
:10D69000B10528F4E3DA82E893E718DB3EC267E8D5
:10D6A0007AE081EF9AE00E94B2108091870A8F326F
:10D6B00029F031E0431669F022E001C021E0A8A082
:10D6C000B9A0C42CD12CE12CF12C22242394240CBD
:10D6D00049C080916F028823C1F080915B0D9091C9
:10D6E0005C0DA0915D0DB0915E0DB695A7959795D7
:10D6F000879520E20197A105B10511F44EE301C021
:10D7000040E266E370E1852D82D93320A9F2809151
:10D710005B0D90915C0DA0915D0DB0915E0DB69585
:10D72000A795979587950197A105B10529F696DAF2
:10D73000E7D9F3C124115FC140E050E0B50183E8AF
:10D740009AE00E94B1359091C90A80916F029923A5
:10D7500009F49AC081110BC0311074C0222DF1E080
:10D76000AF1AB1083FEFA316B30621F746C1809167
:10D770005B0D90915C0DA0915D0DB0915E0DB69525
:10D78000A79597958795452D60E08C159D05AE056D
:10D79000BF0561F586E69DE00E94F0286EE386E60F
:10D7A0009DE00E949CB165E086E69DE00E949CB1F0
:10D7B0008091940A882329F01092A60A04E91AE0BD
:10D7C00002C007E81AE0B2E19B2EF80161918F01D7
:10D7D000662311F0911060C1992009F4BDCF60E279
:10D7E00086E69DE00E949CB19A94F6CF86E69DE085
:10D7F0000E94F02860E286E69DE00E949CB165E010
:10D8000086E69DE00E949CB18091940A882329F0CD
:10D810001092A60A04E91AE002C007E81AE0A2E1A1
:10D820009A2EF80161918F01662311F091103AC18F
:10D83000992009F491CF60E286E69DE00E949CB1B8
:10D840009A94F6CF80915B0D90915C0DA0915D0D47
:10D85000B0915E0DB695A795979587958C159D050A
:10D86000AE05BF0509F07ACFF9D967E87AE083E819
:10D870009AE00E949D3910925B0D10925C0D1092FF
:10D880005D0D10925E0D49C1811103C0311071C050
:10D8900065CF80915B0D90915C0DA0915D0DB09175
:10D8A0005E0DB695A795979587958C159D05AE0548
:10D8B000BF05B1F52091C80D2F8F10E0412F60E01A
:10D8C00086E69DE00E94F02860E286E69DE00E94E8
:10D8D0009CB11F5F143091F7452D60E086E69DE016
:10D8E0000E94F0286EE386E69DE00E949CB165E907
:10D8F000862E6AE0962E74E9672E7AE0772E01E094
:10D9000010E0F30121913F012111D2C014E1101B5D
:10D9100060E286E69DE00E949CB11150C9F7B6CF47
:10D92000452D60E086E69DE00E94F02860E286E6F4
:10D930009DE00E949CB18091940A882329F0109266
:10D94000A70A04E91AE002C007E81AE053E1952E9D
:10D95000F80161918F01662311F09110D8C09920D0
:10D9600009F494CF60E286E69DE00E949CB19A940F
:10D97000F6CF80915B0D90915C0DA0915D0DB09103
:10D980005E0DB695A795979587958C159D05AE0567
:10D99000BF0509F0E3CE62D987E89AE09F938F93A1
:10D9A0008FE290E19F938F938E010F5F1F4F1F9324
:10D9B0000F930E9438BA0F900F900F900F900F9016
:10D9C0000F907E01F5E0EF0EF11CF70180818823B6
:10D9D00049F0992787FD90950E9475B9F7018193C9
:10D9E0007F01F3CFC8010E94DF3E8BE290E10E94ED
:10D9F000523FADDC92C02F5FB2CE80915B0D909113
:10DA00005C0DA0915D0DB0915E0DB695A7959795B3
:10DA10008795422F50E060E070E084179507A607D5
:10DA2000B70788F0822F90E0880F991F0197AA27E7
:10DA300097FDA095BA2F80935B0D90935C0DA093FA
:10DA40005D0DB0935E0D80915B0D90915C0DA0918A
:10DA50005D0DB0915E0DB695A79597958795209130
:10DA6000640D30E02D5F3F4F482F50E024173507FD
:10DA700064F42DEF280F2093640D21E020936F02B2
:10DA8000FCEF4F2E480E55245A945394439483E050
:10DA9000851508F0D7CD41C086E69DE00E949CB177
:10DAA0009A9493CE86E69DE00E949CB19A94B9CE5A
:10DAB000452D602F86E69DE02AA30E94F0282AA12A
:10DAC000622F86E69DE00E949CB10F5F1F4F0431DC
:10DAD000110509F016CF34010CE211E08091650DBB
:10DAE00082FD05C08091C80D3F8D381749F0015067
:10DAF00011090115110591F78FEF881A980AFFCEC9
:10DB000061E070E080E090E00E943DADF0CF86E6FD
:10DB10009DE00E949CB19A941BCFA2960FB6F894F8
:10DB2000DEBF0FBECDBFDF91CF911F910F91FF9050
:10DB3000EF90DF90CF90BF90AF909F908F907F90AD
:10DB40006F905F904F903F902F900895CF92DF920B
:10DB5000EF92FF920F931F93CF93DF9380915B0D12
:10DB600090915C0DA0915D0DB0915E0D813090485B
:10DB7000A105B10540F010925B0D10925C0D109262
:10DB80005D0D10925E0D80915B0D90915C0DA091EA
:10DB90005D0DB0915E0DB695A795979587954091CF
:10DBA000640D50E060E070E084179507A607B707A2
:10DBB00010F48093640DD091640D1091650D12FBEB
:10DBC000112710F9C0E0BFE0CB2ED12CE12CF12CB5
:10DBD00001E040915B0D50915C0D60915D0D709185
:10DBE0005E0DD1112EC080916F02882371F023E069
:10DBF000423051056105710510F443E001C040E277
:10DC000066E170E18C2F0E940765112309F498C129
:10DC100080915B0D90915C0DA0915D0DB0915E0DBA
:10DC20000297A105B10508F08BC118D882E893E7E7
:10DC3000DF91CF911F910F91FF90EF90DF90CF90E8
:10DC400045C8D130A9F580916F02882391F076956F
:10DC500067955795479520E241305105610571055B
:10DC600011F44EE301C040E266E070E18C2F0E94A7
:10DC70000765112309F464C180915B0D90915C0DDF
:10DC8000A0915D0DB0915E0DB695A795979587957E
:10DC90000197A105B10509F053C10E942E66DF91DD
:10DCA000CF911F910F91FF90EF90DF90CF90F7CB26
:10DCB000D230A9F580916F02882391F0769567950F
:10DCC0005795479520E2423051056105710511F4E1
:10DCD0004EE301C040E267EF7FE08C2F0E940765B2
:10DCE000112309F42DC180915B0D90915C0DA091E1
:10DCF0005D0DB0915E0DB695A795979587950297A6
:10DD0000A105B10509F01CC10E942E66DF91CF91DB
:10DD10001F910F91FF90EF90DF90CF90A9CBD33060
:10DD2000A9F580916F02882391F0769567955795B4
:10DD3000479520E2433051056105710511F44EE32A
:10DD400001C040E268EE7FE08C2F0E94076511233E
:10DD500009F4F6C080915B0D90915C0DA0915D0D72
:10DD6000B0915E0DB695A795979587950397A105F8
:10DD7000B10509F0E5C00E942E66DF91CF911F9199
:10DD80000F91FF90EF90DF90CF90B7CBD430A9F5F3
:10DD900080916F02882391F0769567955795479506
:10DDA00020E2443051056105710511F44EE301C0D4
:10DDB00040E268ED7FE08C2F0E940765112309F493
:10DDC000BFC080915B0D90915C0DA0915D0DB091F5
:10DDD0005E0DB695A795979587950497A105B10512
:10DDE00009F0AEC00E942E66DF91CF911F910F9176
:10DDF000FF90EF90DF90CF9097CBD530A9F5809131
:10DE00006F02882391F0769567955795479520E2A4
:10DE1000453051056105710511F44EE301C040E242
:10DE200068EC7FE08C2F0E940765112309F488C0FD
:10DE300080915B0D90915C0DA0915D0DB0915E0D98
:10DE4000B695A795979587950597A105B10509F012
:10DE500077C00E942E66DF91CF911F910F91FF90A6
:10DE6000EF90DF90CF9032CBD630A9F580916F0242
:10DE7000882391F0769567955795479520E246302F
:10DE800051056105710511F44EE301C040E269EBF3
:10DE90007FE08C2F0E940765112309F451C0809107
:10DEA0005B0D90915C0DA0915D0DB0915E0DB695EE
:10DEB000A795979587950697A105B10509F040C0EC
:10DEC0000E942E66DF91CF911F910F91FF90EF90EE
:10DED000DF90CF9040CBD73099F580916F028823A7
:10DEE00091F0769567955795479520E24730510513
:10DEF0006105710511F44EE301C040E260EB7FE083
:10DF00008C2F0E9407651123D9F080915B0D9091B1
:10DF10005C0DA0915D0DB0915E0DB695A79597959E
:10DF200087950797A105B10559F40E942E66DF91E8
:10DF3000CF911F910F91FF90EF90DF90CF900FCA7C
:10DF400080915B0D90915C0DA0915D0DB0915E0D87
:10DF50004097A105B10540F0C0925B0DD0925C0DD9
:10DF6000E0925D0DF0925E0D40915B0D50915C0D65
:10DF700060915D0D70915E0D76956795579547950B
:10DF80008091640D90E00396242F30E08217930770
:10DF90004CF48DEF840F8093640D00936F02DCEFDF
:10DFA000D40FCFEFCF5FDF5FC43008F412CEDF9124
:10DFB000CF911F910F91FF90EF90DF90CF90089538
:10DFC000DBD941E060E086E69DE00E94F02866E053
:10DFD00075E086E69DE00E949BB142E060E086E647
:10DFE0009DE00E94F02866E175E086E69DE00C94D5
:10DFF0009BB1C2D942E060E086E69DE00E94F02835
:10E0000069E275E086E69DE00C949BB11F93CF9387
:10E01000DF93B2D940E060E086E69DE00E94F02800
:10E0200069E375E086E69DE00E949BB142E060E016
:10E0300086E69DE00E94F02867E475E086E69DE0B4
:10E040000E949BB110E043E0612F86E69DE00E94B4
:10E05000F0286BE673E086E69DE00E949BB1CAE083
:10E06000D0E00E94E41E81E00E94574A65E570E01E
:10E0700080E090E00E943DAD2197209791F71F5FCF
:10E08000143109F7DF91CF911F9108951F93CF931A
:10E09000DF9372D940E060E086E69DE00E94F028C0
:10E0A00063E575E086E69DE00E949BB142E060E09A
:10E0B00086E69DE00E94F02867E475E086E69DE034
:10E0C0000E949BB110E043E0612F86E69DE00E9434
:10E0D000F0286BE673E086E69DE00E949BB1CAE003
:10E0E000D0E00E94E41E81E00E94574A6EE670E094
:10E0F00080E090E00E943DAD2197209791F71F5F4F
:10E10000143109F7DF91CF911F9108951F93CF9399
:10E11000DF93EC01FB01608111810E945CBC612FE7
:10E12000CE010196DF91CF911F910C945CBCFF92C0
:10E130000F931F93CF93DF938C01EB010E9454BC8C
:10E14000F82EC80101960E9454BCF8828983DF91A1
:10E15000CF911F910F91FF900895EF92FF920F932F
:10E160001F93CF93DF931F92CDB7DEB77B018C0156
:10E17000061B170B460FC701800F911FF701619116
:10E180007F0149830E945CBC49814E11F4CF0F90FE
:10E19000DF91CF911F910F91FF90EF90089581E053
:10E1A0009091BF0D911180E08093BF0D41E06FEB26
:10E1B0007DE08FEF9FE0D1DF0E941B9821E047E0D8
:10E1C00050E060E070E081E291E70C94506681E0FD
:10E1D0009091BF0D911180E08093BF0D41E06FEBF6
:10E1E0007DE08FEF9FE0B9DF0E941B9821E049E0BE
:10E1F00050E060E070E084E39DE70C945066EF929D
:10E20000FF920F931F93CF93DF931F92CDB7DEB78B
:10E210007B018C01061B170B460FC701800F911F56
:10E2200049830E9454BCF70181937F0149814E13B9
:10E23000F4CF0F90DF91CF911F910F91FF90EF904E
:10E240000895CF92DF92EF92FF920F931F93CF9397
:10E25000DF9341E06FEB7DE08FEF9FE0D0DF8091B7
:10E260005B0D90915C0DA0915D0DB0915E0D8130C4
:10E270009048A105B10540F010925B0D10925C0D25
:10E2800010925D0D10925E0D80915B0D90915C0D72
:10E29000A0915D0DB0915E0DB695A7959795879568
:10E2A0004091640D50E060E070E084179507A60788
:10E2B000B70710F48093640DD091640D1091650D33
:10E2C00012FB112710F9C0E0BDE0CB2ED12CE12CC0
:10E2D000F12C01E040915B0D50915C0D60915D0D62
:10E2E00070915E0DD11130C080916F02882371F062
:10E2F00023E0423051056105710510F443E001C08F
:10E3000040E267E171E18C2F0E940765112309F457
:10E310001FC180915B0D90915C0DA0915D0DB0913E
:10E320005E0D0297A105B10508F012C10E942E668C
:10E3300082E893E7DF91CF911F910F91FF90EF90CB
:10E34000DF90CF900C946666D13079F580916F02A2
:10E35000882391F076956795579547952EE741303C
:10E3600051056105710511F44EE301C040E26BE017
:10E3700071E18C2F0E940765112309F4E9C0809197
:10E380005B0D90915C0DA0915D0DB0915E0DB69509
:10E39000A795979587950197A105B10509F0D8C074
:10E3A0000E942E6687E99BE730C0D230C1F580918C
:10E3B0006F02882391F076956795579547952EE7DC
:10E3C000423051056105710511F44EE301C040E290
:10E3D00061E071E18C2F0E940765112309F4B8C038
:10E3E00080915B0D90915C0DA0915D0DB0915E0DE3
:10E3F000B695A795979587950297A105B10509F060
:10E40000A7C00E942E668EE899E6DF91CF911F91FA
:10E410000F91FF90EF90DF90CF900C946B66D3300C
:10E4200079F580916F02882391F0769567955795DD
:10E43000479520E2433051056105710511F44EE323
:10E4400001C040E265EF70E18C2F0E940765112347
:10E4500009F47EC080915B0D90915C0DA0915D0DE3
:10E46000B0915E0DB695A795979587950397A105F1
:10E47000B10509F06DC00E942E668FEE90E12FC0AD
:10E48000D430B9F580916F02882391F07695679525
:10E490005795479520E2443051056105710511F407
:10E4A0004EE301C040E26EED70E18C2F0E940765E3
:10E4B000112309F44DC080915B0D90915C0DA091EA
:10E4C0005D0DB0915E0DB695A795979587950497CC
:10E4D000A105B105E9F50E942E668AED90E1DF9174
:10E4E000CF911F910F91FF90EF90DF90CF900C9400
:10E4F000523FD53069F580916F02882391F076956F
:10E5000067955795479520E245305105610571059E
:10E5100011F44EE301C040E260ED70E18C2F0E94E7
:10E5200007651123A9F080915B0D90915C0DA0917E
:10E530005D0DB0915E0DB695A7959795879505975A
:10E54000A105B10529F40E942E668CEC90E1C7CF9D
:10E550002091BF0D80915B0D90915C0DA0915D0DA0
:10E56000B0915E0D211135C0D63009F047C0209121
:10E570006F02222389F0B695A7959795879520E29B
:10E580000697A105B10511F44EE301C040E26AEB24
:10E5900070E18C2F0E940765112381F180915B0D42
:10E5A00090915C0DA0915D0DB0915E0DB695A79513
:10E5B000979587950697A105B10501F50E942E66EE
:10E5C000DF91CF911F910F91FF90EF90DF90CF904F
:10E5D000E6CDD63099F420916F022223E9F2B69568
:10E5E000A7959795879520E20697A105B10511F4A7
:10E5F0004EE301C040E268EA70E1CBCF80915B0D51
:10E6000090915C0DA0915D0DB0915E0D0E97A105EE
:10E61000B10540F0C0925B0DD0925C0DE0925D0DB3
:10E62000F0925E0D40915B0D50915C0D60915D0D1F
:10E6300070915E0D76956795579547958091640D1D
:10E6400090E00396242F30E0821793074CF48DEF6F
:10E65000840F8093640D00936F02DCEFD40FCFEF33
:10E66000CF5FDF5FC43008F435CEDF91CF911F91CB
:10E670000F91FF90EF90DF90CF9008958093540D0D
:10E680001092530D0895E2E7F2E001900020E9F7BF
:10E690003197E257F2401E161F0634F010928602A0
:10E6A00082E080936F02089580E2E431F105B4F7CF
:10E6B000DF01AE58BD4F8C933196F7CF2091B20D4C
:10E6C000211108C044E150E0BC0182E792E00E94C1
:10E6D00029BAD9CF08951092850A60E083E89AE0BC
:10E6E0000E949C350E9437978FE190E10E94523F33
:10E6F00081E080933F0A84E695E0E0DF8BE190E1E2
:10E700000C94523F8F929F92AF92BF92DF92EF9202
:10E71000FF920F931F93CF93DF931092C00D8091C0
:10E720005B0D90915C0DA0915D0DB0915E0D8130FF
:10E730009048A105B10540F010925B0D10925C0D60
:10E7400010925D0D10925E0D80915B0D90915C0DAD
:10E75000A0915D0DB0915E0DB695A79597958795A3
:10E760004091640D50E060E070E084179507A607C3
:10E77000B70710F48093640DD091640D1091650D6E
:10E7800012FB112710F9C0E0DD24D394D11138C059
:10E7900080916F028823A9F080915B0D90915C0DB0
:10E7A000A0915D0DB0915E0D23E00297A105B1052A
:10E7B00010F443E001C040E268EE71E18C2F0E944A
:10E7C00007651123E9F080915B0D90915C0DA0919C
:10E7D0005D0DB0915E0D0297A105B10588F40E9410
:10E7E0002E668FE993E8DF91CF911F910F91FF90F3
:10E7F000EF90DF90BF90AF909F908F900C946666E3
:10E800000E94DDA840915B0D50915C0D60915D0D03
:10E8100070915E0D811104C08091850A882379F181
:10E82000D130A9F580916F02882391F07695679594
:10E83000579547952EE7413051056105710511F453
:10E840004EE301C040E263EE71E18C2F0E94076548
:10E850001123E9F080915B0D90915C0DA0915D0D0D
:10E86000B0915E0DB695A795979587950197A105EF
:10E87000B10569F40E942E6684E39DE736C2D1306B
:10E8800031F480916F02811195C21111A6C280915D
:10E89000860A40915B0D50915C0D60915D0D709109
:10E8A0005E0D882309F4ECC080916E0C882309F476
:10E8B000B6C08091850A8823E1F1D23009F074C096
:10E8C00080916F02882391F07695679557954795CB
:10E8D00020E2423051056105710511F44EE301C09B
:10E8E00040E26FEC71E18C2F0E940765112309F45F
:10E8F000DDC080915B0D90915C0DA0915D0DB0919C
:10E900005E0DB695A795979587950297A105B105D8
:10E9100009F0CCC00E942E66DF91CF911F910F911C
:10E92000FF90EF90DF90BF90AF909F908F900C94EE
:10E930008D65D230C9F580916F02882391F076956C
:10E9400067955795479520E242305105610571055D
:10E9500011F44EE301C040E262EC71E18C2F0E94A1
:10E960000765112309F4A2C080915B0D90915C0DA5
:10E97000A0915D0DB0915E0DB695A7959795879581
:10E980000297A105B10509F091C00E942E66DF91A2
:10E99000CF911F910F91FF90EF90DF90BF90AF90BC
:10E9A0009F908F900C948965D33009F07FC080913F
:10E9B0006F02882391F0769567955795479520E2E9
:10E9C000433051056105710511F44EE301C040E289
:10E9D00067EB71E18C2F0E940765112309F466C073
:10E9E00080915B0D90915C0DA0915D0DB0915E0DDD
:10E9F000B695A795979587950397A105B10509F059
:10EA000055C00E942E66DF91CF911F910F91FF900C
:10EA1000EF90DF90BF90AF909F908F905CCED23000
:10EA200011F003E044C080916F02882391F0769545
:10EA30006795579547952EE7423051056105710559
:10EA400011F44EE301C040E269EA71E18C2F0E94AB
:10EA50000765112331F380915B0D90915C0DA091BE
:10EA60005D0DB0915E0DB695A79597958795029728
:10EA7000A105B105B1F60E942E6682EC9AE635C179
:10EA8000D23079F680916F02882319F376956795D5
:10EA9000579547952EE7423051056105710511F4F0
:10EAA0004EE301C040E26EE971E1D0CF04E0809115
:10EAB000850A8111DBC00D1348C080916F02882345
:10EAC000F1F080915B0D90915C0DA0915D0DB09186
:10EAD0005E0DB695A79597958795402F50E060E01D
:10EAE00070E020E284179507A607B70711F44EE3FC
:10EAF00001C040E260E971E18C2F0E94076511239B
:10EB000021F180915B0D90915C0DA0915D0DB09114
:10EB10005E0DB695A79597958795402F50E060E0DC
:10EB200070E084179507A607B70779F40E942E6650
:10EB3000DF91CF911F910F91FF90EF90DF90BF90E9
:10EB4000AF909F908F900C94FA69EE24E394E00EBE
:10EB5000ED1248C080916F028823F1F080915B0D27
:10EB600090915C0DA0915D0DB0915E0DB695A7954D
:10EB7000979587958D2E912CA12CB12C20E288158C
:10EB80009905AA05BB0511F44EE301C040E260E817
:10EB900071E18C2F0E940765112321F180915B0D9B
:10EBA00090915C0DA0915D0DB0915E0DB695A7950D
:10EBB000979587954E2D50E060E070E0841795079B
:10EBC000A607B70779F40E942E66DF91CF911F91B7
:10EBD0000F91FF90EF90DF90BF90AF909F908F903C
:10EBE0000C94C069E2E0EE2EE00EED123EC0809182
:10EBF0006F028823F1F080915B0D90915C0DA091E4
:10EC00005D0DB0915E0DB695A795979587958D2E64
:10EC1000912CA12CB12C2EE788159905AA05BB05CE
:10EC200011F44EE301C040E267E771E18C2F0E94CE
:10EC300007651123D1F080915B0D90915C0DA0913F
:10EC40005D0DB0915E0DB695A795979587954E2D64
:10EC500050E060E070E084179507A607B70729F435
:10EC60000E942E6681E291E740C00D5F0D134AC0FD
:10EC700080916F028823F1F080915B0D90915C0D83
:10EC8000A0915D0DB0915E0DB695A795979587956E
:10EC9000402F50E060E070E02EE784179507A6074C
:10ECA000B70711F44EE301C040E26FE671E18C2F2B
:10ECB0000E940765112331F180915B0D90915C0DED
:10ECC000A0915D0DB0915E0DB695A795979587952E
:10ECD000402F50E060E070E084179507A607B70763
:10ECE00089F40E942E6680E796E6DF91CF911F910E
:10ECF0000F91FF90EF90DF90BF90AF909F908F901B
:10ED00000C946B66FF24F394F00E40915B0D5091D0
:10ED10005C0D60915D0D70915E0D769567955795D0
:10ED200047958F2D90E0A0E0B0E0481759076A079B
:10ED30007B0788F08F2D90E0880F991F0197AA27F5
:10ED400097FDA095BA2F80935B0D90935C0DA093D7
:10ED50005D0DB0935E0D40915B0D50915C0D609127
:10ED60005D0D70915E0D76956795579547958091ED
:10ED7000640D90E00396242F30E0821793074CF443
:10ED80008DEF840F8093640DD0926F02DCEFD40F6F
:10ED9000CFEFCF5FDF5FC43008F4F8CCDF91CF91C5
:10EDA0001F910F91FF90EF90DF90BF90AF909F90D9
:10EDB0008F90089576956795579547952EE7413042
:10EDC00051056105710511F44EE301C040E26BEDA0
:10EDD00071E18C2F0E94076558CD80915B0D909159
:10EDE0005C0DA0915D0DB0915E0DB695A7959795C0
:10EDF00087950197A105B10509F049CD0E942E66BE
:10EE000086EA9DE672CF2091B20D211108C044E13F
:10EE100050E0BC0182E792E00E949CB934CC089596
:10EE2000F2DF81E08093B20D0C94A7691092B20DCD
:10EE30000895CF92DF92EF92FF92CF93CCB1C0951D
:10EE4000CC1FCC27CC1F8091030183FFC260C090F0
:10EE5000600DD090610DE090620DF090630D0E9406
:10EE60000EADC616D706E806F90610F4489B39C061
:10EE7000C093650D8091650D81709091650D91FD38
:10EE8000826090915F0D891721F18130F1F028F0B7
:10EE9000823089F08330A1F01CC0913021F4909130
:10EEA000C80D9F5F05C09230A1F49091C80D91509C
:10EEB0009093C80D0EC0992391F3933051F4F5CF80
:10EEC000923069F3913029F4F0CF933041F39923D4
:10EED00061F380935F0DCF91FF90EF90DF90CF9023
:10EEE0000895C460C5CF0E949B696F98E4E0F1E08B
:10EEF0008081877F8083779A9FB7F894E5E0F1E07F
:10EF00008081886080839FBF5098589A60E088E431
:10EF10000E942EAC9FB7F894E5E0F1E08081846018
:10EF200080839FBF8091030182FB882780F991E055
:10EF3000892780935A0D7DDF1092C80D0895CF92D6
:10EF4000DF92EF92FF9275DF8091030191E082FBE7
:10EF5000882780F9892720915A0D8217C9F082E00D
:10EF600080936F028091030182FB882780F98927B3
:10EF700080935A0D0E949B6980915A0D882309F451
:10EF80009EC083E89AE00E94D9308AEC9EE03BDF85
:10EF9000C090560DD090570DE090580DF090590D3F
:10EFA0000E940EADC616D706E806F90608F094C012
:10EFB0008091C80D482F552747FD509557FF03C036
:10EFC0005195419551094230510584F191E090935A
:10EFD0006F0287FD8F5F482F4595552747FD509558
:10EFE000652F752F80915B0D90915C0DA0915D0D4B
:10EFF000B0915E0D840F951FA61FB71F80935B0D08
:10F0000090935C0DA0935D0DB0935E0D1092C80DB2
:10F010000E940EAD6856754C8F4F9F4F60932B0D1D
:10F0200070932C0D80932D0D90932E0D8091650D76
:10F0300082FF0EC00E940EAD6856754C8F4F9F4FD9
:10F0400060932B0D70932C0D80932D0D90932E0DAE
:10F05000E0917002F09171021995C0902B0DD09043
:10F060002C0DE0902D0DF0902E0D0E940EADC616C9
:10F07000D706E806F90638F4809170029091710283
:10F080008F59934819F580916F02823011F40E94D4
:10F09000BC6980916F02882319F0815080936F02C0
:10F0A0000E940EAD6C597F4F8F4F9F4F6093560D4E
:10F0B0007093570D8093580D9093590D0DC083E8B0
:10F0C0009AE00E94A4318DEB9EE061CF0E94A76977
:10F0D00082E080936F02D7CFFF90EF90DF90CF90C8
:10F0E000089581E008958091650D82FB882780F95D
:10F0F00008950F931F93CF93DF930E94BC6940E064
:10F1000060E086E69DE00E94F02862E775E086E612
:10F110009DE00E949BB141E061E086E69DE00E9497
:10F12000F02865E875E086E69DE00E949BB142E02C
:10F1300061E086E69DE00E94F02869E875E086E6D9
:10F140009DE00E949BB143E061E086E69DE00E9465
:10F15000F0286DE975E086E69DE00E949BB141E0F4
:10F1600060E086E69DE00E94F0286DEA75E086E6A4
:10F170009DE00E949BB10091C80D112707FD1095DD
:10F18000C1E0D0E08091750A9091760A892B09F050
:10F1900071C00E94E41E81E00E94574A2091C80D70
:10F1A000332727FD3095C801821B930B97FF03C0BF
:10F1B00091958195910905970CF44DC02017310761
:10F1C0000CF42197021713070CF42196C430D105D3
:10F1D0002CF4209729F4C1E0D0E002C0C3E0D0E0D5
:10F1E00041E060E086E69DE00E94F0286DE973E072
:10F1F00086E69DE00E949BB142E060E086E69DE0ED
:10F200000E94F0286DE973E086E69DE00E949BB1C4
:10F2100043E060E086E69DE00E94F0286DE973E03F
:10F2200086E69DE00E949BB14C2F60E086E69DE063
:10F230000E94F0286DEA75E086E69DE00E949BB191
:10F240000091C80D112707FD109564E670E080E07D
:10F2500090E00E943DAD47DF882309F493CFD0931F
:10F26000760AC093750A64EF71E080E090E00E9436
:10F270003DAD88CF0E94BC69DF91CF911F910F9166
:10F280000C94A7690F931F93CF93DF930E94BC69DF
:10F2900040E060E086E69DE00E94F0286FEA75E0BD
:10F2A00086E69DE00E949BB141E061E086E69DE03C
:10F2B0000E94F02865E875E086E69DE00E949BB11B
:10F2C00042E061E086E69DE00E94F0286FEB75E089
:10F2D00086E69DE00E949BB141E060E086E69DE00D
:10F2E0000E94F0286DEA75E086E69DE00E949BB1E1
:10F2F0000091C80D112707FD1095C1E0D0E00E94D4
:10F30000E41E81E00E94574A2091C80D332727FD53
:10F310003095C801821B930B97FF03C0919581958F
:10F32000910905970CF441C0201731070CF421977F
:10F33000021713070CF42196C330D1052CF4209743
:10F3400029F4C1E0D0E002C0C2E0D0E041E060E0DA
:10F3500086E69DE00E94F0286DE973E086E69DE078
:10F360000E949BB142E060E086E69DE00E94F028AA
:10F370006DE973E086E69DE00E949BB14C2F60E052
:10F3800086E69DE00E94F0286DEA75E086E69DE045
:10F390000E949BB10091C80D112707FD109564E6EE
:10F3A00070E080E090E00E943DAD9DDE882309F48E
:10F3B000A6CF2197D9F462EC7DE08DEF9FE00E940B
:10F3C000977064EC7DE08BEF9FE00E94977066EC95
:10F3D0007DE089EF9FE00E9497708091C60D90912B
:10F3E000C70D90935808809357081EC01092C30D04
:10F3F0001092C20D1092C50D1092C40D1092C70D3F
:10F400001092C60D62EC7DE08DEF9FE00E94867049
:10F4100064EC7DE08BEF9FE00E94867066EC7DE0FF
:10F4200089EF9FE00E94867064EF71E080E090E0D9
:10F430000E943DAD0E94BC69DF91CF911F910F9159
:10F440000C94A769FC01808190E02AE030E0B901CA
:10F450000E9448B6482FCB01B9010E9448B6805D92
:10F4600080932F0D405D4093300D1092310D8FE24F
:10F470009DE0089520E030E040E251E4FC0160812D
:10F480007181828193810E9452B50E94ECB277FD16
:10F4900002C02BE201C02DE220932F0D9B0177FFCC
:10F4A00004C022273327261B370BC90168EE73E0FF
:10F4B0000E9448B6CB01EAE0F0E0BF010E9448B6E6
:10F4C000805D8093300DC90164E670E00E9448B60B
:10F4D000CB01BF010E9448B6805D8093310DC90108
:10F4E000BF010E9448B6282FCB01BF010E9448B639
:10F4F000805D8093320D8EE28093330D205D2093EA
:10F50000340D1092350D8FE29DE008958F929F92F9
:10F51000AF92BF92CF92DF92EF92FF92FC01808078
:10F520009180A280B38020E030E048EC52E4C50135
:10F53000B4010E9452B56B017C0120E030E0A901CA
:10F540000E9480B418161CF4C701B60103C0C7019D
:10F55000B60190580E94ECB26B017C0120E030E0D3
:10F56000A901C501B4010E947DB287FF12C08DE2DE
:10F5700080932F0DC701B60128EE33E040E050E044
:10F580000E947DB6CA01B9012AE030E040E050E0B7
:10F5900036C0C701B60120E137E240E050E00E94EA
:10F5A0007DB6AAE08A2E912CA12CB12CCA01B901FA
:10F5B000A50194010E947DB6662391F0605D609381
:10F5C0002F0DC701B60128EE33E040E050E00E9465
:10F5D0007DB6CA01B901A50194010E947DB613C090
:10F5E00080E280932F0DC701B60128EE33E040E0A2
:10F5F00050E00E947DB6CA01B901A50194010E94A4
:10F600007DB6662311F0605D01C060E26093300D4D
:10F61000C701B60124E630E040E050E00E947DB62C
:10F62000FAE08F2E912CA12CB12CCA01B901A501B1
:10F6300094010E947DB6605D6093310DC701B601F3
:10F64000A50194010E947DB6662381F0605D609300
:10F65000340DCA01B901A50194010E947DB6605D17
:10F660006093330D8EE28093320D15C0CA01B9014B
:10F67000A50194010E947DB6662329F0605D609328
:10F68000330D8EE203C080E28093330D8093320D00
:10F6900080E28093340D1092350D8FE29DE0FF9053
:10F6A000EF90DF90CF90BF90AF909F908F90089594
:10F6B000FC012081318137FF07C08DE280932F0D3F
:10F6C00031952195310914C02436310574F0C901F2
:10F6D00064E670E00E9448B6CB016AE070E00E94E8
:10F6E00048B6805D80932F0D06C080E280932F0D79
:10F6F0002A30310564F0EAE0F0E0C901BF010E9460
:10F7000048B6CB01BF010E9448B6805D01C080E2CF
:10F710008093300DC9016AE070E00E9448B6805DB8
:10F720008093310D1092320D8FE29DE00895CF92BB
:10F73000DF92EF92FF920F931F93CF93DF9360912D
:10F7400014027091150280911602909117020E9486
:10F750002F2860933F0D7093400D8093410D90933F
:10F76000420D6091100270911102809112029091ED
:10F7700013020E943B2860933B0D70933C0D8093D5
:10F780003D0D90933E0D80915B0D90915C0DA0918D
:10F790005D0DB0915E0D81309048A105B10540F03E
:10F7A00010925B0D10925C0D10925D0D10925E0D2B
:10F7B00080915B0D90915C0DA0915D0DB0915E0DFF
:10F7C000B695A795979587954091640D50E060E0B8
:10F7D00070E084179507A607B70710F48093640DAF
:10F7E000D091640D1091650D12FB112710F9C0E046
:10F7F000B7E0CB2ED12CE12CF12C01E040915B0D38
:10F8000050915C0D60915D0D70915E0DD11130C015
:10F8100080916F02882371F023E042305105610529
:10F82000710510F443E001C040E269E670E18C2FFD
:10F830000E940765112309F4D7C080915B0D909158
:10F840005C0DA0915D0DB0915E0D0297A105B10513
:10F8500008F0CAC00E942E6681E291E7DF91CF9145
:10F860001F910F91FF90EF90DF90CF900C94666600
:10F87000D130D1F580916F028823B9F076956795E4
:10F880005795479588E698E0413051056105710527
:10F8900021F40EDF9C014EE303C00ADF9C0140E22D
:10F8A00062E670E18C2F0E943E65112309F49CC032
:10F8B00080915B0D90915C0DA0915D0DB0915E0DFE
:10F8C000B695A795979587950197A105B10509F07C
:10F8D0008BC00E942E6620E031E040E050E068E6F8
:10F8E00078E08BE590E176C0D230D1F580916F025F
:10F8F0008823B9F0769567955795479586E698E001
:10F90000423051056105710521F4D2DE9C014EE3C0
:10F9100003C0CEDE9C0140E267E570E18C2F0E94BF
:10F920003E65112309F460C080915B0D90915C0DE0
:10F93000A0915D0DB0915E0DB695A79597958795B1
:10F940000297A105B10509F04FC00E942E6623E978
:10F9500030E040E050E066E678E083E590E13AC0D0
:10F96000D33009F041C080916F028823B9F07695B9
:10F970006795579547958EE49AE0433051056105A8
:10F98000710521F495DE9C014EE303C091DE9C01DC
:10F9900040E269E470E18C2F0E943E65112321F161
:10F9A00080915B0D90915C0DA0915D0DB0915E0D0D
:10F9B000B695A795979587950397A105B105A1F4ED
:10F9C0000E942E662FEF30E040E050E06EE47AE0D7
:10F9D0008FE390E1DF91CF911F910F91FF90EF9016
:10F9E000DF90CF900C94B56480915B0D90915C0D8D
:10F9F000A0915D0DB0915E0D0897A105B10540F095
:10FA0000C0925B0DD0925C0DE0925D0DF0925E0DA8
:10FA100040915B0D50915C0D60915D0D70915E0D9C
:10FA200076956795579547958091640D90E003967C
:10FA3000242F30E0821793074CF48DEF840F8093CE
:10FA4000640D00936F02DCEFD40FCFEFCF5FDF5F69
:10FA5000C43008F4D3CEDF91CF911F910F91FF9066
:10FA6000EF90DF90CF900895CF92DF92EF92FF92C8
:10FA70000F931F93CF93DF9341E06FEB7DE08FEF08
:10FA80009FE00E94FF7062EC7DE08DEF9FE00E949E
:10FA9000977064EC7DE08BEF9FE00E94977066ECBE
:10FAA0007DE089EF9FE00E94977080915B0D9091BF
:10FAB0005C0DA0915D0DB0915E0D81309048A10567
:10FAC000B10540F010925B0D10925C0D10925D0D2F
:10FAD00010925E0D80915B0D90915C0DA0915D0D7B
:10FAE000B0915E0DB695A795979587954091640D59
:10FAF00050E060E070E084179507A607B70710F4A0
:10FB00008093640DD091640D1091650D12FB112747
:10FB100010F9C0E0F1E1CF2ED12CE12CF12C01E065
:10FB200040915B0D50915C0D60915D0D70915E0D8B
:10FB3000D11130C080916F02882371F023E04230F0
:10FB400051056105710510F443E001C040E26BEA24
:10FB50007FE08C2F0E940765112309F4C3C18091B7
:10FB60005B0D90915C0DA0915D0DB0915E0D0297C3
:10FB7000A105B10508F0B6C10E942E6682E893E7A0
:10FB8000DF91CF911F910F91FF90EF90DF90CF9079
:10FB90000C946666D130D1F580916F028823B9F05C
:10FBA00076956795579547958DE592E041305105DB
:10FBB0006105710521F47CDD9C014EE303C078DD15
:10FBC0009C0140E265EA7FE08C2F0E943E65112394
:10FBD00009F488C180915B0D90915C0DA0915D0D41
:10FBE000B0915E0DB695A795979587950197A1055C
:10FBF000B10509F077C10E942E6627EE33E04AE096
:10FC000050E06DE572E08FE99FE03CC0D23009F032
:10FC100043C080916F028823B9F076956795579518
:10FC2000479588E698E0423051056105710521F459
:10FC30003FDD9C014EE303C03BDD9C0140E268E9EF
:10FC40007FE08C2F0E943E65112309F44BC1809107
:10FC50005B0D90915C0DA0915D0DB0915E0DB69520
:10FC6000A795979587950297A105B10509F03AC127
:10FC70000E942E6620E031E040E050E068E678E047
:10FC800081E99FE0DF91CF911F910F91FF90EF905D
:10FC9000DF90CF900C94B564D330D1F580916F0292
:10FCA0008823B9F0769567955795479586E698E04D
:10FCB000433051056105710521F4FADC9C014EE3E6
:10FCC00003C0F6DC9C0140E26DE87FE08C2F0E94CF
:10FCD0003E65112309F406C180915B0D90915C0D86
:10FCE000A0915D0DB0915E0DB695A79597958795FE
:10FCF0000397A105B10509F0F5C00E942E6623E91E
:10FD000030E040E050E066E678E089E89FE0BACF76
:10FD1000D430D1F580916F028823B9F0769567953C
:10FD2000579547958EE49AE0443051056105710579
:10FD300021F4BEDC9C014EE303C0BADC9C0140E22E
:10FD40006FE77FE08C2F0E943E65112309F4CAC043
:10FD500080915B0D90915C0DA0915D0DB0915E0D59
:10FD6000B695A795979587950497A105B10509F0D4
:10FD7000B9C00E942E662FEF30E040E050E06EE404
:10FD80007AE085E79FE07ECFD530D1F580916F0294
:10FD90008823B9F076956795579547958BE592E05E
:10FDA000453051056105710521F482DC9C014EE36B
:10FDB00003C07EDC9C0140E260E77FE08C2F0E9464
:10FDC0003E65112309F48EC080915B0D90915C0D0E
:10FDD000A0915D0DB0915E0DB695A795979587950D
:10FDE0000597A105B10509F07DC00E942E6627EE9A
:10FDF00033E04AE050E06BE572E08BE69FE042CFF3
:10FE0000D630C1F580916F02882391F07695679581
:10FE10005795479520E2463051056105710511F46B
:10FE20004EE301C040E26BE57FE08C2F0E94076546
:10FE3000112309F457C080915B0D90915C0DA09146
:10FE40005D0DB0915E0DB695A79597958795069730
:10FE5000A105B10509F046C00E942E6686E59FE027
:10FE6000DF91CF911F910F91FF90EF90DF90CF9096
:10FE70000C94523FD730B1F580916F02882391F0F6
:10FE800076956795579547952EE74730510561055B
:10FE9000710511F44EE301C040E268E47FE08C2F6D
:10FEA0000E9407651123F1F080915B0D90915C0D2C
:10FEB000A0915D0DB0915E0DB695A795979587952C
:10FEC0000797A105B10571F40E942E6680E393E8BF
:10FED000DF91CF911F910F91FF90EF90DF90CF9026
:10FEE0000C946B662091BF0D80915B0D90915C0D21
:10FEF000A0915D0DB0915E0D211136C0D83009F092
:10FF000048C020916F02222389F0B695A795979556
:10FF1000879520E20897A105B10511F44EE301C0D1
:10FF200040E266E37FE08C2F0E940765112389F190
:10FF300080915B0D90915C0DA0915D0DB0915E0D77
:10FF4000B695A795979587950897A105B10509F5E9
:10FF50000E942E66DF91CF911F910F91FF90EF903D
:10FF6000DF90CF900C94E770D83099F420916F0215
:10FF70002223E1F2B695A7959795879520E20897F9
:10FF8000A105B10511F44EE301C040E264E27FE057
:10FF9000CACF80915B0D90915C0DA0915D0DB091E9
:10FFA0005E0D4297A105B10540F0C0925B0DD09265
:10FFB0005C0DE0925D0DF0925E0D40915B0D5091F5
:10FFC0005C0D60915D0D70915E0D7695679557950E
:10FFD00047958091640D90E00396242F30E08217BE
:10FFE00093074CF48DEF840F8093640D00936F02A0
:10FFF000DCEFD40FCFEFCF5FDF5FC43008F490CDDC
:020000021000EC
:10000000DF91CF911F910F91FF90EF90DF90CF90F4
:100010000895FC01808191818436910524F164E684
:1000200070E00E9448B6CB012AE030E0B9010E949E
:1000300048B6805D80932F0D80819181B9010E9427
:1000400048B6CB01B9010E9448B6805D8093300D5F
:1000500080819181B9010E9448B6805D8093310D05
:100060001092320D23C08A309105BCF02AE030E0B6
:10007000B9010E9448B6CB01B9010E9448B6805D23
:1000800080932F0D80819181B9010E9448B6805DD7
:100090008093300D1092310D09C06AE070E00E942B
:1000A00048B6805D80932F0D1092300D8FE29DE059
:1000B00008958F929F92AF92BF92CF92DF92EF926C
:1000C000FF92CF9320E030E040E251E4FC016081F8
:1000D0007181828193810E9452B50E94ECB297FD9A
:1000E00002C02BE201C02DE220932F0D6B017C0199
:1000F00097FF08C0F094E094D094C094C11CD11C28
:10010000E11CF11CC701B60120E137E240E050E0FC
:100110000E947DB69AE0892E912CA12CB12CCA01A7
:10012000B901A50194010E947DB6605D6093300D18
:10013000C701B60128EE33E040E050E00E947DB6F2
:10014000CA01B901A50194010E947DB6605D60936A
:10015000310DC701B60124E630E040E050E00E94D6
:100160007DB6CA01B901A50194010E947DB6605D0A
:100170006093320DC701B601A50194010E947DB6BE
:10018000C62FCA01B901A50194010E947DB6605D28
:100190006093330D8EE28093340DC05DC093350DB6
:1001A0001092360D8FE29DE0CF91FF90EF90DF909F
:1001B000CF90BF90AF909F908F900895CF92EF9285
:1001C0000F937FE1C72EE0E2EE2E0FE02EE045E038
:1001D00066E286E69DE00E94DB290F91EF90CF90CA
:1001E0000895CF93DF93FC016491EC01219666237F
:1001F00031F086E69DE00E94C82ACE01F4CFDF915F
:10020000CF9108950F931F93CF93DF938C01EB0150
:1002100041E061E086E69DE00E94F028C801E1DF50
:100220006AE386E69DE00E949CB1FE0101900020F9
:10023000E9F76C2F6E1B6C5E41E086E69DE00E9444
:10024000F028BE0186E69DE0DF91CF911F910F91CE
:100250000C949BB1CF92DF92EF92FF920F931F937A
:1002600080915B0D90915C0DA0915D0DB0915E0D44
:100270000097A105B10509F442C0BC01882777FDAC
:100280008095982F0E941FB32091370D3091380D23
:100290004091390D50913A0D0E9452B59B01AC012D
:1002A0006091700A7091710A8091720A9091730A3C
:1002B0000E94A4B16093700A7093710A8093720ACD
:1002C0009093730A10925B0D10925C0D10925D0D6D
:1002D00010925E0DF0E5CF2EFAE0DF2EE12CF12C2E
:1002E00000E81FE320E73AE04CE65AE068E67AE0EF
:1002F00084E69AE00E94549E81E080936F02809190
:100300006F02882339F080E79AE0B4D8BC0188E70F
:1003100090E178DF8091650D82FF0EC021E040E022
:1003200050E0BA0182E098E61F910F91FF90EF90A4
:10033000DF90CF900C9450661F910F91FF90EF903B
:10034000DF90CF900895CF93DF931F921F92CDB788
:10035000DEB780915B0D90915C0DA0915D0DB09129
:100360005E0DB7FF08C010925B0D10925C0D1092ED
:100370005D0D10925E0D8091430D9091440DA09102
:10038000450DB091460D40915B0D50915C0D609113
:100390005D0D70915E0D84179507A607B70744F4AD
:1003A00080935B0D90935C0DA0935D0DB0935E0DFB
:1003B00080916F028823A9F08091470D9091480D9C
:1003C00020915B0D30915C0D820F931F9A8389837E
:1003D000CE0101966DD9BC0180914D0D90914E0DCD
:1003E00011DF8091650D82FF1DC0E0914B0DF091F2
:1003F0004C0D8091470D9091480D20915B0D3091EF
:100400005C0D820F931F9183808340914F0D50911B
:10041000500D60E070E021E08091510D9091520DFF
:100420000E9450660F900F90DF91CF9108954F92E8
:100430005F926F927F928F929F92AF92BF92CF9274
:10044000DF92EF92FF920F931F93CF93DF934C01B4
:100450005B017A0180915B0D90915C0DA0915D0D27
:10046000B0915E0D892B8A2B8B2B09F47BC00E94E7
:100470007E41E501CC0FDD1FCC0FDD1F8E010C5935
:10048000154F60915B0D70915C0D882777FD80950D
:10049000982F0E941FB32091370D3091380D409155
:1004A000390D50913A0D0E9452B5F80120813181E9
:1004B000428153810E94A4B12B013C0120E030E035
:1004C000A9010E947DB2F80187FD05C040825182DA
:1004D0006282738204C01082118212821382B70179
:1004E000882777FD8095982F0E941FB36B017C01B0
:1004F0008E010C59154F9B01AC01F801608171818F
:10050000828193810E9480B418162CF4F801C08275
:10051000D182E282F38210925B0D10925C0D1092F8
:100520005D0D10925E0DCA53DA4F20E030E040E7D7
:1005300052E4688179818A819B810E9484B2C0E5FE
:10054000CC2ECAE0DC2E7B018C0120E73AE04CE6A1
:100550005AE068E67AE084E69AE00E94549E81E0E0
:1005600080936F0280916F02882361F0C501880F2C
:10057000991F880F991F8C59954F0E943A7ABC0198
:10058000C40140DE8091650D82FF18C021E040E08B
:1005900050E0BA0182E098E6DF91CF911F910F9170
:1005A000FF90EF90DF90CF90BF90AF909F908F9093
:1005B0007F906F905F904F900C945066DF91CF9139
:1005C0001F910F91FF90EF90DF90CF90BF90AF9071
:1005D0009F908F907F906F905F904F90089546ED21
:1005E00050E060E070E082E790E121CF46EC50E01F
:1005F00061E070E084E790E11ACF49EC50E062E0FE
:1006000070E086E790E113CF0F931F93CF93DF93B2
:100610008C01EB0141E060E086E69DE00E94F0285D
:10062000C801DFDD6AE386E69DE00E949CB1FE0121
:1006300001900020E9F7BE016E1B7F0B6B5E7F4FC0
:100640007695679543E086E69DE00E94F028BE011E
:1006500086E69DE0DF91CF911F910F910C949BB1A5
:10066000CF93DF9300D01F92CDB7DEB780915B0DA3
:1006700090915C0DA0915D0DB0915E0D0097A1056C
:10068000B105F9F02091570830915808280F391F0B
:1006900030935808209357082091C60D3091C70D0C
:1006A000280F391F3093C70D2093C60D10925B0D94
:1006B00010925C0D10925D0D10925E0D81E08093A2
:1006C0006F0280916F028823A9F06091C60D70912E
:1006D000C70D882777FD8095982F0E941FB36983E7
:1006E0007A838B839C83CE010196E3DCBC0188E195
:1006F0009FE08ADF8091650D82FF08C021E040E025
:1007000050E0BA0184E39DE70E94506662EC7DE010
:100710008DEF9FE00E94867064EC7DE08BEF9FE0A0
:100720000E94867066EC7DE089EF9FE00E948670F3
:100730000F900F900F900F90DF91CF9108958F92AF
:100740009F92AF92BF92CF92DF92EF92FF920F9360
:100750001F93CF93DF93CDB7DEB728970FB6F894EA
:10076000DEBF0FBECDBF8091550D882321F0815093
:100770008093550D03C081E080936F0280916F02DA
:10078000882309F459C28091C10D8F5F8093C10DF8
:100790008E3129F40E949B691092C10D0EC06AE04F
:1007A0000E9427B6911109C020E044E064E186E68A
:1007B0009DE00E94002A0E94916520E030E040E028
:1007C0005FE3609160087091610880916208909188
:1007D00063080E94A4B10E94ECB278876F83609195
:1007E000680870916908882777FD8095982F0E9486
:1007F0001FB320E030E040E05FE30E94A4B10E941C
:10080000ECB27E836D8340E060E086E69DE00E946E
:10081000F02862E086E69DE00E949CB1CE0107963A
:100820000E94587BBC0186E69DE00E949BB16FE26E
:1008300086E69DE00E949CB1CE010596EADBBC01F4
:1008400086E69DE00E949BB185E19FE0CADC6CE9F1
:1008500073E086E69DE00E949BB140E06AE086E698
:100860009DE00E94F02862EC75E086E69DE00E9423
:100870009BB12CEA35EC47E257E360916C0A70912A
:100880006D0A80916E0A90916F0A0E94A4B16983EB
:100890007A838B839C83CE0101960E94867ABC0169
:1008A00086E69DE00E949BB160E286E69DE00E94A4
:1008B0009CB141E060E086E69DE00E94F02820E0E7
:1008C00030E040E05FE360915A0870915B088091EE
:1008D0005C0890915D080E94A4B10E94ECB27887F8
:1008E0006F836091660870916708882777FD80950F
:1008F000982F0E941FB320E030E040E05FE30E94A9
:10090000A4B10E94ECB27E836D8360E086E69DE038
:100910000E949CB1CE0107960E94587BBC0186E6DE
:100920009DE00E949BB16FE286E69DE00E949CB133
:10093000CE0105966EDBBC0186E69DE00E949BB170
:1009400082E19FE04EDC6CE973E086E69DE00E9468
:100950009BB141E06AE086E69DE00E94F0286CE9E8
:1009600073E086E69DE00E949BB166E086E69DE02E
:100970000E949CB18DE592E00E94587BBC0186E606
:100980009DE00E949BB165E286E69DE00E949CB1DD
:1009900069E973E086E69DE00E949BB142E060E079
:1009A00086E69DE00E94F0288FE09FE01ADC8091AF
:1009B000850A8823A9F180916E0C882319F1809112
:1009C000180D9091190DA0911A0DB0911B0D009763
:1009D000A105B105B9F0BC01CD016D597F4F8F4F15
:1009E0009F4F24E630E040E050E00E945BB660910B
:1009F000200D7091210D8091220D9091230D0E9468
:100A00005BB601C020E030E03A832983CE01019635
:100A10000E94587BBC0186E69DE00E949BB103C00A
:100A20008BE09FE0DEDB65E286E69DE00E949CB104
:100A300068E973E086E69DE00E949BB142E06AE0CF
:100A400086E69DE00E94F0286CE973E086E69DE072
:100A50000E949BB167E086E69DE00E949CB1809178
:100A6000720890917308A0917408B0917508892B51
:100A70008A2B8B2BE1F10E940EAD20E6C22E2AEECE
:100A8000D22EE12CF12CA70196010E945BB6490100
:100A90005A01609172087091730880917408909166
:100AA0007508A70196010E945BB6C401821B930BD7
:100AB0006CE370E00E9434B6182F6983CE01019672
:100AC0000E94227ABC0186E69DE00E949BB16AE307
:100AD00086E69DE00E949CB11983CE0101960E949A
:100AE000227ABC0186E69DE00E949BB103C085E0AE
:100AF0009FE077DB6CE973E086E69DE00E949BB1A6
:100B000043E060E086E69DE00E94F0286AE873E03A
:100B100082E792E00E940BBA892B09F074C064E965
:100B20007AE08BE79DE00E940BBA892BD1F0EBE7CE
:100B3000FDE0DF010D900020E9F7AD0141505109C2
:100B40004B575D4060E070E0CF010E94DBB964E983
:100B50007AE08BE79DE00E9414BA1092B10D1092DA
:100B6000B00DE4E9FAE001900020E9F7E559FA4018
:100B7000759708F445C00091B00D1091B10DC12CCE
:100B8000D12C8091B00D9091B10D9801281B390B9B
:100B90002431310534F001969093B10D8093B00D5E
:100BA00038C0C114D104B9F7F801ED57F54F7F01F2
:100BB0009189602F681B43E0911115C086E69DE086
:100BC0000E94F028D70150966C9186E69DE00E9425
:100BD0009CB11092B10D1092B00D00E010E0CC2449
:100BE000C394D12CCECF86E69DE00E94F028F70179
:100BF000608986E69DE00E949CB10F5F1F4FC1CFC8
:100C00006BE77DE002C062E772E086E69DE00E944D
:100C10009BB102E712E0D8018D918D0180322CF456
:100C200060E286E69DE00E949CB1B2E006381B07B8
:100C300091F78AE08093550D8091650D82FB88279E
:100C400080F99091540D992399F09091530D992327
:100C500039F0811119C01092530D1092540D14C027
:100C6000882391F00E942E6681E08093530D0CC082
:100C7000882351F021E040E050E0BA0182E893E798
:100C80000E9450660E949B6980915D0290915E0275
:100C900020915B0D30915C0D8436910534F4820F08
:100CA000931F853691054CF416C08436910599F052
:100CB000820F931F8436910574F410925B0D10928D
:100CC0005C0D10925D0D10925E0D84E690E09093A5
:100CD0005E0280935D0220915D0230915E02809100
:100CE0005B0D90915C0D2436310569F48B309105D4
:100CF0001CF0865A9F4F09C0863FEFEF9E078CF489
:100D000082599F4F02C0820F931F90935E0280937F
:100D10005D0210925B0D10925C0D10925D0D1092B1
:100D20005E0D80915D0290915E028A3091051CF407
:100D30008AE090E005C0883E934034F087EE93E06F
:100D400090935E0280935D0228960FB6F894DEBF02
:100D50000FBECDBFDF91CF911F910F91FF90EF900C
:100D6000DF90CF90BF90AF909F908F900895CF93DA
:100D7000DF93C0EBDEE0FE018491882341F0909187
:100D8000C00095FFFCCF8093C6003196F5CFE8EE0A
:100D9000F4E18491882341F09091C00095FFFCCF4D
:100DA0008093C6003196F5CF8091C00085FFFCCFBF
:100DB0008AE08093C600FE018491E0EBFEE0882388
:100DC00049F09091C00095FFFCCF8093C60031960A
:100DD0008491F5CF4091CF135091D0136091D113EE
:100DE0007091D21380EE94E10E94BB3E4091D313E8
:100DF0005091D4136091D5137091D6138DED94E179
:100E00000E94BB3E4091D7135091D8136091D913E3
:100E10007091DA138AED94E10E94BB3E4091DB139E
:100E20005091DC136091DD137091DE1387ED94E136
:100E30000E94BB3E8091C00085FFFCCF8AE080937A
:100E4000C600FE018491E0EBFEE0882349F090911A
:100E5000C00095FFFCCF8093C60031968491F5CFFA
:100E6000EDEBF4E18491882341F09091C00095FF6F
:100E7000FCCF8093C6003196F5CF8091C00085FFEE
:100E8000FCCF8AE08093C600FE018491E0EBFEE097
:100E9000882349F09091C00095FFFCCF8093C60055
:100EA00031968491F5CF4091DF135091E01360911A
:100EB000E1137091E21384EB94E10E94BB3E4091F8
:100EC000E3135091E4136091E5137091E61381EB05
:100ED00094E10E94BB3E4091E7135091E81360916A
:100EE000E9137091EA138EEA94E10E94BB3E4091AF
:100EF000EB135091EC136091ED137091EE138BEAAC
:100F000094E10E94BB3E8091C00085FFFCCF8AE047
:100F10008093C600FE018491E0EBFEE0882349F057
:100F20009091C00095FFFCCF8093C60031968491CC
:100F3000F5CFEDE8F4E18491882341F09091C00071
:100F400095FFFCCF8093C6003196F5CF8091C0000D
:100F500085FFFCCF8AE08093C600FE018491E0EB20
:100F6000FEE0882349F09091C00095FFFCCF80936C
:100F7000C60031968491F5CF4091BF135091C013B4
:100F80006091C1137091C21384E894E10E94CD3E38
:100F90004091C3135091C4136091C5137091C6134F
:100FA00081E894E10E94CD3E4091C7135091C8134F
:100FB0006091C9137091CA138EE794E10E94CD3EEF
:100FC0004091CB135091CC136091CD137091CE13FF
:100FD0008BE794E10E94CD3E8091C00085FFFCCF5D
:100FE0008AE08093C600FE018491E0EBFEE0882356
:100FF00049F09091C00095FFFCCF8093C6003196D8
:101000008491F5CFE6E4F4E18491882341F0909156
:10101000C00095FFFCCF8093C6003196F5CF80913C
:10102000C00085FFFCCF8AE08093C600FE0184915A
:10103000E0EBFEE0882349F09091C00095FFFCCFE3
:101040008093C60031968491F5CF4091B7135091AB
:10105000B8136091B9137091BA138DE394E10E94B3
:10106000BB3E4091B3135091B4136091B51370918E
:10107000B6138AE394E10E94BB3E8091C00085FFD5
:10108000FCCF8AE08093C600FE018491E0EBFEE095
:10109000882349F09091C00095FFFCCF8093C60053
:1010A00031968491F5CFE7E8F3E18491882341F00C
:1010B0009091C00095FFFCCF8093C6003196F5CF8C
:1010C0008091C00085FFFCCF8AE08093C600FE01BE
:1010D0008491E0EBFEE0882349F09091C00095FFF9
:1010E000FCCF8093C60031968491F5CF4091BB131D
:1010F0005091BC136091BD137091BE138EE793E1C4
:101100000E94BB3E4091A3135091A4136091A5137C
:101110007091A6138BE793E10E94BB3E4091EF13C1
:101120005091F0136091F1137091F21388E793E1FD
:101130000E94CD3E4091AF135091B0136091B11316
:101140007091B21385E793E10E94BB3E4091AB13CF
:101150005091AC136091AD137091AE1382E793E19F
:101160000E94BB3E4091A7135091A8136091A91310
:101170007091AA138FE693E10E94BB3E8091C0005C
:1011800085FFFCCF8AE08093C600FE018491E0EBEE
:10119000FEE0882349F09091C00095FFFCCF80933A
:1011A000C60031968491F5CFEDE5F3E18491882373
:1011B00041F09091C00095FFFCCF8093C60031961E
:1011C000F5CF8091C00085FFFCCF8AE08093C600F8
:1011D000FE018491E0EBFEE0882349F09091C0008D
:1011E00095FFFCCF8093C60031968491F5CF409156
:1011F000580A5091590A60915A0A70915B0A84E525
:1012000093E10E94BB3E40915C0A50915D0A60915F
:101210005E0A70915F0A81E593E10E94BB3E4091B6
:10122000600A5091610A6091620A7091630A8EE4CB
:1012300093E10E94BB3E8091C00085FFFCCF8AE015
:101240008093C600FE018491E0EBFEE0882349F024
:101250009091C00095FFFCCF8093C6003196849199
:10126000F5CFE0E4F3E18491882341F09091C00050
:1012700095FFFCCF8093C6003196F5CF8091C000DA
:1012800085FFFCCF8AE08093C600FE018491E0EBED
:10129000FEE0882349F09091C00095FFFCCF809339
:1012A000C60031968491F5CF4091180250911902F1
:1012B00060911A0270911B0286E393E10E94BB3E8B
:1012C000609114027091150280911602909117029C
:1012D0000E942F28AB01BC0183E393E10E94BB3E37
:1012E000609110027091110280911202909113028C
:1012F0000E943B28AB01BC0180E393E10E94BB3E0E
:101300008091C00085FFFCCF8AE08093C600FE017B
:101310008491E0EBFEE0882349F09091C00095FFB6
:10132000FCCF8093C60031968491F5CFECEFF2E1CB
:101330008491882341F09091C00095FFFCCF809369
:10134000C6003196F5CF8091C00085FFFCCF8AE0C2
:101350008093C600FE018491E0EBFEE0882349F013
:101360009091C00095FFFCCF8093C6003196849188
:10137000F5CF409133025091340260913502709163
:10138000360282EF92E10E94BB3E20E030E040E76F
:1013900052E460912B0270912C0280912D02909169
:1013A0002E020E9452B5AB01BC018FEE92E10E9469
:1013B000BB3E4091480A5091490A60914A0A709197
:1013C0004B0A8CEE92E10E94BB3E8091C00085FFEB
:1013D000FCCF8AE08093C600FE018491E0EBFEE042
:1013E000882349F09091C00095FFFCCF8093C60000
:1013F00031968491F5CFE0ECF2E18491882341F0BD
:101400009091C00095FFFCCF8093C6003196F5CF38
:101410008091C00085FFFCCF8AE08093C600FE016A
:101420008491E0EBFEE0882349F09091C00095FFA5
:10143000FCCF8093C60031968491F5CF4091440A49
:101440005091450A6091460A7091470A86EB92E1F5
:101450000E94BB3E20E030E040E752E4609127026A
:10146000709128028091290290912A020E9452B51F
:10147000AB01BC0183EB92E10E94BB3E8091C000B6
:1014800085FFFCCF8AE08093C600FE018491E0EBEB
:10149000FEE0882349F09091C00095FFFCCF809337
:1014A000C60031968491F5CFE9E5F2E18491882375
:1014B00041F09091C00095FFFCCF8093C60031961B
:1014C000F5CF8091C00085FFFCCF8AE08093C600F5
:1014D000FE018491E0EBFEE0882349F09091C0008A
:1014E00095FFFCCF8093C60031968491F5CF409153
:1014F0004D0A50E060E070E08FE492E10E94CD3E42
:101500008091C00085FFFCCF8AE08093C600FE0179
:101510008491E0EBFEE0882349F09091C00095FFB4
:10152000FCCF8093C60031968491F5CF8091740AE8
:101530008823A1F1ECE3F2E18491882341F09091BA
:10154000C00095FFFCCF8093C6003196F5CF809107
:10155000C00085FFFCCF8AE08093C600FE01C491E5
:10156000E0EBFEE0CC2349F08091C00085FFFCCF8A
:10157000C093C6003196C491F5CF4091530250916B
:101580005402609155027091560282E392E10E94EA
:10159000BB3E8091C00085FFFCCF11C0E6E1F2E1C7
:1015A0008491882341F09091C00095FFFCCF8093F7
:1015B000C6003196F5CF8091C00085FFFCCF8AE050
:1015C0008093C600DF91CF910895AF92BF92CF92E2
:1015D000DF92EF92FF920F931F93CF93DF93CDB7DC
:1015E000DEB7E0970FB6F894DEBF0FBECDBF80E147
:1015F000EBEFF2E0DE01919601900D928A95E1F712
:1016000080E1EBE0F3E0DE01519601900D928A95C6
:10161000E1F780E1EBE1F3E0DE01119601900D923C
:101620008A95E1F76E0181E2C80ED11C8FECE82E9D
:1016300083E1F82E8E010F5E1F4F6FED73E1AE0157
:101640004F5F5F4F9FEBA92E93E1B92E20E030E072
:10165000F60181919191A191B1916F01F70181936F
:101660009193A193B1937F01F80181919191A191FF
:10167000B1918F01FB0181939193A193B193BF012C
:10168000FA0181919191A191B191AF01F5018193FD
:101690009193A193B1935F012F5F3F4F24303105A8
:1016A000B9F60E94EDA880E090E8ABE3B5E4809342
:1016B000B7139093B813A093B913B093BA13809350
:1016C000B3139093B413A093B513B093B6131092C1
:1016D000BB131092BC131092BD131092BE1380E284
:1016E0009EE4A0E0B0E08093EF139093F013A093FA
:1016F000F113B093F2131092A3131092A41310924B
:10170000A5131092A61380E090E0A0EAB1E48093C4
:10171000AF139093B013A093B113B093B2138DECA9
:101720009CECACECBEE38093AB139093AC13A09312
:10173000AD13B093AE1380E090E0A0EAB0E48093E4
:10174000A7139093A813A093A913B093AA13109270
:10175000600A1092610A1092620A1092630A109253
:101760005C0A10925D0A10925E0A10925F0A109253
:10177000580A1092590A10925A0A10925B0A82ED86
:1017800090E09093BE0D8093BD0D82E390E0909326
:10179000BC0D8093BB0D1092BA0D1092B90D8FEF56
:1017A00090E09093B80D8093B70D84E690E090930D
:1017B000B60D8093B50D1092B40D1092B30D83E366
:1017C00093EBA3E2B2E48093180290931902A093E2
:1017D0001A02B0931B0260E070E08CE990E40E9472
:1017E0002928609314027093150280931602909337
:1017F000170265E87BE28CEA92E40E943528609348
:1018000010027093110280931202909313020E94AF
:10181000971E80E090E0A0E8BFE380930C029093D5
:101820000D02A0930E02B0930F0210924D0A80E0B9
:1018300090E0A0E4B0E48093330290933402A0934C
:101840003502B093360240E050E064E372E4409326
:101850002B0250932C0260932D0270932E02109253
:10186000480A1092490A10924A0A10924B0A1092A2
:10187000440A1092450A1092460A1092470A40E024
:1018800050E060E071E44093270250932802609397
:10189000290270932A021092740A80935302909343
:1018A0005402A0935502B09356020E94C64BE0EB3F
:1018B000FEE08491882341F09091C00095FFFCCF19
:1018C0008093C6003196F5CFE4EFF1E1849188234F
:1018D00041F09091C00095FFFCCF8093C6003196F7
:1018E000F5CF8091C00085FFFCCF8AE08093C600D1
:1018F000E0960FB6F894DEBF0FBECDBFDF91CF915B
:101900001F910F91FF90EF90DF90CF90BF90AF901D
:1019100008951F920F920FB60F9211240BB60F92DB
:101920002F933F934F935F936F938F939F93EF9377
:10193000FF936091C60020914A0E30914B0EC90171
:1019400001968F77992740914C0E50914D0E841738
:10195000950741F0F901E653F24F608390934B0EE7
:1019600080934A0EFF91EF919F918F916F915F91BC
:101970004F913F912F910F900BBE0F900FBE0F9084
:101980001F9018959A01AB01211581EE380741058A
:10199000510549F182E08093C00060E079E08DE379
:1019A00090E00E947DB62150310941095109CA01D8
:1019B000B90122E030E040E050E00E947DB6309373
:1019C000C5002093C4008091C10080618093C10054
:1019D0008091C10088608093C1008091C1008068BF
:1019E0008093C10008951092C00020E130E0E7CF5D
:1019F00020914C0E30914D0E80914A0E90914B0EDD
:101A00008217930771F0F901E653F24F80812F5F3F
:101A10003F4F2F77332730934D0E20934C0E90E09D
:101A200008958FEF9FEF089580914C0E90914D0E89
:101A300090934B0E80934A0E08954F925F926F924F
:101A40007F928F929F92AF92BF92CF92DF92EF924E
:101A5000FF920F931F93CF93DF93CDB7DEB7A0977D
:101A60000FB6F894DEBF0FBECDBF5C014115510526
:101A700061057105E9F420E030E040E350E060E00A
:101A800070E0A0960FB6F894DEBF0FBECDBFDF9119
:101A9000CF911F910F91FF90EF90DF90CF90BF906B
:101AA000AF909F908F907F906F905F904F905BC0B2
:101AB0008E010F5F1F4FC12CD12C76014801422EA1
:101AC000512C612C712C8FEFC81AD80AE80AF80A39
:101AD000CB01BA01A30192010E945BB6CA01F801D1
:101AE00061938F01A901BC01411551056105710583
:101AF00051F7F1E0CF1AD108E108F108F401EC0D3B
:101B0000FD1D80818A3010F440E301C047E3480F97
:101B1000552747FD5095652F752F20E030E0C50112
:101B200022D081E0C81AD108E108F108EFEFCE1603
:101B3000DE06EE06FE0611F7A0960FB6F894DEBF9D
:101B40000FBECDBFDF91CF911F910F91FF90EF900E
:101B5000DF90CF90BF90AF909F908F907F906F90CD
:101B60005F904F9008952115310539F48091C000A0
:101B700085FFFCCF4093C60008952A30310509F453
:101B800024C05BCF9A01462F552747FD5095652FFE
:101B9000752FE9CFCF93DF93EC0120E030E04DE0EB
:101BA00050E060E070E0DFDF20E030E04AE050E04D
:101BB00060E070E0CE01DF91CF91D5CF9A01AB010B
:101BC000662757FD6095762FCECFCF92DF92EF92AA
:101BD000FF92CF93DF93EC016A017B0177FF0FC087
:101BE00020E030E04DE250E060E070E0BCDFF094D7
:101BF000E094D094C094C11CD11CE11CF11C2AE0DB
:101C0000B701A601CE01DF91CF91FF90EF90DF9059
